:04070000DFEFF0F047
:08070800046ED8CF05F0E0CF2C
:1007100006F00001E9CF0CF0EACF07F0E1CF08F0D6
:10072000E2CF09F0D9CF0AF0DACF0BF0F3CF12F015
:10073000F4CF13F0FACF14F0F5CF15F0F6CF16F092
:10074000F7CF17F0F8CF18F0FBCF19F000C00EF07C
:1007500001C00FF002C010F003C011F09DAAB4EF69
:1007600003F09EBA87EF1EF0F2AABAEF03F0F2B4DC
:10077000F2EF1BF0A3AAC0EF03F0A4BAE6EF1EF05D
:100780009DA0C6EF03F09EB0E5EF1AF0F0AACCEF03
:1007900003F0F0B4BEEF1AF0F0A8D2EF03F0F0B21D
:1007A0009CEF1AF0F0A6D8EF03F0F0B0ADEF1AF01E
:1007B000F2A8DEEF03F0F2B28BEF1AF0A0A2E4EFA2
:1007C00003F0A1B2F4EF1CF00EC000F00FC001F076
:1007D00010C002F011C003F00CC0E9FF07C0EAFF2F
:1007E000078E08C0E1FF09C0E2FF0AC0D9FF0BC0B5
:1007F000DAFF12C0F3FF13C0F4FF14C0FAFF15C0F4
:10080000F5FF16C0F6FF17C0F7FF18C0F8FF19C0B4
:10081000FBFF045006C0E0FF05C0D8FF1000F76AD8
:10082000320FF66E080EF722000EF86E0900F55032
:100830001200280C0106F76A4A0FF66E080EF7221E
:10084000000EF86E0900F5501200536F6E792045C6
:1008500056492D4433302020202020202000F76AE4
:10086000720FF66E080EF722000EF86E0900F550B2
:100870001200536F6E79204556492D4433302F4472
:10088000333120202000F76A9A0FF66E080EF72207
:10089000000EF86E0900F550120056616464696F2D
:1008A000204164642D612D43616D20202000F76A92
:1008B000C20FF66E080EF722000EF86E0900F55012
:1008C0001200536F6E79204556492D443130302047
:1008D000202020202000F76AEA0FF66E080EF7228B
:1008E000000EF86E0900F5501200536F6E79204526
:1008F00056492D4437302020202020202000F76A40
:10090000120FF66E090EF722000EF86E0900F55070
:100910001200536F6E79204252432D333030202025
:10092000202020202000F76A3A0FF66E090EF722E9
:10093000000EF86E0900F5501200536F6E792042D8
:1009400052432D4837303020202020202000F76AE5
:10095000620FF66E090EF722000EF86E0900F550D0
:100960001200536F6E79204252432D5A3730302097
:10097000202020202000F76A8A0FF66E090EF72249
:10098000000EF86E0900F5501200536F6E79204288
:1009900052432D5A33333020202020202000F76A84
:1009A000B20FF66E090EF722000EF86E0900F55030
:1009B0001200536F6E79204556492D48443120204E
:1009C000202020202000F76ADA0FF66E090EF722A9
:1009D000000EF86E0900F550120056414444494F8C
:1009E0002052455645414C2048442D313800F76A85
:1009F000020FF66E0A0EF722000EF86E0900F5508F
:100A000012004365696C696E675649455720484432
:100A10002D3138202000F76A2A0FF66E0A0EF722D1
:100A2000000EF86E0900F550120056414444494F3B
:100A30002048442D32302020202020202000F76A3A
:100A4000520FF66E0A0EF722000EF86E0900F550EE
:100A5000120056414444494F2048442D313920204A
:100A6000202020202000F76A7A0FF66E0A0EF72267
:100A7000000EF86E0900F550120056414444494FEB
:100A80002048442D31382020202020202000F76AE3
:100A9000A20FF66E0A0EF722000EF86E0900F5504E
:100AA000120056616464696F204365696C696E6702
:100AB000564945572000F76ACA0FF66E0A0EF7220C
:100AC000000EF86E0900F550120043616E6E6F6EF5
:100AD0002056432D43353069202020202000F76A1E
:100AE000F20FF66E0A0EF722000EF86E0900F550AE
:100AF000120050616E61736F6E696320484531303A
:100B0000302020202000F76A1A0FF66E0B0EF72215
:100B1000000EF86E0900F55012004E6F7420466FFB
:100B2000756E642020202020202020202000F76ADD
:100B3000420FF66E0B0EF722000EF86E0900F5500C
:100B4000120054696C7420446972656374696F6E35
:100B50003A20496E766572740000F76A6E0FF66E81
:100B60000B0EF722000EF86E0900F55012005469C2
:100B70006C7420446972656374696F6E3A204E6FBD
:100B8000726D616C0000F76A9A0FF66E0B0EF72219
:100B9000000EF86E0900F55012005A6F6F6D204478
:100BA0006972656374696F6E3A20496E7665727416
:100BB0000000F76AC60FF66E0B0EF722000EF86EF5
:100BC0000900F55012005A6F6F6D20446972656319
:100BD00074696F6E3A204E6F726D616C0000F76A37
:100BE000F20FF66E0B0EF722000EF86E0900F550AC
:100BF000120050616E20446972656374696F6E3AC9
:100C000020496E7665727400F76A1C0FF66E0C0E42
:100C1000F722000EF86E0900F550120050616E20A8
:100C2000446972656374696F6E3A204E6F726D61CC
:100C30006C00F76A460FF66E0C0EF722000EF86E87
:100C40000900F5501200486F737420536572696192
:100C50006C20496E7075743A20456E61626C6564F3
:100C60000000F76A760FF66E0C0EF722000EF86E93
:100C70000900F5501200486F737420536572696162
:100C80006C20496E7075743A2044697361626C65BA
:100C90006400F76AA60FF66E0C0EF722000EF86ECF
:100CA0000900F550120053657269616C2045636854
:100CB0006F3A20456E61626C65640000F76AD00F80
:100CC000F66E0C0EF722000EF86E0900F5501200B9
:100CD00053657269616C204563686F3A204469739B
:100CE00061626C656400F76AFA0FF66E0C0EF7220B
:100CF000000EF86E0900F5501200537769746368AE
:100D0000696E67204D6F64653A2053656C20466FAD
:100D10006C6C6F772045585420410000F76A300F03
:100D2000F66E0D0EF722000EF86E0900F550120057
:100D3000537769746368696E67204D6F64653A2004
:100D40004D616E75616C0000F76A5C0FF66E0D0EFA
:100D5000F722000EF86E0900F55012000000F76A45
:100D6000720FF66E0D0EF722000EF86E0900F550A8
:100D70001200537769746368696E67204D6F64650C
:100D80003A2053656C20466F6C6C6F772045585441
:100D900020420000F76AA80FF66E0D0EF722000E33
:100DA000F86E0900F55012004E6F7420466F756E94
:100DB0006400F76AC60FF66E0D0EF722000EF86E8D
:100DC0000900F5501200446961676E6F73746963BE
:100DD000204D6F64653A204F6E00F76AEE0FF66E95
:100DE0000D0EF722000EF86E0900F550120044694E
:100DF00061676E6F73746963204D6F64653A204F4D
:100E000066660000F76A180FF66E0E0EF722000EE7
:100E1000F86E0900F550120053657269616C204943
:100E20006E666F3A204F6E00F76A3C0FF66E0E0E3C
:100E3000F722000EF86E0900F55012005365726932
:100E4000616C20496E666F3A204F66660000F76A53
:100E5000620FF66E0E0EF722000EF86E0900F550C6
:100E600012004C434420446973706C61793A204FFE
:100E70006E00F76A860FF66E0E0EF722000EF86E01
:100E80000900F55012004C434420446973706C61B2
:100E9000793A204F66660000F76AAC0FF66E0E0EC8
:100EA000F722000EF86E0900F550120054616C6CC8
:100EB000792049646C65204C6576656C3A204869F8
:100EC00067680000F76AD80FF66E0E0EF722000E64
:100ED000F86E0900F550120054616C6C7920496479
:100EE0006C65204C6576656C3A204C6F7700F76A2C
:100EF000020FF66E0F0EF722000EF86E0900F55085
:100F00001200446973706C617920566964656F20C2
:100F100053656C65637465643A204368616E6E6501
:100F20006C204100F76A380FF66E0F0EF722000EA4
:100F3000F86E0900F5501200446973706C617920F5
:100F4000566964656F2053656C65637465643A2007
:100F50004368616E6E656C204200F76A6E0FF66E34
:100F60000F0EF722000EF86E0900F5501200202037
:100F70002053797374656D204D656E7520202000B7
:100F8000F76A940FF66E0F0EF722000EF86E090046
:100F9000F5501200202053657269616C20496E7013
:100FA000757420202000F76ABA0FF66E0F0EF72234
:100FB000000EF86E0900F55012002020536572698A
:100FC000616C204563686F2020202000F76AE00FE5
:100FD000F66E0F0EF722000EF86E0900F5501200A3
:100FE0002020436C656172204D656D6F7279202001
:100FF0002000F76A060FF66E100EF722000EF86E4C
:101000000900F55012002020436C65617220507277
:101010006573657473202000F76A2C0FF66E100E4E
:10102000F722000EF86E0900F55012002020205320
:10103000657269616C20496E666F20202000F76A36
:10104000520FF66E100EF722000EF86E0900F550E2
:1010500012002020506F7765722055702050726505
:1010600073657400F76A780FF66E100EF722000EA3
:10107000F86E0900F55012002020507265736574F7
:10108000204C6F636174696F6E00F76A9E0FF66E95
:10109000100EF722000EF86E0900F5501200202005
:1010A00052657475726E20746F204D61696E2000F8
:1010B000F76AC40FF66E100EF722000EF86E0900E4
:1010C000F550120020202050616E20446972204D9E
:1010D000656E75202000F76AEA0FF66E100EF72293
:1010E000000EF86E0900F55012002020202020414B
:1010F0006C6C20506F72747320202000F76A100F00
:10110000F66E110EF722000EF86E0900F55012006F
:10111000202020202020506F727420303120202089
:101120002000F76A360FF66E110EF722000EF86EE9
:101130000900F5501200202020202020506F7274EA
:101140002030322020202000F76A5C0FF66E110E4E
:10115000F722000EF86E0900F55012002020202022
:101160002020506F72742030332020202000F76A36
:10117000820FF66E110EF722000EF86E0900F55080
:101180001200202020202020506F72742030342044
:1011900020202000F76AA80FF66E110EF722000E2D
:1011A000F86E0900F5501200202020202020506FFA
:1011B00072742030352020202000F76ACE0FF66EA2
:1011C000110EF722000EF86E0900F55012002020D3
:1011D00020202020506F72742030362020202000E4
:1011E000F76AF40FF66E110EF722000EF86E090082
:1011F000F5501200202054696C7420446972204D0F
:10120000656E75202000F76A1A0FF66E120EF7222F
:10121000000EF86E0900F550120020202052657370
:1012200063616E2043616D6572617300F76A400F00
:10123000F66E120EF722000EF86E0900F55012003D
:101240002020205363616E2050616E61736F6E6960
:101250006300F76A660FF66E120EF722000EF86E44
:101260000900F550120020202044656661756C74F9
:101270002043616D65726100F76A8C0FF66E120E85
:10128000F722000EF86E0900F550120020202044CD
:10129000656661756C742050726573657400F76AD9
:1012A000B20FF66E120EF722000EF86E0900F5501E
:1012B000120020202050616E53656E736974697648
:1012C00069747900F76AD80FF66E120EF722000ED5
:1012D000F86E0900F5501200202054696C745365B3
:1012E0006E736974697669747900F76AFE0FF66E39
:1012F000120EF722000EF86E0900F55012002020A1
:1013000020202050616E20537065656420202000ED
:10131000F76A240FF66E130EF722000EF86E09001E
:10132000F550120020202020202053746172740098
:10133000F76A440FF66E130EF722000EF86E0900DE
:10134000F5501200202020202020204F666600004B
:10135000F76A640FF66E130EF722000EF86E09009E
:10136000F5501200202020202020204F6E20000069
:10137000F76A840FF66E130EF722000EF86E09005E
:10138000F55012002020202020204E6F726D616CDD
:101390000000F76AA60FF66E130EF722000EF86E25
:1013A0000900F5501200202020202020496E76658B
:1013B00072740000F76AC80FF66E130EF722000E63
:1013C000F86E0900F55012002020202020204E6FDA
:1013D0006E65202020200000F76AEC0FF66E130ED9
:1013E000F722000EF86E0900F55012002020202090
:1013F00020457874726F6E2020200000F76A100F6D
:10140000F66E140EF722000EF86E0900F550120069
:10141000202020416E616C6F6720576179200000A9
:10142000F76A340FF66E140EF722000EF86E0900FC
:10143000F55012002020456469726F6C2D34482CE1
:1014400032530000F76A580FF66E140EF722000EA2
:10145000F86E0900F55012002020456469726F6C27
:101460002D34532C32480000F76A7C0FF66E140EB0
:10147000F722000EF86E0900F55012002020456496
:1014800069726F6C2D33532C33480000F76AA00F3C
:10149000F66E140EF722000EF86E0900F5501200D9
:1014A000202020496E6E6F766174696F6E20000097
:1014B000F76AC40FF66E140EF722000EF86E0900DC
:1014C000F55012002020202020204F7468657220E3
:1014D00020200000F76AE80FF66E140EF722000EC7
:1014E000F86E0900F5501200202020202020204D09
:1014F000616E75616C00F76A0A0FF66E150EF722C1
:10150000000EF86E0900F550120020202020466FD2
:101510006C6C6F772045585420410000F76A300FFB
:10152000F66E150EF722000EF86E0900F550120047
:1015300020202020466F6C6C6F7720455854204245
:101540000000F76A560FF66E150EF722000EF86EC1
:101550000900F5501200202020416374697665204F
:10156000486967680000F76A7A0FF66E150EF72271
:10157000000EF86E0900F55012002020204163741F
:10158000697665204C6F77200000F76A9E0FF66E33
:10159000150EF722000EF86E0900F55012002020FB
:1015A00020202020205965730000F76ABE0FF66ED8
:1015B000150EF722000EF86E0900F55012002020DB
:1015C0002020202020204E6F0000F76ADE0FF66EEC
:1015D000150EF722000EF86E0900F55012002020BB
:1015E000202020486F6D652043616D657261200089
:1015F000F76A040FF66E160EF722000EF86E090059
:10160000F550120020202020205072657365742050
:10161000313220202000F76A2A0FF66E160EF722CC
:10162000000EF86E0900F550120020202020204105
:101630006C6C204C6F63616C20202000F76A500FA7
:10164000F66E160EF722000EF86E0900F550120025
:1016500020203620496E43616D2036204C6F636137
:101660006C00F76A760FF66E160EF722000EF86E13
:101670000900F5501200204E6F2043616D2020209C
:1016800020506F7274203000F76A9C0FF66E160EB1
:10169000F722000EF86E0900F5501200204845317F
:1016A00030302020202020506F7274203000F76AE4
:1016B000C20FF66E160EF722000EF86E0900F550F6
:1016C00012002056432D43353069202020506F7280
:1016D00074203000F76AE80FF66E160EF722000E3F
:1016E000F86E0900F5501200205620484431382089
:1016F000202020506F7274203000F76A0E0FF66EB3
:10170000170EF722000EF86E0900F5501200205651
:101710002052455645414C2020506F7274203000B5
:10172000F76A340FF66E170EF722000EF86E0900F6
:10173000F5501200205620435620484420202050C7
:101740006F7274203000F76A5A0FF66E170EF72288
:10175000000EF86E0900F550120020562048443261
:101760003020202020506F7274203000F76A800FE4
:10177000F66E170EF722000EF86E0900F5501200F3
:101780002056204844313920202020506F72742088
:101790003000F76AA60FF66E170EF722000EF86EED
:1017A0000900F55012002056414444494F3F3F2064
:1017B00020506F7274203000F76ACC0FF66E170E4F
:1017C000F722000EF86E0900F55012002045564928
:1017D0002D4433302F3331506F7274203000F76A4C
:1017E000F20FF66E170EF722000EF86E0900F55094
:1017F0001200204556492D443330202020506F726E
:1018000074203000F76A180FF66E180EF722000EDB
:10181000F86E0900F5501200204164642D412D43FB
:10182000616D20506F7274203000F76A3E0FF66EC3
:10183000180EF722000EF86E0900F5501200204530
:1018400056492D443130302020506F7274203000C2
:10185000F76A640FF66E180EF722000EF86E090094
:10186000F5501200204556492D4437302020205095
:101870006F7274203000F76A8A0FF66E180EF72226
:10188000000EF86E0900F550120020425243482D18
:101890003730302020506F7274203000F76AB00F5C
:1018A000F66E180EF722000EF86E0900F5501200C1
:1018B00020456C6D6F202020202020506F727420F6
:1018C0003000F76AD60FF66E180EF722000EF86E8B
:1018D0000900F5501200204252432D3330302020B1
:1018E00020506F7274203000F76AFC0FF66E180EED
:1018F000F722000EF86E0900F55012002042524304
:101900002D5A3730302020506F7274203000F76A23
:10191000220FF66E190EF722000EF86E0900F55030
:101920001200204252432D5A3333302020506F7220
:1019300074203000F76A480FF66E190EF722000E79
:10194000F86E0900F5501200204556492D484431E3
:10195000202020506F7274203000F76A6E0FF66EF0
:10196000190EF722000EF86E0900F5501200204300
:10197000562F43564D50202020506F727420300057
:10198000F76A940FF66E190EF722000EF86E090032
:10199000F550120020496E76616C69642043616DD8
:1019A00065726100F76AB80FF66E190EF722000E25
:1019B000F86E0900F5501200204556492D44333089
:1019C000287229506F7274203000F76ADE0FF66EAD
:1019D000190EF722000EF86E0900F55012002020B3
:1019E000202020202000F76AFA0FF66E190EF72249
:1019F000000EF86E0900F55012004F6E20202020D6
:101A000020200000F76A180FF66E1A0EF722000E5B
:101A1000F86E0900F55012004F6666202020202045
:101A20000000F76A360FF66E1A0EF722000EF86EF7
:101A30000900F55012004F6E202020200000F76AA8
:101A4000520FF66E1A0EF722000EF86E0900F550CE
:101A500012004F66662020200000F76A6E0FF66EB7
:101A60001A0EF722000EF86E0900F55012004F6EA4
:101A700020202000F76A880FF66E1A0EF722000E5B
:101A8000F86E0900F55012004F6666202000F76AD4
:101A9000A20FF66E1A0EF722000EF86E0900F5502E
:101AA00012004F6E0000F76ABA0FF66E1A0EF72298
:101AB000000EF86E0900F55012004F666600F76AD6
:101AC000D20FF66E1A0EF722000EF86E0900F550CE
:101AD00012002020204578742043544C20412030AF
:101AE00020202000F76AF80FF66E1A0EF722000E7B
:101AF000F86E0900F550120020202045787420432C
:101B0000544C2042203020202000F76A1E0FF66E31
:101B10001B0EF722000EF86E0900F550120020206F
:101B200020202043616D2053656C20302020200050
:101B3000F76A440FF66E1B0EF722000EF86E0900CE
:101B4000F55012002043616D2053656C2030204E0B
:101B50006F2043616D00F76A6A0FF66E1B0EF72265
:101B6000000EF86E0900F550120020496E20436106
:101B70006D2053746F72652030300000F76A900F4B
:101B8000F66E1B0EF722000EF86E0900F5501200DB
:101B9000202052656164696E672043616D657261E2
:101BA0000000F76AB60FF66E1B0EF722000EF86EF5
:101BB0000900F5501200202053746F72696E67207F
:101BC0005072657365740000F76ADC0FF66E1B0EC9
:101BD000F722000EF86E0900F55012002053746FC2
:101BE0007265203030205072657365740000F76AAA
:101BF000020FF66E1C0EF722000EF86E0900F5506B
:101C000012002053746F7265203030204661696C79
:101C100065640000F76A280FF66E1C0EF722000EAE
:101C2000F86E0900F550120020496E2043616D20C6
:101C3000507265736574203030200000F76A500FD1
:101C4000F66E1C0EF722000EF86E0900F550120019
:101C500020204C6F6164696E6720507265736574F3
:101C60000000F76A760FF66E1C0EF722000EF86E73
:101C70000900F55012002020205072657365742011
:101C80003030202020200000F76A9C0FF66E1C0EDA
:101C9000F722000EF86E0900F550120020202050A7
:101CA0007265736574203030204261640000F76A09
:101CB000C20FF66E1C0EF722000EF86E0900F550EA
:101CC00012002020204E6F20507265736574203002
:101CD00030200000F76AE80FF66E1C0EF722000EA7
:101CE000F86E0900F55012002020457874205669DE
:101CF00064656F2041204F6E0000F76A0E0FF66E8C
:101D00001D0EF722000EF86E0900F550120020207B
:101D100020446973706C6179204F66660000F76A31
:101D2000320FF66E1D0EF722000EF86E0900F55008
:101D30001200202045787420566964656F20422087
:101D40004F6E0000F76A580FF66E1D0EF722000E58
:101D5000F86E0900F5501200204261636B4C696710
:101D60006874436D70204F666600F76A7E0FF66EEA
:101D70001D0EF722000EF86E0900F55012002042E9
:101D800061636B4C69676874436D70204F6E20000F
:101D9000F76AA40FF66E1D0EF722000EF86E09000A
:101DA000F550120020424C43204E6F205375707046
:101DB0006F7274202000F76ACA0FF66E1D0EF722AC
:101DC000000EF86E0900F55012002020427269677B
:101DD00068746E657373205570202000F76AF00FE9
:101DE000F66E1D0EF722000EF86E0900F550120077
:101DF00020204272696768746E65737320446E2098
:101E00002000F76A160FF66E1E0EF722000EF86E0F
:101E10000900F550120020204272696768746E65EF
:101E20007373204175746F00F76A3C0FF66E1E0ED7
:101E3000F722000EF86E0900F550120020204272C1
:101E4000696768746E657373204D616E2000F76A70
:101E5000620FF66E1E0EF722000EF86E0900F550A6
:101E6000120020202020466F637573204E6561723A
:101E700020202000F76A880FF66E1E0EF722000E53
:101E8000F86E0900F550120020202020466F63757F
:101E900073204661722020200000F76AAE0FF66EB4
:101EA0001E0EF722000EF86E0900F55012002020D9
:101EB0002020466F637573204175746F20200000E9
:101EC000F76AD40FF66E1E0EF722000EF86E0900A8
:101ED000F550120020202020466F637573204D615D
:101EE0006E75616C0000F76AFA0FF66E1E0EF7222F
:101EF000000EF86E0900F5501200204175746F57FE
:101F00006869746542616C204F666600F76A200F4D
:101F1000F66E1F0EF722000EF86E0900F550120043
:101F2000204175746F576869746542616C204F6E0B
:101F30002000F76A460FF66E1F0EF722000EF86EAD
:101F40000900F550120020415742204E6F20537572
:101F500070706F7274202000F76A6C0FF66E1F0E9F
:101F6000F722000EF86E0900F5501200205072653D
:101F70007365742050474D204D6F64652000F76AEB
:101F8000920FF66E1F0EF722000EF86E0900F55044
:101F90001200204C6F6164696E6720507265736532
:101FA00074313200F76AB80FF66E1F0EF722000E7A
:101FB000F86E0900F5501200204E6F2050726573C4
:101FC0006574313220466F756E640000F76AE00F69
:101FD000F66E1F0EF722000EF86E0900F550120083
:101FE0000C50726F64756374696F6E5669657753D0
:101FF0004A00F76A060FF66E200EF722000EF86E02
:102000000900F55012000A00F76A1C0FF66E200E48
:10201000F722000EF86E0900F550120020205374CC
:10202000617274696E67205570202000F76A400F56
:10203000F66E200EF722000EF86E0900F550120021
:102040002046696E64696E672043616D65726173D5
:102050000000F76A660FF66E200EF722000EF86E8B
:102060000900F550120020436C656172696E6720AB
:102070005072657365747300F76A8C0FF66E200EEC
:10208000F722000EF86E0900F550120020436C652F
:102090006172696E6720416C6C2020200000F76A35
:1020A000B20FF66E200EF722000EF86E0900F55002
:1020B000120020204E6F74206F6E20507265736581
:1020C00074200000F76AD80FF66E200EF722000E7B
:1020D000F86E0900F5501200204C6F6164696E675C
:1020E0002044656661756C747300F76AFE0FF66EC6
:1020F000200EF722000EF86E0900F550120020465F
:10210000696E64696E6720457874726F6E00F76A55
:10211000220FF66E210EF722000EF86E0900F55020
:10212000120020466F756E64202020457874726F0F
:102130006E00F76A460FF66E210EF722000EF86E5B
:102140000900F550120020457874726F6E205761B7
:102150006974203330730000F76A6C0FF66E210E3D
:10216000F722000EF86E0900F55012002045787431
:10217000726F6E2057616974203230730000F76A05
:10218000920FF66E210EF722000EF86E0900F55040
:10219000120020457874726F6E2057616974203187
:1021A00030730000F76AB80FF66E210EF722000EAA
:1021B000F86E0900F550120020457874726F6E2099
:1021C0005265737461727400F76ADC0FF66E210E4B
:1021D000F722000EF86E0900F550120020457874C1
:1021E000726F6E204E6F7420466F756E6400F76AD2
:1021F000020FF66E220EF722000EF86E0900F5505F
:1022000012002046696E6420416E616C6F675761F1
:1022100079202000F76A280FF66E220EF722000EB2
:10222000F86E0900F550120020466F756E6420416B
:102230006E616C6F675761790000F76A4E0FF66E3A
:10224000220EF722000EF86E0900F5501200204110
:102250006E616C6F6757617920333020736563005E
:10226000F76A740FF66E220EF722000EF86E090060
:10227000F550120020416E616C6F67576179203212
:10228000302073656300F76A9A0FF66E220EF7220C
:10229000000EF86E0900F550120020416E616C6F5F
:1022A000675761792031302073656300F76AC00F8A
:1022B000F66E220EF722000EF86E0900F55012009D
:1022C00020416E616C6F675761792052657374723B
:1022D0007400F76AE60FF66E220EF722000EF86E13
:1022E0000900F550120020416E616C6F67576179EB
:1022F000204E6F46696E6400F76A0C0FF66E230E6F
:10230000F722000EF86E0900F55012002020506FE1
:10231000776572696E672055702020200000F76A8B
:10232000320FF66E230EF722000EF86E0900F550FC
:1023300012000A2020506F776572696E6720446F23
:10234000776E20004C6F6164205072657365742055
:102350006B3D254C58200A0D000052656164202514
:1023600032782025327820254C5820254C582025BD
:102370004C5820254C5820254C580A0D000053611C
:10238000766520507265736574206B3D254C58202E
:102390000A0D0000536176652025327820253278B9
:1023A00020254C5820254C5820254C5820254C5889
:1023B00020254C580A0D0000446F46696E64416345
:1023C000746976655072657365747320506F7274AA
:1023D000202564206261640A0D00506F727420250C
:1023E00064204550524F4D204C6F636174696F6E8D
:1023F00020254C580A0D0000536561726368696EB0
:102400006720666F7220417474616368656420435D
:10241000616D657261730D0A0000506F7274202542
:10242000643A2020000050616E61736F6E69632012
:1024300044657465637465640D0A000043616E6FE2
:102440006E2044657465637465640D0A00000D0AAE
:102450002057616974466565644261636B20546905
:102460006D656F7574203230303020286D73290D02
:102470000A000D0A2057616974466565644261630C
:102480006B2000000A0D2043616D65726154797004
:102490006520000054696D656F75740A0D20000099
:1024A0000D0A56414444494F2048442D31380D0A05
:1024B00000000D0A56414444494F205245564541BB
:1024C0004C2048442D31380D0A000D0A5641444431
:1024D000494F204365696C696E67564945572048E6
:1024E000442D31380D0A00000D0A56414444494F2D
:1024F0002048442D32300D0A00000D0A5641444454
:10250000494F2048442D31390D0A00000D0A556EFF
:102510006B6E6F776E2056414444494F0D0A0000A0
:102520000D0A536F6E79204556492D4433302F33B1
:1025300031200D0A00000D0A536F6E79204556496F
:102540002D4433300D0A00000D0A56616464696F32
:10255000204164642D412D43616D0D0A00000D0A78
:10256000536F6E79204556492D443130300D0A00A5
:102570000D0A536F6E79204556492D4437300D0AA8
:1025800000000D0A536F6E7920425243482D3730B8
:10259000300D0A000D0A456C6D6F2043616D657248
:1025A000610D0A000D0A536F6E79204252432D339C
:1025B00030300D0A00000D0A536F6E7920425243ED
:1025C0002D5A3730300D0A000D0A536F6E792042B4
:1025D00052432D5A3333300D0A000D0A536F6E7972
:1025E000204556492D4844310D0A00000D0A566118
:1025F0006464696F204365696C696E675649455725
:102600000D0A0000496E76616C69642043616D6556
:1026100072610D0A00000D0A536F6E79204556490C
:102620002D4433302872290D0A00496E76616C6999
:10263000642043616D6572610D0A000054696D6527
:102640006F75740A0D2000000A0D2041542F4D446F
:102650005F4D6F6465496E7120002054696D656F30
:1026600075740A0D20000D0A2057616974536F6E4E
:102670007941636B2054696D656F757420256C64B6
:1026800020286D73290D0A000D0A205761697453C3
:102690006F6E7941636B28256C64292000000D0A58
:1026A0002057616974536F6E792054696D656F7539
:1026B0007420256C6420286D73290D0A00000D0A12
:1026C0002057616974536F6E792000000D0A2057FE
:1026D000616974536F6E792000002054696D656FD5
:1026E000757420256C6420286D73290D0A000D0A6D
:1026F0002057616974536F6E792000002054696D12
:10270000656F757420256C6420286D73290D0A008F
:102710000A0D2042616420436F6D6D616E640A0D85
:1027200000000D0A205761697443616E6F6E20547A
:10273000696D656F757420256C6420286D73290D93
:102740000A000D0A205761697443616E6F6E2000A4
:102750000D0A205761697443616E6F6E41636B208F
:1027600054696D656F757420256C6420286D73291C
:102770000D0A00000D0A205761697443616E6F6E87
:1027800041636B2000005761697443616E6F6E4155
:10279000636B202532782C25327820282532782941
:1027A0000D0A0000446F55706461746543616D6586
:1027B000726153746174653A205374617465466C38
:1027C00061673D202532582C204C6173743D2532C1
:1027D000582C204163746976653D2532580A0D3EB8
:1027E0000000446F55706461746543616D6572618A
:1027F00053746174653A20446966666572656E63F8
:10280000653D2532780A0D00446F5570646174652A
:1028100043616D65726153746174653A20546F2031
:102820004D616E75616C0A0D3E00446F55706461B8
:10283000746543616D65726153746174653A2052C9
:1028400065736574204272696768746E657373207E
:10285000746F2064656661756C740A0D3E00446F88
:1028600055706461746543616D6572615374617420
:10287000653A20546F204175746F0A0D3E00446F15
:1028800055706461746543616D6572615374617400
:10289000653A20546F204D616E75616C0A0D3E00E3
:1028A0000D0A205761697450616E61736F6E6963C0
:1028B0002054696D656F757420256C6420286D73D4
:1028C000290D0A000D0A205761697450616E617309
:1028D0006F6E696320000D0A205761697450616E44
:1028E00061736F6E6963526573702054696D656FB3
:1028F000757420256C6420286D73290D0A000D0A5B
:10290000205761697450616E61736F6E69635265BF
:10291000737020000A0D50726F64756374204E61ED
:102920006D653A20257325730A0D000020202020B4
:10293000436F6D70696C65643A2025732061742063
:1029400025730A0D000030382D4175672D31310097
:1029500030383A35333A353200000D0A5379737402
:10296000656D2053657474696E67733A0A0D0A0DBC
:1029700044656661756C742043616D6572613A20CF
:1029800025640A0D44656661756C74205072657328
:1029900065743A2025640A0D00000D0A54696C74B0
:1029A0005370656564202050616E537065656420C6
:1029B000205A6F6F6D5370656564202050616E659D
:1029C0006C204C69676874730A0D00002020202574
:1029D000642020202020202020202564202020206A
:1029E000202020202564202020202020202020209E
:1029F00025640A0D0A0D00000D0A4A6F7973746987
:102A0000636B2053656E73697469766974792020ED
:102A100050616E202054696C742049646C65205AA2
:102A20006F6E650A0D00202020202020202020200D
:102A3000202020202020202020202020202564204D
:102A400020202564202020202020202025640A0D1D
:102A50000A0D00000A0D507265736574733A0A0D11
:102A60000A0D000043616D20507265204D6F646552
:102A70006C2020202020202020202020202020200A
:102A8000202050616E20202054696C7420205A6FE1
:102A90006F6D20466F63757320204272696768749A
:102AA0006E6573730000205B4272696768742C4620
:102AB0006F6375732C4157422C424C435D0A0D0ADB
:102AC0000D00202564202020253264202531387314
:102AD00020253258254C582020254C582020254CA4
:102AE000582020254C582020202020254C5800001C
:102AF0000A0D436F6D6D616E6420436F6D706C6580
:102B000074650A0D3E000A0D43616D204D6F6465CA
:102B10006C0A0D0020256420204E6F2043616D65F6
:102B200072610A0D00000A0D436F6D6D616E6420C5
:102B3000436F6D706C6574650A0D3E000A0D436F3E
:102B40006D6D616E6420436F6D706C6574650A0D08
:102B50003E000A0D436F6D6D616E6420436F6D70B2
:102B60006C6574650A0D3E003E2573204E6F74201F
:102B7000466F756E640A0D3E00000A0D436F6D6D61
:102B8000616E6420436F6D706C6574650A0D3E0064
:102B90000A0D0A0D526561642049324320552564AF
:102BA00020416464726573733D2532582052656715
:102BB00069737465723D25325820526573706F6E6B
:102BC00073653D2532580A0D00000A0D0A0D526545
:102BD0006164204932432055256420416464726554
:102BE00073733D2532582052656769737465723D71
:102BF00025325820526573706F6E73653D254C58B1
:102C00000A0D00000A0D0A0D5265616420536563C8
:102C10006F6E6461727920493243205525642041EA
:102C20006464726573733D25325820526567697319
:102C30007465723D25325820526573706F6E7365EE
:102C40003D2532580A0D00000A0D0A0D52656164D7
:102C5000205365636F6E6461727920493243205559
:102C6000256420416464726573733D253258205297
:102C7000656769737465723D2532582052657370BB
:102C80006F6E73653D254C580A0D00000A0D0A0D44
:102C900057726974652055256420416464726573B8
:102CA000733D2532582C52656769737465723D25F2
:102CB00032582C446174613D253258200A0D0000C1
:102CC0000A0D0A0D57726974652055256420416408
:102CD00064726573733D2532582C5265676973744D
:102CE00065723D2532582C446174613D254C582055
:102CF0000A0D00000A0D0A0D5772697465205365AC
:102D0000636F6E646172792055256420416464723A
:102D10006573733D2532582C52656769737465720B
:102D20003D2532582C446174613D253258200A0DEE
:102D300000000A0D0A0D5772697465205365636FB0
:102D40006E646172792055256420416464726573F4
:102D5000733D2532582C52656769737465723D2541
:102D600032582C446174613D254C58200A0D0000F6
:102D70000A0D3E2043616D657261202564204E6F0F
:102D80007420617661696C61626C650A0D3E200099
:102D90000A0D3E204A6F79737469636B204E657526
:102DA0007472616C205A6F6E65202564200A0D3E96
:102DB00020004F6E2043616D65726120496E697419
:102DC0002C2073656E6420486F6D6520636F6D6D98
:102DD000616E640A0D3E20004F6E2043616D657286
:102DE0006120496E69742C2073656E642050726591
:102DF00073657420313220636F6D6D616E64207372
:102E0000657175656E63650A0D3E20000A0D3E20F2
:102E10004A6F79737469636B2050616E2053656EDD
:102E20007369746976697479202564200A0D3E20DF
:102E300000000A0D3E53657444656661756C74202C
:102E40002564200A0D3E20000A0D3E44656661752A
:102E50006C7443616D202564200A0D3E20000A0D2C
:102E60003E204A6F79737469636B2050616E205302
:102E7000656E7369746976697479202564200A0D1A
:102E80003E20000045787465726E616C2054726952
:102E90006767657273206172652041637469766546
:102EA00020486967680A0D0045787465726E616C28
:102EB000205472696767657273206172652041638F
:102EC00074697665204C6F770A0D000050726F634D
:102ED0006573732055313420254C5820254C580AF1
:102EE0000D002563494E503A25643B0043544C2065
:102EF0004125640A0D3E0000342A3023000025637A
:102F0000494E503A25643B256354414B3A25642E83
:102F100025643B002563494E503A25643B004354E9
:102F20004C204225640A0D3E000056616C696461C4
:102F300074652043757272656E7453746174652E86
:102F400043616D6572615B25645D202532580A0D11
:102F500000004E6F2D56616C696461746520437585
:102F60007272656E7453746174652E43616D65721F
:102F7000615B25645D202532580A0D004C6F616449
:102F800020507265736574732043616D2025640A57
:102F90000D0043616D6572612025640A0D3E0000DD
:102FA00050726F636573732055313520254C58205E
:102FB000254C580A0D00496E43616D2053746F72A1
:102FC000652025640A0D3E0053746F7265202564E8
:102FD0000A0D3E005072657365742025640A0D3E2B
:102FE000000050616E61736F6E696320466F637598
:102FF000733A20546F204175746F0A0D3E00506182
:103000006E61736F6E696320466F6375733A205407
:103010006F204D616E75616C0A0D3E0050616E61EE
:10302000736F6E6963204272696768743A20546FE7
:10303000204175746F0A0D3E000050616E61736F20
:103040006E6963204272696768743A20546F204D3C
:10305000616E75616C0A0D3E000050726573657497
:103060002025640A0D3E0000446973706C6179206C
:10307000434841204F6E0A0D3E00446973706C61F5
:1030800079204F66660A0D3E0000446973706C61DA
:103090007920434842204F6E0A0D3E004469737008
:1030A0006C6179204F66660A0D3E000056616C69BE
:1030B000646174652043757272656E7453746174D3
:1030C000652E43616D6572615B25645D2025325814
:1030D0000A0D00004E6F2D56616C696461746520A5
:1030E00043757272656E7453746174652E43616DBD
:1030F0006572615B25645D202532580A0D004C6FB6
:10310000616420507265736574732043616D20257E
:10311000640A0D0043616D6572612025640A0D3EED
:10312000000050726F636573732055313620254C53
:103130005820254C580A0D00424C43204F66660A21
:103140000D3E0000424C43204F6E0A0D3E00506F72
:10315000776572204F66660A0D3E0000506F7765F6
:1031600072204F6E0A0D3E004272696768742055E6
:10317000700A0D3E000042726967687420446F77E0
:103180006E0A0D3E000042726967687420417574D2
:103190006F0A0D3E0000427269676874204D616ECF
:1031A00075616C0A0D3E0000466F637573204E65B5
:1031B00061720A0D3E00466F637573204661720AA4
:1031C0000D3E0000466F637573204175746F0A0DE4
:1031D0003E00415742204F66660A0D3E00004157AF
:1031E00042204F6E0A0D3E002043616D202532586B
:1031F000202C205374617465202532580A0D00007C
:10320000426164204765742055313420495352206F
:10321000254C5820254C580A0D0042616420476512
:1032200074205531352049535220254C5820254CC7
:10323000580A0D00426164204765742055313620DC
:1032400049535220254C5820254C580A0D004368FC
:1032500065636B20552532642D50696E3D253032F3
:10326000642C205265733D5270253032642C204D01
:1032700061696E5F4A50332D253032642F41756489
:10328000696F3A4A50312D342C204C333A5031205A
:103290002620380A0D00436865636B20552532648B
:1032A0002D50696E3D253032642C205265733D529D
:1032B00070253032642C204D61696E5F4A50332D89
:1032C000253032642F417564696F3A4A50322D348B
:1032D0002C204C333A5032202620370A0D00436808
:1032E00065636B20552532642D50696E3D25303263
:1032F000642C205265733D5270253032642C204D71
:1033000061696E5F4A50332D253032642F417564F8
:10331000696F3A4A50332D342C204C343A503120C6
:103320002620380A0D00436865636B2055253264FA
:103330002D50696E3D253032642C205265733D520C
:1033400070253032642C204D61696E5F4A50332DF8
:10335000253032642F417564696F3A4A50332D34F9
:103360002C204C343A5032202620370A0D00436876
:1033700065636B20552532642D50696E3D253032D2
:10338000642C205265733D5270253032642C204DE0
:1033900061696E5F4A50342D253032640A0D000099
:1033A000436865636B205525643A50696E3D25304E
:1033B00032642C205265733D52253032642C2042F9
:1033C0007574746F6E3D253032640A0D00004D61D6
:1033D000696E566964656F204572726F7220506F16
:1033E00072743D2532780A0D3E20000050726576D9
:1033F000696577566964656F204572726F722050F7
:103400006F72743D2532780A0D3E2000C69E9E964E
:10341000F5CCC9FF020EC6BE05D09EA6FED7000E93
:10342000C5BC010E016E000CC69CC586C5B6FED794
:1034300000B0C59A00A0C58AC588C5B8FED7C9CF57
:1034400001F0000C0C01F06BC580C5B0FED70A0E70
:10345000006E002EFED700D0EE51FE0BF16FF56F1F
:103460000001D4DF0A0E006E002EFED700D0EFCC94
:10347000F5FCCCDF0A0E006E002EFED700D0C58210
:10348000C5B2FED70A0E006E002EFED700D00C018A
:10349000EE510109F16FF56F0001B8DF0A0E006E01
:1034A000002EFED700D0006ABFDF01C0F0FC0A0E7C
:1034B000006E002EFED700D0C584C5B4FED70D0E19
:1034C000006E002EFED70C01F0CC01F00001000CC4
:1034D0000C01EB6BEA6BEC6BE951FE0BED6FE8CC8A
:1034E000EEFCEF6F0001AEDF01C0ECFC0C01E95116
:1034F0000109ED6FE8CCEEFCEF6F0001A3DF01C026
:10350000EBFC0C01EA6BEC51EA13EACC01F0EBCCDA
:1035100002F00001000C0C01E76BE66B4E80400EE0
:10352000E86F080EE96F0001D3DF02C0E7FC01C0BD
:10353000E6FCF292E4EF03F00C01E76BE66B4E82DF
:10354000440EE86F080EE96F0001C2DF02C0E7FC1D
:1035500001C0E6FCF092E4EF03F00C01E76BE66BD0
:103560004E84420EE86F080EE96F0001B1DF02C021
:10357000E7FC01C0E6FCF090E4EF03F00C01E76B20
:10358000E66B4E86460EE86F080EE96F0001A0DF7D
:1035900002C0E7FC01C0E6FCF094E4EF03F00C018C
:1035A000E951016AE85D03E2E8CC00F00CD0006A62
:1035B000080EEA6FE8370036E951005CD8B0006EBB
:1035C0000136EA2FF7D70001000C0101AA51040DC2
:1035D000F3500C01E76BE66F036A0101BA510C016D
:1035E000E625016EE75103220150AE0FE96E010E90
:1035F0000320EA6EC282C2B2FED7C4CFEFFF010140
:10360000AA51040DF3500C01E76BE66F036A010148
:10361000BA510C01E625016EE75103220150AE0FAD
:10362000E96E010E0320EA6EEF507B0827E20101EC
:10363000AA51040DF3500C01E76BE66F036A010118
:10364000BA510C01E625016EE75103220150AE0F7D
:10365000E96E010E0320EA6EEF5084080FE3D89064
:103660000101AA35036ABB0FE96E010E0320EA6E61
:10367000EC6AED52800EEF6E77D00C01D89001010C
:10368000AA35036ABB0F016E010E032201C0E6FCDE
:1036900003C0E7FC0101AA51040DF3500C01E96BD2
:1036A000E86FAE0EE825E96E010EE921EA6EEF50F3
:1036B000E96BE86F0101AA51040DF3500C01EB6BAB
:1036C000EA6F010EEA25016E000EEB21036E015038
:1036D000AE0FE96E010E0320EA6EEF50036AE82791
:1036E0000350E9230101AA51040DF3500C01EB6BC7
:1036F000EA6F020EEA25016E000EEB21036E015007
:10370000AE0FE96E010E0320EA6EEF50036AE82760
:103710000350E9230101AA51040DF3500C01EB6B96
:10372000EA6F030EEA25016E000EEB21036E0150D5
:10373000AE0FE96E010E0320EA6EEF50036AE82730
:103740000350E923E931036EE831026E033202329D
:103750003F0E0316E7CCEAFFE6CCE9FF03C0ECFF1F
:10376000ED5202C0EFFF0101010EBA25030BBA6F43
:10377000010EAA250C01E76FE86F030EE96F000147
:103780000EDF00C0AAF10101AA35006E0036FC0E62
:103790000016C250C30B0010C26E5F2E1FD05E2AEF
:1037A0000001602B1B0E5F6E5DA80DD06207625397
:1037B0000AE15D98C6C116F2C7C117F2C6C115F27B
:1037C0004C804C824B8C5ABE02D05DA006D060511A
:1037D000030803E25A9E5D90478A01019E90000112
:1037E000E4EF03F0F294E4EF03F0C580C5B0FED738
:1037F0000A0E006E002EFED700D00C01F151FE0B18
:10380000F46FF56F000102DE0A0E006E002EFED787
:1038100000D0F2CCF5FCFADD0A0E006E002EFED7C9
:1038200000D0F3CCF5FCF2DD0A0E006E002EFED7C0
:1038300000D0C584C5B4FED70D0E006E002EFED795
:10384000000C0C01EB510109EE6FEDCCEFFCF06BBD
:10385000F06BEACCF1FCF26FEDCCF3FC0001C5DFBC
:103860000C01EB51FE0BEE6FECCCEFFCF06BEACCF5
:10387000F1FCF26FECCCF3FC0001B7DF000C0C01A3
:10388000EC6BEB6B010EEA5DF40F51E20C0F0001E3
:103890009DEF1CF00C01EC6B080EEB6F48D00C0197
:1038A000EC6B040EEB6F43D00101C3A105D00C01FA
:1038B000EC6B010EEB6F04D00C01EC6B020EEB6FA6
:1038C00036D00101C3A105D00C01EC6B020EEB6FE9
:1038D00004D00C01EC6B010EEB6F29D0800E0C01B3
:1038E000EC6FEB6B24D0400E0C01EC6FEB6B1FD038
:1038F000200E0C01EC6FEB6B1AD0100E0C01EC6F6C
:10390000EB6B15D0080E0C01EC6FEB6B10D0040EB6
:103910000C01EC6FEB6B0BD0020E0C01EC6FEB6B40
:1039200006D0010E0C01EC6FEB6B01D00C01EBCC5F
:1039300001F0ECCC02F00001000CE824F76AF73645
:103940005B0FF66E390EF722000EF86EFB6E0A0062
:10395000F550FA6E0800F550F96E223918390E3913
:103960000439FA38F038E638DC38C238A8389E38DE
:1039700094380C01EC6BEB6BEA5102080EE3010E7C
:10398000EA5D006E400EEB6FEC6B005205E0D890E4
:10399000EB37EC37002EFBD721D0EA5104080EE3B9
:1039A000030EEA5D006E400EEC6FEB6B005205E01B
:1039B000D890EB37EC37002EFBD710D0EA51060831
:1039C0000DE3050EEA5D006E400EEB6FEC6B0052EE
:1039D00005E0D890EB37EC37002EFBD7EBCC01F0AD
:1039E000ECCC02F00001000C0C01E66BE86BE76B1D
:1039F000E96B5AAA03D05A9CA08281D1A0925A8C1A
:103A00005AA060D051504F14EA6F52505014EB6FCF
:103A1000EA5304E1EB5302E15AA20BD04F50FF0AE4
:103A2000006E5050FF0A036E00505116035052169C
:103A300004D04F505112505052125350010A0001FD
:103A400005E0030A0EE0010A1AE024D04C0E0C0136
:103A5000EA6FEB6B52C0EDFC51C0ECFC0001F1DEF3
:103A60001BD052C0EAFC0C01EB6BEB6B480EF16F04
:103A7000010EF26F52C0F3FC0001B7DE0DD04A0E0A
:103A80000C01EA6FEB6B52C0EDFC51C0ECFC000185
:103A9000D8DE02D05A8200D05AA205D0536A526AA8
:103AA000516A5A905A925AA006D0A0825A9C0C0190
:103AB00026D108D000015AB406D05A9C5A945A967E
:103AC0000C011DD100015AA607D05A945A960C0138
:103AD000E66B5B6A14D100015AA40ED15B52D8B4D4
:103AE0000BD10C01E66B5BC0E9FCE9510C080EE35D
:103AF000036AE9514F0FE96E020E0320EA6EEF529E
:103B000003E1E9CCE6FC02D0E92BEFD7E65318E15C
:103B10005B2C01D015D0010E5B6E5BC0E9FCE95156
:103B20000C080EE3036AE9514F0FE96E020E032001
:103B3000EA6EEF5203E1E9CCE6FC02D0E92BEFD7C5
:103B4000E653D8B475D0FF0E541A551A300E5416D9
:103B5000556AE6515C5C02E15A7801D05A985AB82D
:103B600008D0E6CCEAFC00018ADE01505412025073
:103B7000551210C2EAFC0001FCDE02C0E8FC01C0E4
:103B8000E7FC0201105102081AE30C01E751581436
:103B9000EA6FE8515914EB6FEA530BE1EB5309E17B
:103BA000E7515412E8515512E7515812E851591291
:103BB00004D03F0E5416596A586A27D00201FF0EEE
:103BC000561A571A56500C01E715EA6F5750E81568
:103BD000EB6FEA530AE1EB5308E13F0E5616571616
:103BE000E7515612E851571203D03F0E561657169A
:103BF000FF0E561A571A4A0EEA6FEB6B57C0EDFCD0
:103C000056C0ECFC00011DDE0C01FF0E541A551AC3
:103C10004C0EEA6FEB6B55C0EDFC54C0ECFC0001A0
:103C200010DEE6CC5CF0010E0C01E6255B6E5ED08A
:103C30005B2C5CD0FF0E541A551AF00E5416556AC0
:103C400010C2EAFC000195DE02C0E8FC01C0E7FCFE
:103C500002011051020824E354500C01E715EA6FE9
:103C60005550E815EB6FEA530AE1EB5308E1300ECB
:103C70005416556AE7515412E851551203D0300ECC
:103C80005416556AFF0E541A551A4C0EEA6FEB6B18
:103C900055C0EDFC54C0ECFC0001D3DD26D0020180
:103CA000FF0E561A571A56500C01E715EA6F575077
:103CB000E815EB6FEA530AE1EB5308E13F0E5616A5
:103CC0005716E7515612E851571203D03F0E5616B9
:103CD0005716FF0E561A571A4A0EEA6FEB6B57C06B
:103CE000EDFC56C0ECFC0001ACDD0C01E9510D0807
:103CF00002E2010E5B6E00015A9CA0820C01A192AF
:103D00000001E4EF03F09EA8FED7AD6E000C0C019D
:103D1000E66B9EAA57D09EAAFED7AECFE6FC036AFA
:103D2000000165516A0FE96E000E0320EA6EE6CCD1
:103D3000EFFF036A65516A0FE96E000E0320EA6E19
:103D4000EF500D0801E1672B010E6525FF0802E128
:103D5000656B01D0652B5D8E49BC2ED00101C5A9D4
:103D60002DD00C01E651210806E0E651220803E0BF
:103D7000E651300809E100016951800806E2695105
:103D8000890803E30C01E66B00010C01E651080809
:103D90000AE1E6510001B7DF200EB5DF0C01E65164
:103DA0000001B1DF0C01E6511F0807E2E6517E0871
:103DB00004E3E6510001A7DF0C010101E6CC69F044
:103DC0000C01A7D79E9A0001E4EF03F00C01E66B0B
:103DD000A4AA21D0A4AAFED76ECFE6FC49AE05D096
:103DE000E651000190DF15D00C01036A0001665115
:103DF0006A0FE96E010E0320EA6EE6CCEFFF0101C7
:103E00006981010E000166253F0802E2666B01D060
:103E1000662B0C01DDD7A49A0001E4EF03F0342AED
:103E200030230000342A30230000436F6D312052CC
:103E3000656365697665204572726F722873293DE6
:103E40002532780A0D00436F6D3220526563656933
:103E50007665204572726F722873293D2532780A83
:103E60000D000A0D43616D6572612050617373200E
:103E7000436F6D706C6574650A0D3E000A0D4361F9
:103E80006D657261205061737320436F6D706C6556
:103E900074650A0D3E000A0D43616D657261205024
:103EA00061737320436F6D706C6574650A0D3E001D
:103EB0005461736B466C61677320307830662028DC
:103EC000254C58290A0D000050726F64756374699F
:103ED0006F6E56696577534A25730A0D00002020DE
:103EE0002020436F6D70696C65643A2025732061F2
:103EF000742025730A0D000030382D4175672D316F
:103F0000310030383A35333A353200005461736B42
:103F1000466C6167732030783066302028254C5815
:103F2000290A0D005461736B466C61677320307809
:103F3000306630302028254C58290A0D0000546185
:103F4000736B466C616773203078663030302028A0
:103F5000254C58290A0D0000446F44556D7000002F
:103F6000456E61626C652053657269616C0A0D0073
:103F70005461736B466C6167733220307830662011
:103F800028254C58290A0D005461736B466C6167F3
:103F900073322030783066302028254C58290A0D9D
:103FA00000005461736B53696D756C6174652030EA
:103FB00078303030662028254C58290A0D0054618D
:103FC000736B53696D756C61746520307830663041
:103FD0002028254C58290A0D00005461736B536941
:103FE0006D756C617465203078306630302028251E
:103FF0004C58290A0D005461736B53696D756C61DF
:104000007465203078663030302028254C58290AD5
:104010000D005461736B53696D756C61746531206B
:104020003078303030662028254C58290A0D0000A1
:104030005461736B53696D756C61746531203078B0
:10404000303066302028254C58290A0D0000342ACB
:1040500030230000080EEA6ED30EE96EEF500EE03A
:10406000050E016E006A002EFED7012EFBD72E0E24
:10407000006E002EFED700D0EF2EF2D7000C080EF7
:10408000EA6EE50EE96EEF500EE0050E016E006A75
:10409000002EFED7012EFBD72E0E006E002EFED76F
:1040A00000D0EF2EF2D7000C0801DB39F00B006EC8
:1040B0000F0E8C1400108C6E00008C80020E006EAF
:1040C000002EFED700008C900001000C8350006E83
:1040D00000380F0B016E000C0F0E9514F009956E51
:1040E0008C8400008C800000F1DF01C0DBF88C9034
:1040F00000008C8000D000D0E9DF01C0DAF88C909D
:104100000F0E9514956E0801DB39006EF00E001647
:104110000050DA11016E000190EF20F08C92DCD794
:1041200001C0DAF8080101AE02D00001F8D78C9284
:10413000D8B18C8200008C9400008C90D939DA6F51
:104140000F0EDA17DAC8DBF80001AEDF0801D9512B
:104150000F0BDA6FDB6F0001A7DF000C0F0E951459
:10416000956E9590959295948C928C948C900F0E60
:104170000801E56F000183DF010E0401C36FC35125
:1041800003080DE3030E0801DB6F00018DDF050E50
:104190000801E56F000173DF0401C32BF0D7020EA5
:1041A0000801DB6F000180DF0401C36BC35103080A
:1041B0000FE3036AC35100010FEC04F00401C46F64
:1041C0000801D86BD96F0001A9DF0401C32BEED71A
:1041D0000001E0EFF4F0D3C8D5F8D2C8D4F8D5C8C0
:1041E00003F00801D4C8E9FFD5C8EAFFEF5206E0A2
:1041F000D42BD8B4D52B0001F2D70801D251D45D0D
:10420000006ED351D559036E00C001F00001000CBF
:104210000801D52D01D003D0400ED66F01D0D66B4A
:10422000010ED45DD627D6518009D76FD86BD96FD0
:10423000000174DF000C0801D3510C0A000105E0F5
:10424000060A0FE0020A15E01BD00801D86B010E28
:10425000D96F000163DF020E0801E56F00010FDF77
:1042600017D0010E0801D46F020ED56F0001D0DF08
:104270000FD00801D86B100ED96F00014FDF08D0A6
:10428000010E0801D86FD3C8D9F8000147DF00D06C
:10429000000C0801D16BD0C8D3F8CFC8D2F8000108
:1042A0009ADF0152D8B48ED0D0C8D3F8CFC8D2F894
:1042B00092DF01500801D15DD8B085D0036AD15199
:1042C000CF25E96ED0510320EA6EEF50010A0001BC
:1042D0000DE0030A26E0010A3FE0080A58E0070A59
:1042E0005EE0060A5CE0020A5AE059D00801D153A8
:1042F00017E1010ED46FD56F00018ADF200E08018F
:10430000D36F000198DF010E0801D46F020ED56F44
:1043100000017EDF200E0801D36F00018CDF080151
:104320004ED00801D15317E1010ED46FD56F0001B3
:104330006FDF3E0E0801D36F00017DDF010E080123
:10434000D46F020ED56F000163DF200E0801D36F1A
:10435000000171DF080133D00801D15317E1010ECC
:10436000D46FD56F000154DF200E0801D36F000118
:1043700062DF010E0801D46F020ED56F000148DF25
:104380003E0E0801D36F000156DF080118D0010E60
:104390000801D46FD56F00013BDF080110D0036A1C
:1043A0000801D151CF25E96ED0510320EA6EEFCF3D
:1043B000D2F8D2C8D3F800013EDF080100D0D12BDB
:1043C000000172D708010001000C010E016E16EF0A
:1043D000F5F01B6AF2BE1B8EF29E4C0E0C01EA6FCA
:1043E000040EEB6FED6BEC6B000121EC1CF01BBEBF
:1043F000F28E1B6AF2BE1B8EF29E4C0E0C01EA6F0F
:10440000060EEB6FED6BEC6B000121EC1CF01BBE9C
:10441000F28E1B6AF2BE1B8EF29E4C0E0C01F16FE7
:104420000B0EF26FF36B0001F5EC1BF01BBEF28E6E
:104430001B6AF2BE1B8EF29E480E0C01EA6F040E40
:10444000EB6FED6BEC6B000121EC1CF01BBEF28EF0
:104450001B6AF2BE1B8EF29E480E0C01EA6F060E1E
:10446000EB6FED6BEC6B000121EC1CF01BBEF28ED0
:104470001B6AF2BE1B8EF29E480E0C01F16F0A0EF3
:10448000F26FF36B0001F5EC1BF01BBEF28E1B6AA2
:10449000F2BE1B8EF29E4A0E0C01EA6F040EEB6F09
:1044A000ED6BEC6B000121EC1CF01BBEF28E1B6A65
:1044B000F2BE1B8EF29E4A0E0C01EA6F060EEB6FE7
:1044C000ED6BEC6B000121EC1CF01BBEF28E1B6A45
:1044D000F2BE1B8EF29E4A0E0C01F16F0A0EF26FB5
:1044E000F36B0001F5EC1BF01BBEF28E1B6AF2BEF3
:1044F0001B8EF29E400E0C01EA6F040EEB6FED6B0B
:10450000EC6B000121EC1CF01BBEF28E1B6AF2BEAC
:104510001B8EF29E400E0C01EA6F060EEB6FED6BE8
:10452000EC6B000121EC1CF01BBEF28E1B6AF2BE8C
:104530001B8EF29E400E0C01F16F0A0EF26FF36BB0
:104540000001F5EC1BF01BBEF28E1B6AF2BE1B8E47
:10455000F29E440E0C01EA6F040EEB6FED6BEC6BF8
:10456000000121EC1CF01BBEF28E1B6AF2BE1B8EFA
:10457000F29E440E0C01EA6F060EEB6FFF0EED6F1C
:10458000EC6F000121EC1CF01BBEF28E1B6AF2BE28
:104590001B8EF29E440E0C01F16F0A0EF26FF36B4C
:1045A0000001F5EC1BF01BBEF28E1B6AF2BE1B8EE7
:1045B000F29E420E0C01EA6F040EEB6FED6BEC6B9A
:1045C000000121EC1CF01BBEF28E1B6AF2BE1B8E9A
:1045D000F29E420E0C01EA6F060EEB6FFF0EED6FBE
:1045E000EC6F000121EC1CF01BBEF28E1B6AF2BEC8
:1045F0001B8EF29E420E0C01F16F0A0EF26FF36BEE
:104600000001F5EC1BF01BBEF28E1B6AF2BE1B8E86
:10461000F29E460E0C01EA6F040EEB6FED6BEC6B35
:10462000000121EC1CF01BBEF28E1B6AF2BE1B8E39
:10463000F29E460E0C01EA6F060EEB6FFF0EED6F59
:10464000EC6F000121EC1CF01BBEF28E1B6AF2BE67
:104650001B8EF29E460E0C01F16F0A0EF26FF36B89
:104660000001F5EC1BF01BBEF28E3FEFF5F00401EC
:10467000F751010A00010AE0030AD8B491D0010AF7
:10468000D8B418D1030AD8B49FD19ED1020EEA6ED5
:104690005C0EE96E000EADEC07F00A000900F55063
:1046A000EE6E0009FBE1020EEA6E6E0EE96E000E80
:1046B000C0EC07F00A000900F550EE6E0009FBE1BE
:1046C000020EEA6E800EE96E000ED3EC07F00A00CF
:1046D0000900F550EE6E0009FBE1020EEA6E920E43
:1046E000E96E000EE6EC07F00A000900F550EE6EE8
:1046F0000009FBE1020EEA6EA40EE96E000EF9EC71
:1047000007F00A000900F550EE6E0009FBE1020E09
:10471000EA6EB60EE96E000E0CEC08F00A00090015
:10472000F550EE6E0009FBE1020EEA6EC80EE96E6E
:10473000000E1FEC08F00A000900F550EE6E0009AB
:10474000FBE1020EEA6EDA0EE96E000E32EC08F0C2
:104750000A000900F550EE6E0009FBE1020EEA6E58
:10476000EC0EE96E000E45EC08F00A000900F55069
:10477000EE6E0009FBE1010E0301C46F036AC45130
:10478000CD0FE96E030E0320EA6E080EEF6E036A8A
:10479000C451D10FE96E030E0320EA6EEF6A99D17E
:1047A000020EEA6E5C0EE96E000E58EC08F00A008C
:1047B0000900F550EE6E0009FBE1020EEA6E6E0E86
:1047C000E96E000E6BEC08F00A000900F550EE6E81
:1047D0000009FBE1020EEA6E800EE96E000E7EEC2F
:1047E00008F00A000900F550EE6E0009FBE1020E28
:1047F000EA6E920EE96E000E91EC08F00A000900D4
:10480000F550EE6E0009FBE1020EEA6EA40EE96EB1
:10481000000EA4EC08F00A000900F550EE6E000945
:10482000FBE1020EEA6EB60EE96E000EB7EC08F080
:104830000A000900F550EE6E0009FBE1020EEA6E77
:10484000C80EE96E000ECAEC08F00A000900F55027
:10485000EE6E0009FBE1020EEA6EDA0EE96E000E62
:10486000DDEC08F00A000900F550EE6E0009FBE1EE
:10487000020EEA6EEC0EE96E000E45EC08F00A003E
:104880000900F550EE6E0009FBE1020E0301C46F52
:10489000036AC451CD0FE96E030E0320EA6E080EC1
:1048A000EF6E036AC451D10FE96E030E0320EA6E66
:1048B000EF6A0FD1020EEA6E5C0EE96E000EF0ECAC
:1048C00008F00A000900F550EE6E0009FBE1020E47
:1048D000EA6E6E0EE96E000E6BEC08F00A0009003D
:1048E000F550EE6E0009FBE1020EEA6E800EE96EF5
:1048F000000E7EEC08F00A000900F550EE6E00098B
:10490000FBE1020EEA6E920EE96E000E91EC08F0E9
:104910000A000900F550EE6E0009FBE1020EEA6E96
:10492000A40EE96E000EA4EC08F00A000900F55090
:10493000EE6E0009FBE1020EEA6EB60EE96E000EA5
:10494000B7EC08F00A000900F550EE6E0009FBE133
:10495000020EEA6EC80EE96E000ECAEC08F00A00FC
:104960000900F550EE6E0009FBE1020EEA6EDA0E68
:10497000E96E000EDDEC08F00A000900F550EE6E5D
:104980000009FBE1020EEA6EEC0EE96E000E45EC4A
:1049900008F00A000900F550EE6E0009FBE1030E75
:1049A0000301C46F036AC451CD0FE96E030E0320E7
:1049B000EA6E080EEF6E036AC451D10FE96E030E62
:1049C0000320EA6EEF6A85D0020EEA6E5C0EE96E95
:1049D000E26A340EE16EE752E6CFEEFFFCE1020E32
:1049E000EA6E6E0EE96EE26A220EE16EE752E6CFE3
:1049F000EEFFFCE1020EEA6E800EE96E000E03ECA3
:104A000009F00A000900F550EE6E0009FBE1020E04
:104A1000EA6E920EE96E000E16EC09F00A0009002B
:104A2000F550EE6E0009FBE1020EEA6EA40EE96E8F
:104A3000000E29EC09F00A000900F550EE6E00099D
:104A4000FBE1020EEA6EB60EE96E000E3CEC09F0D8
:104A50000A000900F550EE6E0009FBE1020EEA6E55
:104A6000C80EE96E000E4FEC09F00A000900F5507F
:104A7000EE6E0009FBE1020EEA6EDA0EE96E000E40
:104A800062EC09F00A000900F550EE6E0009FBE146
:104A9000020EEA6EEC0EE96E000E75EC09F00A00EB
:104AA0000900F550EE6E0009FBE10301C46B036AD7
:104AB000C451CD0FE96E030E0320EA6E120EEF6EA5
:104AC000036AC451D10FE96E030E0320EA6EEF6A48
:104AD00000D00001000C0801E66703D0E76702D0B0
:104AE00007D0E72BE5C8EEFFE62FFCD7E72FFAD774
:104AF0000001000CD0C8D6F8CFC8D5F80801D353B0
:104B000002E1D45327E0D2C803F0D1C8E9FFD2C8EC
:104B1000EAFFEF521FE0D6C803F0D551D52BD8B429
:104B2000D62BD76F03C0D8F8D2C803F0D151D12B00
:104B3000D8B4D22BE96E03C0EAFFEFCFD9F8D8C8BA
:104B4000EAFFD7C8E9FFD9C8EFFFD351D8B4D407DB
:104B5000D307D5D7D35302E1D4530FE0D6C803F01F
:104B6000D551D52BD8B4D62BE96E03C0EAFFEF6A36
:104B7000D351D8B4D407D307EDD7CFC801F0D0C8EC
:104B800002F00001000C010169B32AD0080EEA6EA0
:104B9000A90EE96E0801E56BE76B130EE66F0001E5
:104BA0009ADF080E0801D06FA90ECF6F020ED26FE8
:104BB0005C0ED16FD46B120ED36F00019BDF0C0E15
:104BC0000801A96F080ED06FA90ECF6F000149EC44
:104BD00021F0050E0801E56F00013FEC20F0010116
:104BE000080EEA6EBC0EE96E0801E56BE76B130E6A
:104BF000E66F000170DF080E0801D06FBC0ECF6FAA
:104C0000A8C8D2F8A7C8D1F8D46B120ED36F000190
:104C100071DF0A0E0801BC6F080ED06FBC0ECF6F9B
:104C2000000149EC21F0000C0401D8C4E9FFD9C40B
:104C3000EAFFEFCFDCF4DBC403F0DAC4E9FFDBC446
:104C4000EAFFEF50DC5D15E1D9C403F0D8C4E9FFF9
:104C500003C0EAFFEF5203E1000E016E1FD0D9C47A
:104C600003F0D851D82BD8B4D92BDA2BD8B4DB2BFE
:104C7000DCD7D9C403F0D8C4E9FFD9C4EAFFEFCF29
:104C8000DCF4DBC403F0DAC4E9FFDBC4EAFFEF5075
:104C9000DC5D02E2FF0E01D0010E016E000193EF18
:104CA00026F00401C36BC56BC46B200EC66FC76FC3
:104CB000C86FC96FCA6FCB6FCC6FCD6FCE6FCF6F20
:104CC000D06FD16FD26FD36FD46FD56FD66B030E09
:104CD000C56FE70EC46FC36BC35111081BE3036AB2
:104CE000C351C60FE96E040E0320EA6EF2CFDAF468
:104CF000F29EC5C4AAFFC4C4A9FFA69CA69EA68016
:104D0000A850DABFF28EEF6E010EC427000EC52345
:104D1000C32BE2D7040ED96FC60ED86FDB6B340EEF
:104D2000DA6F000181D7015204E1010E016E04D057
:104D300003D0000E016E00D0BDEFF5F00401DF6B73
:104D4000DE6BE06BF2CFE1F4F29E030EAA6EFF0E73
:104D5000A96EA69CA69EA680A850E1BFF28EE06F29
:104D6000DF6BDE6BDF5103081CE3DFC4AAFFDEC488
:104D7000A9FFFF0EA86EA69CA69EA684F250006E08
:104D8000F29E0F01550EA76EAA0EA76EA682A6B2BE
:104D9000FED7A6940050F2120401DE2BD8B4DF2B0C
:104DA000E1D7E051010819E3030EAA6EFF0EA96EC8
:104DB000E0C4A8FFA69CA69EA684F250006EF29EB8
:104DC0000F01550EA76EAA0EA76EA682A6B2FED739
:104DD000A6940050F21217D00401030EAA6EFF0E23
:104DE000A96EA86AA69CA69EA684F250006EF29EAA
:104DF0000F01550EA76EAA0EA76EA682A6B2FED709
:104E0000A6940050F212000159EF27F00401DF6B65
:104E1000DE6BE06BE16BE26BDF6B200EDE6FE06B55
:104E2000E05105082EE3E16BE1510B0828E3E26B4A
:104E3000E2510B0822E3DF51036EDE51DE2BD8B4C2
:104E4000DF2BE36F03C0E4F4E4C4AAFFE3C4A9FFCB
:104E5000A86AA69CA69EA684F250006EF29E0F0140
:104E6000550EA76EAA0EA76EA682A6B2FED7A6946E
:104E70000050F2120401E22BDBD7E12BD5D7E02B57
:104E8000CFD7E06BE0510C080AE3036AE0514F0F03
:104E9000E96E020E0320EA6EEF6AE02BF3D7000101
:104EA000000C0401DA6BD96BDC6BDB6BDD6B000192
:104EB00045D7AA6AA96A010EA86EA69CA69EA684DA
:104EC000F250006EF29E0F01550EA76EAA0EA76E4D
:104ED000A682A6B2FED7A6940050F212AA6A010ECC
:104EE000A96EA86EA69CA69EA684F2CF00F0F29EA4
:104EF000550EA76EAA0EA76EA682A6B2FED7A694DE
:104F00000050F212AA6A020EA96E0F0EA86EA69C9D
:104F1000A69EA684F2CF00F0F29E550EA76EAA0EB2
:104F2000A76EA682A6B2FED7A6940050F212AA6A75
:104F3000100EA96EA86AA69CA69EA684F2CF00F0C9
:104F4000F29E550EA76EAA0EA76EA682A6B2FED737
:104F5000A6940050F212AA6A030EA96E120EA86E51
:104F6000A69CA69EA684F2CF00F0F29E550EA76ED8
:104F7000AA0EA76EA682A6B2FED7A6940050F21281
:104F8000AA6A0F0EA96EA86AA69CA69EA684F2CF56
:104F900000F0F29E550EA76EAA0EA76EA682A6B2CC
:104FA000FED7A6940050F212AA6A040EA96EA86E4B
:104FB000A69CA69EA684F2CF00F0F29E550EA76E88
:104FC000AA0EA76EA682A6B2FED7A6940050F21231
:104FD000AA6A050EA96EA86EA69CA69EA684F2CF0C
:104FE00000F0F29E550EA76EAA0EA76EA682A6B27C
:104FF000FED7A6940050F212AA6A060EA96E180EE9
:10500000A86EA69CA69EA684F2CF00F0F29E550E36
:10501000A76EAA0EA76EA682A6B2FED7A6940050CF
:10502000F212AA6A070EA96E040EA86EA69CA69E8E
:10503000A684F2CF00F0F29E550EA76EAA0EA76EC0
:10504000A682A6B2FED7A6940050F212F2CFDEF4EA
:10505000F29E030EAA6EFF0EA96EA69CA69EA680C7
:10506000A8500401DEBFF28EDF6FAA6A080EA96E97
:10507000DFC4A8FFA69CA69EA684F250006EF29EF6
:105080000F01550EA76EAA0EA76EA682A6B2FED776
:10509000A6940050F212AA6A090EA96E190EA86E03
:1050A000A69CA69EA684F2CF00F0F29E550EA76E97
:1050B000AA0EA76EA682A6B2FED7A6940050F21240
:1050C000AA6A0A0EA96E180EA86EA69CA69EA684B1
:1050D000F2CF00F0F29E550EA76EAA0EA76EA68222
:1050E000A6B2FED7A6940050F212AA6A0B0EA96EC1
:1050F000180EA86EA69CA69EA684F2CF00F0F29E83
:10510000550EA76EAA0EA76EA682A6B2FED7A694CB
:105110000050F212AA6A0C0EA96E0E0EA86EA69C82
:10512000A69EA684F2CF00F0F29E550EA76EAA0EA0
:10513000A76EA682A6B2FED7A6940050F212AA6A63
:105140000D0EA96EA86AA69CA69EA684F2CF00F0BA
:10515000F29E550EA76EAA0EA76EA682A6B2FED725
:10516000A6940050F212AA6A0E0EA96EA86AA69C16
:10517000A69EA684F2CF00F0F29E550EA76EAA0E50
:10518000A76EA682A6B2FED7A6940050F212AA6A13
:10519000120EA96EA86AA69CA69EA684F2CF00F065
:1051A000F29E550EA76EAA0EA76EA682A6B2FED7D5
:1051B000A6940050F212000129DE030E0401DA6FFA
:1051C000E70ED96FDD6BDD51110827E3036ADD516E
:1051D000340FE96E000E0320EA6EEFCFDEF4DAC47E
:1051E000AAFFD9C4A9FFDEC4A8FFA69CA69EA684D8
:1051F000F250006EF29E0F01550EA76EAA0EA76E1A
:10520000A682A6B2FED7A6940050F212010E0401A7
:10521000D927000EDA23DD2BD6D7DC6BDB6BDD6BF9
:10522000DD51110843E3036ADD51220FE96E000EE0
:105230000320EA6EEFCFDEF4DE512F0803E2DE51E9
:10524000390802E2000E01D0010E01082DE1DC5305
:105250002BE1DB51050828E3036ADD51220FE96EDB
:10526000000E0320EA6EEFCFDEF4DAC4AAFFD9C441
:10527000A9FFDEC4A8FFA69CA69EA684F250006EDD
:10528000F29E0F01550EA76EAA0EA76EA682A6B2B9
:10529000FED7A6940050F2120401DB2BD8B4DC2B0D
:1052A000010ED927000EDA23DD2BBAD70001000C3E
:1052B0000C01E151E303F3CF01F0F4CF00F0E4037C
:1052C000F3500026E251E303F3500020026E000188
:1052D000000C0900F6CFE6F8F7CFE7F8F8CFE8F8CA
:1052E000F5509EA8FED7AD6EE6C8F6FFE7C8F7FFFB
:1052F000E8C8F8FF0801E52F01D002D00001E9D786
:105300000001000C0801E7BF10D00F0E006EE63957
:1053100000160A0E005C03E2300E002602D0E751B0
:10532000002600509EA8FED7AD6E0F0EE6170A0E9F
:10533000E65D02E2300E02D0E79FE751E627E65134
:105340009EA8FED7AD6E0001000C0501276B266BF1
:10535000286BFF0E296F245303E02451060804E252
:10536000000E016EA9D208D0255303E025510C0888
:1053700003E2000E016EA0D2276B900E266F010E85
:10538000245D036A2A6F03C02BF527C5E2FC26C5FE
:10539000E1FC03C0E4FCE8CFE3FC000189DF02C0CC
:1053A00027F501C026F5200E05012627000E27232C
:1053B000010E255D0C0DF350036A262703502723A9
:1053C0000101C4A126D0440EF66E230EF76E000E26
:1053D000F86E0E0E0801E56F00017BDF27C5E6F8C9
:1053E000370E0801E76F00018DDF26C5E6F8370E9E
:1053F0000801E76F000186DF200E9EA8FED7AD6E84
:105400000A0E9EA8FED7AD6E0D0E9EA8FED7AD6EFD
:1054100001010A0E050126252A6F000E27212B6F98
:10542000F2CF2CF5F29E2BC5AAFF2AC5A9FFA69C98
:10543000A69EA680A8502CBFF28E296F2751036E1E
:105440002651262BD8B4272B2A6F03C02BF5F2CF79
:105450002CF5F29E2BC5AAFF2AC5A9FFA69CA69EE5
:10546000A680A8502CBFF28E286F2839006E0F0E30
:10547000001600500B08D8A464D0D8900201103553
:10548000036AEA0FE96E010E0320EA6EEF50006E28
:10549000E92AEF50E906036E020E035C05E1010EF6
:1054A000005C000127E00201020E035C04E10052EF
:1054B000000120E00201030E035C04E10052000140
:1054C00022E00201010E035C05E1010E005C000117
:1054D00023E00201010E035C05E1020E005C000105
:1054E00024E00201010E035C04E10052000126E009
:1054F000020124D005012951160802E1296B02D0CE
:10550000FF0E296F1DD005012951170802E1296BF3
:1055100002D0FF0E296F14D005012951140802E1B1
:10552000296B02D0FF0E296F0BD0050129511508F8
:1055300002E1296B02D0FF0E296F02D0050100D0D5
:1055400001D0296B2953D8A4B4D12851F00BD8B479
:10555000B0D12851F00B2A6F0101D351F00B050196
:105560002A5DD8A4A6D128C5D3F12751036E2651B0
:10557000262BD8B4272B2A6F03C02BF5F2CF2CF59E
:10558000F29E2BC5AAFF2AC5A9FFA69CA69EA680AF
:10559000A8502CBFF28E0101D46F05012751036E74
:1055A0002651262BD8B4272B2A6F03C02BF5F2CF18
:1055B0002CF5F29E2BC5AAFF2AC5A9FFA69CA69E84
:1055C000A680A8502CBFF28E0101D66FD56B0501C5
:1055D0002751036E2651262BD8B4272B2A6F03C0E0
:1055E0002BF5F2CF2CF5F29E2BC5AAFF2AC5A9FFF9
:1055F000A69CA69EA680A8502CBFF28E0101D513B2
:1056000005012751036E2651262BD8B4272B2A6F6C
:1056100003C02BF5F2CF2CF5F29E2BC5AAFF2AC5AD
:10562000A9FFA69CA69EA680A8502CBFF28E0101C1
:10563000D86FD76B05012751036E2651262BD8B49E
:10564000272B2A6F03C02BF5F2CF2CF5F29E2BC52A
:10565000AAFF2AC5A9FFA69CA69EA680A8502CBF7B
:10566000F28E0101D71305012751036E2651262B17
:10567000D8B4272B2A6F03C02BF5F2CF2CF5F29E5E
:105680002BC5AAFF2AC5A9FFA69CA69EA680A85046
:105690002CBFF28E0101DA6FD96B05012751036E21
:1056A0002651262BD8B4272B2A6F03C02BF5F2CF17
:1056B0002CF5F29E2BC5AAFF2AC5A9FFA69CA69E83
:1056C000A680A8502CBFF28E0101D91305012751E5
:1056D000036E2651262BD8B4272B2A6F03C02BF537
:1056E000F2CF2CF5F29E2BC5AAFF2AC5A9FFA69CD6
:1056F000A69EA680A8502CBFF28E0101DC6FDB6B4A
:1057000005012751036E2651262BD8B4272B2A6F6B
:1057100003C02BF5F2CF2CF5F29E2BC5AAFF2AC5AC
:10572000A9FFA69CA69EA680A8502CBFF28E0101C0
:10573000DB13D339006E0F0E001600500B0808E182
:10574000DE6BDD6B0501262BD8B4272B1CD00101A5
:1057500005012751036E2651262BD8B4272B2A6F1B
:1057600003C02BF5F2CF2CF5F29E2BC5AAFF2AC55C
:10577000A9FFA69CA69EA680A8502CBFF28E010170
:10578000DE6FDD6B0501F2CF2AF5F29E27C5AAFF79
:1057900026C5A9FFA69CA69EA680A8502ABFF28E69
:1057A0000101DD13C4A180D05A0EF66E230EF76EF0
:1057B000000EF86E050E0801E56F00018ADDD3C109
:1057C000E6F8570E0801E76F00019CDD200E9EA849
:1057D000FED7AD6ED4C1E6F8570E0801E76F0001A1
:1057E00091DD200E9EA8FED7AD6ED6C1E6F8370E2D
:1057F0000801E76F000186DDD5C1E6F8370E080124
:10580000E76F00017FDD200E9EA8FED7AD6ED8C1E8
:10581000E6F8370E0801E76F000174DDD7C1E6F83E
:10582000370E0801E76F00016DDD200E9EA8FED740
:10583000AD6EDAC1E6F8370E0801E76F000162DDF0
:10584000D9C1E6F8370E0801E76F00015BDD200ED5
:105850009EA8FED7AD6EDCC1E6F8370E0801E76FF3
:10586000000150DDDBC1E6F8370E0801E76F0001EB
:1058700049DD200E9EA8FED7AD6EDEC1E6F8370EDC
:105880000801E76F00013EDDDDC1E6F8370E0801D3
:10589000E76F000137DD0A0E9EA8FED7AD6E0D0E34
:1058A0009EA8FED7AD6E0101010E016E050104D068
:1058B00003D0000E016E00D00001000CF2CFEFF417
:1058C000F29EAA6AA96AA69CA69EA680A850040178
:1058D000EFBFF28E0101C66FF2CFEFF4F29EAA6A1B
:1058E000010EA96EA69CA69EA680A8500401EFBF3B
:1058F000F28E0101C76FF2CFEFF4F29EAA6A020E98
:10590000A96EA69CA69EA680A8500401EFBFF28EA9
:105910000101C86FF2CFEFF4F29EAA6A100EA96ED1
:10592000A69CA69EA680A8500401EFBFF28E01019E
:10593000CB6FF2CFEFF4F29EAA6A030EA96EA69C7B
:10594000A69EA680A8500401EFBFF28E0101C96F88
:10595000F2CFEFF4F29EAA6A0F0EA96EA69CA69E45
:10596000A680A8500401EFBFF28E0101CA6FF2CFEA
:10597000EFF4F29EAA6A040EA96EA69CA69EA680CB
:10598000A8500401EFBFF28E0101CC6FF2CFEFF40B
:10599000F29EAA6A050EA96EA69CA69EA680A85095
:1059A0000401EFBFF28E0101CD6FF2CFEFF4F29E52
:1059B000AA6A060EA96EA69CA69EA680A8500401FF
:1059C000EFBFF28E0101C56FF2CFEFF4F29EAA6A2B
:1059D000070EA96EA69CA69EA680A8500401EFBF44
:1059E000F28E0101C46FF2CFEFF4F29EAA6A080EA4
:1059F000A96EA69CA69EA680A8500401EFBFF28EB9
:105A00000101C36FF2CFEFF4F29EAA6A090EA96EEC
:105A1000A69CA69EA680A8500401EFBFF28E0101AD
:105A2000CE6FF2CFEFF4F29EAA6A0A0EA96EA69C80
:105A3000A69EA680A8500401EFBFF28E0101CF6F91
:105A4000F2CFEFF4F29EAA6A0B0EA96EA69CA69E58
:105A5000A680A8500401EFBFF28E0101D06FF2CFF3
:105A6000EFF4F29EAA6A0C0EA96EA69CA69EA680D2
:105A7000A8500401EFBFF28E0101D16FF2CFEFF415
:105A8000F29EAA6A0D0EA96EA69CA69EA680A8509C
:105A90000401EFBFF28E0101C16FF2CFEFF4F29E6D
:105AA000AA6A0E0EA96EA69CA69EA680A850040106
:105AB000EFBFF28E0101C26FF2CFEFF4F29EAA6A3D
:105AC000120EA96EA69CA69EA680A8500401EFBF48
:105AD000F28E0101D26FD151280802E2280ED16F57
:105AE000CF51180802E2180ECF6FD051180802E209
:105AF000140ED06FC6C124F5C7C125F5000125DC01
:105B0000010E016E2FEF68F0036A63516A0FE96EB0
:105B1000000E0320EA6EEFCF44F50501010E0001EF
:105B200063250501466F1B6AF2BE1B8EF29EE8CF0D
:105B3000E8FCFF0E0C01E96F0001CFEC1AF01BBE70
:105B4000F28E00C063F06551635D01E15D9E050169
:105B500044C501F00001000C0501266B5DAE06D0C6
:105B60000001D2DF01C026F50501F8D70001676BFF
:105B7000000C0900F55211E0F6CFE1FCF7CFE2FC92
:105B8000F8CFE3FCF5509EA8FED7AD6EE1CCF6FF52
:105B9000E2CCF7FFE3CCF8FFECD7000C05012A6B51
:105BA000296B2B6B27C5EAFF26C5E9FF0801E56BCA
:105BB000E76B28C5E6F800016BEC25F005012A6BC0
:105BC000296B2A51030814E303E12951E70810E384
:105BD000020E0801D36F00012AEC20F0675303E0A6
:105BE000050106D000010501292BD8B42A2BE9D7DD
:105BF0000001675303E1000E016E79D005012B6BA4
:105C00005DAE73D0036A2B512625016E2751032206
:105C100001C02CF503C02DF5000176DF2DC5EAFF8C
:105C20002CC5E9FF01C0EFFF036A05012B512625B2
:105C3000E96E27510320EA6EEF500D083FE10001A5
:105C40006707050126C5E9FF27C5EAFFEF504508AC
:105C500018E1010E2625E96E000E2721EA6EEF50AD
:105C6000300809E0010E2625E96E000E2721EA6EB4
:105C7000EF50310806E1000E016E000138D008D067
:105C800005012B51020805E2010E016E00012FD023
:105C900005012B6B320E0801D36F00012AEC20F0B6
:105CA00027C5EAFF26C5E9FF0801E56BE76B28C5B4
:105CB000E6F800016BEC25F016D00501036A2B51C4
:105CC0002625E96E27510320EA6EEF500A0805E009
:105CD0002B2B28512B5D01E32B6B0A0E0801D36F90
:105CE00000012AEC20F005018BD7000E016E0001A7
:105CF000000C0501146B146B12C5EAFF11C5E9FF16
:105D00000801E56BE76B13C5E6F800016BEC25F0C5
:105D10006753D8B46CD05DAE6AD0036A05011451E4
:105D20001125016E1251032201C015F503C016F5AD
:105D30000001EADE16C5EAFF15C5E9FF01C0EFFF65
:105D4000036A050114511125E96E12510320EA6E10
:105D5000EF500D083BE100016707050111C5E9FFA0
:105D600012C5EAFFEF50450816E1010E1125E96E54
:105D7000000E1221EA6EEF50300809E0010E1125E5
:105D8000E96E000E1221EA6EEF50310804E1000EB8
:105D9000016E30D006D01451020803E2010E016EEC
:105DA00029D0146B320E0801D36F00012AEC20F0C9
:105DB00012C5EAFF11C5E9FF0801E56BE76B13C5E2
:105DC000E6F800016BEC25F011D00501036A1451CF
:105DD0001125E96E12510320EA6EEF500A0805E022
:105DE000142B1351145D01E3146B000194D7000EC2
:105DF000016E05010001000C0401F26BF391F3B197
:105E000014D10001A9DE1E0EF66E3E0EF76E000ED6
:105E1000F86EAFDEF0C427F5EFC426F5F1C428F51F
:105E2000BDDE015211E19D9A640E0801D36F00019D
:105E30002AEC20F091DE9D8AC00EF212640E080159
:105E4000D36F00012AEC20F0F0C427F5EFC426F54B
:105E5000F1C428F5A3DE012CDBD00401EFC4E9FF77
:105E6000F0C4EAFFEF50450816E1010EEF25E96E98
:105E7000000EF021EA6EEF5066080DE1020EEF25EC
:105E8000E96E000EF021EA6EEF50660804E1010EA3
:105E9000016ECDD049D0EFC4E9FFF0C4EAFFEF5066
:105EA000520842E1010EEF25E96E000EF021EA6E84
:105EB000EF50650839E1020EEF25E96E000EF02182
:105EC000EA6EEF50630830E1030EEF25E96E000E35
:105ED000F021EA6EEF506F0827E1040EEF25E96E1E
:105EE000000EF021EA6EEF506E081EE1050EEF2560
:105EF000E96E000EF021EA6EEF50660815E1060E1D
:105F0000EF25E96E000EF021EA6EEF5069080CE112
:105F1000070EEF25E96E000EF021EA6EEF506708DC
:105F200003E1010E016E83D0F0C412F5EFC411F548
:105F3000F1C413F50001DDDE012C69D00401EFC4CA
:105F4000E9FFF0C4EAFFEF50450816E1010EEF2526
:105F5000E96E000EF021EA6EEF5066080DE1020EC8
:105F6000EF25E96E000EF021EA6EEF50660804E1BD
:105F7000010E016E5CD049D0EFC4E9FFF0C4EAFF26
:105F8000EF50520842E1010EEF25E96E000EF021BC
:105F9000EA6EEF50650839E1020EEF25E96E000E5A
:105FA000F021EA6EEF50630830E1030EEF25E96E51
:105FB000000EF021EA6EEF506F0827E1040EEF2586
:105FC000E96E000EF021EA6EEF506E081EE1050E3C
:105FD000EF25E96E000EF021EA6EEF50660815E13C
:105FE000060EEF25E96E000EF021EA6EEF5069080B
:105FF0000CE1070EEF25E96E000EF021EA6EEF507E
:10600000670803E1010E016E12D08ED700011CD784
:10601000640E0801D36F00012AEC20F00401F22B7A
:10602000F251020801E2F381EAD6000E016E00018E
:10603000F6EF68F0580E0801E76F036A000164513B
:106040006A0FE96E010E0320EA6EEFCFE7F8080150
:10605000010E000164253F0B646F6651645D02E12F
:10606000010169910801E7C801F00001000C640E0C
:106070000801E56F00013FEC20F00101C4A108D048
:106080000D0E9EA8FED7AD6E0A0E9EA8FED7AD6E71
:1060900000016651645D1BE0CDDF01C0F0F4010139
:1060A000C4A10ED0F0C4E6F8570E0801E76F000156
:1060B00082EC29F0200E9EA8FED7AD6E07D001011C
:1060C000320E0801E56F00013FEC20F0E2D7000C32
:1060D000200E0801AEA9300EAF6FADC800F0ADAF15
:1060E00007D0001E002A00C0ADF82D0EAF6FAE8F96
:1060F00001501B6AF2BE1B8EF29EADC8E8FC640E16
:106100000C01E96F0001CFEC1AF01BBEF28E00C04B
:10611000ADF8300E01240801B06F1B6AF2BE1B8E71
:10612000F29EADC8E8FC0A0E0C01E96F0001CFEC4D
:106130001AF01BBEF28E300E00240801B26F300E32
:106140000124B16FAFC800F0AEA702D0AEAFAE95DC
:10615000AEB90BD0AEAF22D0AEB520D000C0B0F8F3
:10616000AEB31CD000C0B1F819D0300EB05D16E14E
:1061700000C0B0F8200EAF6FAEA704D0AE95AE83CE
:10618000AEAFAE93300EB15D09E100C0B1F8200EA4
:10619000B06FAEA7F7D7AE93AEAFAE91AEA504D0B9
:1061A000AF519EA8FED7AD6EAEA304D0B0519EA84D
:1061B000FED7AD6EAEA104D0B1519EA8FED7AD6E94
:1061C000B2519EA8FED7AD6E0001000CA4A8FED768
:1061D0006D6E000C0801D46BD56BD2C8E9FFD3C833
:1061E000EAFFEFCFD5F8D553D8B47DD00101C4A1D3
:1061F00008D00D0E9EA8FED7AD6E0A0E9EA8FED743
:10620000AD6E010E0801D46FD451D55D6CE3010170
:10621000C4A153D0D339006E0F0E001600500D08E4
:1062200034E1036A0801D451D225E96ED351032029
:10623000EA6EEF501F0812E2036AD451D225E96ECC
:10624000D3510320EA6EEFCFD6F8D6519EA8FED7E1
:10625000AD6E200E9EA8FED7AD6E15D0036AD45148
:10626000D225E96ED3510320EA6EEFCFD6F8D6C817
:10627000E6F8570EE76F000182EC29F0200E9EA889
:10628000FED7AD6E080117D00101036A0801D45191
:10629000D225E96ED3510320EA6EEFCFD6F8D6C8E7
:1062A000E6F8570EE76F000182EC29F0200E9EA859
:1062B000FED7AD6E080108D00101010E0801E56F9F
:1062C00000013FEC20F00801036AD451D225E96EA9
:1062D000D3510320EA6EEFCFD6F8D651000176DF16
:1062E0000801D42B91D70001000CEACFEDF8E9CFDB
:1062F000ECF80801E6AF08D0EC8FECA9EC2BE51F19
:10630000E61FE52BD8B4E62BE639F009E86FE8275D
:10631000E20FE96F320FEB6FE6510F0BE927E92728
:10632000EB27E90FEA6FEA27EA27E5390F0BEA279F
:10633000EB27EA37EB37EB1FEB37E5510F0BEB277A
:10634000E837070EE76F0A0EEA07EB27FDE3E907D8
:10635000EA27FDE3E807E927FDE3E707E827FDE390
:10636000080EEA6EE70EE96E070EEC15EC9DE906E5
:10637000EC1507E1ECB9E92AECB903D0200E006E68
:106380001CD0E926EB0EE95CD8B4EC8DEF50006E22
:1063900008E1ECBD06D0ECB914D0ECB702D0200E69
:1063A0000BD0ECAF06D02D0E006EED50EC9DEC9FA7
:1063B00004D0EC87EC99300E002600509EA8FED742
:1063C000AD6EEE50ECADDED70001000C0801C06BE5
:1063D000C16BC36BC26BC491010169B149D0C3C821
:1063E000E2FCC2C8E1FC0C01E46B320EE36F000179
:1063F00058EC29F002C0C6F801C0C5F80801B35135
:10640000025C2BE303E1B251C55D27E30101C4A1A6
:1064100020D0660EF66E260EF76E000EF86E170E82
:106420000801E56F000169EC29F0100EE96EB3C8B0
:10643000E6F8B2C8E5F859DF800EF66E260EF76E64
:10644000000EF86E070E0801E56F000169EC29F0F7
:106450000101000E016EF9D00801320EE56F000156
:106460003FEC20F00801C22BD8B4C32BB5D70101F3
:10647000080EEA6EB40EE96E0801E56BE76B0C0ED0
:10648000E66F00016BEC25F00101C4A11CD0880E61
:10649000F66E260EF76E000EF86E0F0E0801E56F11
:1064A000000169EC29F0100EE96EB3C8E6F8B2C835
:1064B000E5F81BDF290E9EA8FED7AD6E200E9EA824
:1064C000FED7AD6E010169A1C0D00001B3DD01C0EE
:1064D000C0F80801C4A169D0C03D37D00101C4A1F2
:1064E0000DD0C0C8E6F8370E0801E76F000182EC56
:1064F00029F0200E9EA8FED7AD6E01010801B5510E
:10650000410803E0B551420806E1010E016E0101A8
:106510009CD019D00801B551510803E0B55152087B
:106520000EE1080EEA6EB40EE96EE56BE76B0C0E39
:10653000E66F00016BEC25F00801C49105D0000E58
:10654000016E010182D008012FD0036AC151B40F3E
:10655000E96E080E0320EA6EC0C8EFFF0101C4A176
:1065600017D0036A0801C151B40FE96E080E032069
:10657000EA6EEFCFC5F8C5C8E6F8370EE76F000141
:1065800082EC29F0200E9EA8FED7AD6E07D0010147
:10659000320E0801E56F00013FEC20F00801C12B2D
:1065A000C1510B0801E2C49149D0C051900826E1C5
:1065B000C16B036AC151B40FE96E080E0320EA6E85
:1065C000C0C8EFFF0101C4A115D0036A0801C15181
:1065D000B40FE96E080E0320EA6EEFCFC5F8C5C808
:1065E000E6F8370EE76F000182EC29F0200E9EA836
:1065F000FED7AD6E0801C12BC48120D00101C4A11A
:1066000016D05B0E9EA8FED7AD6EC0C8E6F8370E5A
:106610000801E76F000182EC29F05D0E9EA8FED70D
:10662000AD6E200E9EA8FED7AD6E07D00101320ED2
:106630000801E56F00013FEC20F00801320EE56F24
:1066400000013FEC20F001013ED70001000C0801E1
:10665000D26B010169A10DD00001ECDC01C0D2F8C0
:106660000A0E0801D36F00012AEC20F00801F1D7CF
:1066700001010001000C060E08019D6F810E9E6F46
:10668000010E9F6F040EA06F070EA16FA26BFF0E8D
:10669000A36F090EA46F810EA56F010EA66F060EE3
:1066A000A76F010EA86FA96BAA6B030EAB6FAC6F3F
:1066B000FF0EAD6FB16B9A517F0BAE6F9B517F0B8D
:1066C000AF6F9C517F0BB06FAE5305E1010EAE6F03
:1066D000030EAB6F09D09A51800B800803E1010EC5
:1066E000AB6F02D0020EAB6FAEC8A9F8AF5305E195
:1066F000010EAF6F030EAC6F09D09B51800B800869
:1067000003E1010EAC6F02D0020EAC6FAFC8AAF865
:106710000101D339006E0F0E001600500A0807E081
:10672000D339006E0F0E001600500B0824E1D33948
:10673000006E0F0E001600500B08D8A471D0D89030
:1067400002011035036AEA0FE96E010E0320EA6EBA
:10675000ECCFB3F8ED52EFCFB2F80801B251020816
:10676000D8B402D0010107D0B32D01D002D001016D
:1067700002D0010155D00801AB51030803E1AC512F
:10678000030839E00101DF83080E0801D36FA40E6E
:10679000D26F00011FDD0101D339006E0F0E00160C
:1067A0000050010807E0D339006E0F0E00160050AC
:1067B000050809E1030E0801B36FE80EB26F00018E
:1067C00005DE16D00101D339006E0F0E0016005001
:1067D00003080FE1D2530DE00801B36BFA0EB26F5C
:1067E0000001F4DDD2C1B1F8B1C8E5F83FEC20F00A
:1067F000010114D008010101DFA310D0DF93080EBE
:106800000801D36FA40ED26F0001E4DC030E08016F
:10681000B36FE80EB26F0001D9DD0101000117DF8F
:106820000801B05302E1A26B0DD09C51800B80088F
:1068300005E1B051070B2009A26F04D0B051070B3E
:106840003009A26FA25337E0080ED36F9D0ED26FAE
:106850000001C0DC0101DF81D339006E0F0E00168C
:106860000050010807E0D339006E0F0E00160050EB
:10687000050809E1030E0801B36FE80EB26F0001CD
:10688000A5DD16D00101D339006E0F0E00160050A1
:1068900003080FE1D2530DE00801B36BFA0EB26F9B
:1068A000000194DDD2C1B1F8B1C8E5F83FEC20F0A9
:1068B000010114D008010101DFA110D0DF91080E01
:1068C0000801D36F9D0ED26F000184DC030E080116
:1068D000B36FE80EB26F000179DD01010001B7DE90
:1068E000000C0801D351090805E3300ED325016ED1
:1068F00005D004D0370ED325016E00D00001000C66
:106900000801E16BE36BE26BE491080EEA6ED40ED2
:10691000E96EE56BE76B0D0EE66F00016BEC25F0A1
:10692000010169B14AD0E3C8E2FCE2C8E1FC0C0114
:10693000E46B190EE36F000158EC29F002C0E6F891
:1069400001C0E5F80801D351025C2BE303E1D25109
:10695000E55D27E30101C4A120D0220EF66E270ECB
:10696000F76E000EF86E150E0801E56F000169EC78
:1069700029F0100EE96ED3C8E6F8D2C8E5F8B5DC08
:106980003A0EF66E270EF76E000EF86E070E08012F
:10699000E56F000169EC29F00101000E016EA3D042
:1069A0000801190EE56F00013FEC20F00801E22B11
:1069B000D8B4E32B0001B4D70101C4A10AD0420E20
:1069C000F66E270EF76E000EF86E0001B9EC2DF092
:1069D000010169A186D0036A0801E151D40F016E5B
:1069E000080E032201C0E5F803C0E6F800011AEC26
:1069F00030F0E6C8EAFFE5C8E9FF01C0EFFF01019A
:106A0000C4A115D0036A0801E151D40FE96E080E44
:106A10000320EA6EEFCFE5F8E5C8E6F8370EE76F3A
:106A2000000182EC29F0200E9EA8FED7AD6E080171
:106A3000E4B117D0036AE151D40FE96E080E0320C8
:106A4000EA6EEF50FE080CE1036AE151D40FE96EE3
:106A5000080E0320EA6EEFCFD4F8E481010EE16F57
:106A600035D0036AE151D40FE96E080E0320EA6EB7
:106A7000EF50EF081EE10101C4A108D00D0E9EA841
:106A8000FED7AD6E0A0E9EA8FED7AD6E0801D75197
:106A9000300809E1D851300806E1010E016E01010C
:106AA00022D005D00801000E016E01011CD006D0D5
:106AB0000801320EE56F00013FEC20F00801E151C2
:106AC0000B0802E3E12B02D0E16BE491010169B113
:106AD00007D0320E0801E56F00013FEC20F0010104
:106AE00078D7000E016E0001000C080E08019D6FA2
:106AF000FF0E9E6F300E9F6FA06FA16B600EA26F96
:106B0000300EA36FA46FEF0EA56F070EA66FFF0EDA
:106B1000A76F300EA86FA96FAA6BA20EAB6F300ED5
:106B2000AC6FEF0EAD6F090EAE6FFF0EAF6F300E94
:106B3000B06FB16FB26B500EB36FB46BB56BB66B19
:106B4000EF0EB76F090EB86FFF0EB96F300EBA6F48
:106B5000BB6FBC6B510EBD6FBE6BBF6BC06BEF0EDE
:106B6000C16F080EC26FFF0EC36F300EC46FC56FCA
:106B7000C66BB40EC76F310EC86FC96BEF0ECA6F0C
:106B80009A517F0BCB6F9B517F0BCC6F9C517F0B2E
:106B9000CD6FCD5316E104016A513008D8A402D05C
:106BA00008010FD0000153DD080E0801D36FA60EB7
:106BB000D26F0001EAEC30F0ACC86AF40101DF9159
:106BC0000801CB531DE1CC531BE10401685130088F
:106BD00006E169513008D8A402D0080111D00001A3
:106BE00036DD080E0801D36F9D0ED26F0001EAEC6E
:106BF00030F0A3C868F4A4C869F40101DF93080168
:106C0000CB5305E1CC5303E1CD5301E13CD1CB5350
:106C100003E1300EA36F09D09A51800B800803E185
:106C2000320EA36F02D0310EA36FCC5303E1300EAE
:106C3000A46F09D09B51800B800803E1310EA46F33
:106C400002D0320EA46F036ACCC8D2F803C0D3F8C6
:106C50000C01E26B1E0EE16F03C0E4FCCCC8E3FC48
:106C6000000158EC29F0080E08010124CE6F000E37
:106C70000220CF6F036ACBC8D2F803C0D3F80C014F
:106C8000E26B210EE16F03C0E4FCCBC8E3FC000122
:106C900058EC29F0080E08010124D06F000E0220E4
:106CA000D16FD15306E1D051090803E3D16B0A0E2D
:106CB000D06FD151020809E2FF0A03E1D051200848
:106CC00004E2030ED16F200ED06FCF5306E1CE51F8
:106CD000090803E3CF6B0A0ECE6FCF51010809E21A
:106CE000FF0A03E1CE516E0804E2020ECF6F6E0E72
:106CF000CE6FD1510F0BD26FD36F0001F2DD01C007
:106D0000B4F80801D0C800F0003A0F0E0016005089
:106D10000F0BD26FD36F0001E4DD01C0B5F808019D
:106D2000D0510F0BD26FD36F0001DBDD01C0B6F87D
:106D30000801CF510F0BD26FD36F0001D2DD01C01C
:106D4000BEF80801CEC800F0003A0F0E0016005041
:106D50000F0BD26FD36F0001C4DD01C0BFF8080173
:106D6000CE510F0BD26FD36F0001BBDD01C0C0F855
:106D70000801CB5318E0A351300815E00101DF836F
:106D80000801CB510101E05D0DE0CBC8E0F100014D
:106D90005EDC080E0801D36FAE0ED26F0001EAEC84
:106DA00030F001010801CC5318E0A451300815E07F
:106DB0000101DF830801CC510101E15D0DE0CCC888
:106DC000E1F1000144DC080E0801D36FB80ED26F68
:106DD0000001EAEC30F001010801A4510401695DF1
:106DE00005E10801A3510401685D0EE0A3C868F441
:106DF000A4C869F400012BDC080E0801D36F9D0EB6
:106E0000D26F0001EAEC30F00801CD533CE09C5118
:106E1000800B800803E1320EAC6F02D0310EAC6FF4
:106E20000101DF810801CD510101E25D18E0CDC80B
:106E3000E2F10801CD51070B3009C96F000107DCF1
:106E4000080E0801D36FC20ED26F0001EAEC30F0D9
:106E5000030E0801D36FE80ED26F000151DD080167
:106E6000AC5104016A5D0EE0ACC86AF4000127EC85
:106E700033F0080E0801D36FA60ED26F0001EAECC2
:106E800030F0040108010001000C8E0E006EBBC83A
:106E900001F0BAC802F0036A015209E102C001F030
:106EA000026A080E005E015202E1006A08D0D89022
:106EB00001BE04D0023601360006F9D7019E000C4F
:106EC0000801BA51D8B4A5D0C66FBE51D8B4A1D06C
:106ED000C65F05E37F0EC627D8B09BD006D0810ED3
:106EE000C65FD8A096D0D8B494D0C6C800F0016AC6
:106EF000026A036AC56BBBC8C4F8C48FBCC8C3F8B8
:106F0000BDC8C2F8190EC66FC151C25F0DE2010EB5
:106F1000C35F0AE2C45F08E2C55F06E2C52BC42B6B
:106F2000C32BC151C22728D0C051C35F12E2010E4A
:106F3000C45F0FE2C55F0DE2C52BC42BC051C32750
:106F4000C151C22719E3C32B17E1C42B15E1C52B8F
:106F500013D0BF518009C45F0EE2010EC55F0BE282
:106F6000C52BBF518009C427C051C327E9E3C42BF7
:106F7000E7E1C52BE5D70380C62F01D00BD0D89011
:106F8000C237C337C437C537D89003360236013607
:106F9000C737BAD7C7A106D0D89001320232033220
:106FA000C73302D0000635E0C7BF1ED0D890C23725
:106FB000C337C437C537C151C25F07E2010EC35F93
:106FC00004E2C45F02E2C55F1AE3C051C35F05E299
:106FD000010EC45F02E2C55F12E3BF518009C45FC6
:106FE00003E2010EC55F0BE3032A09E1022A07E170
:106FF000012A05E1002A0DE0013202320332BBC84A
:10700000C6F8BF51C61BC6AF02D0018E06D0019E86
:1070100004D0006A016A026A036A0001000C0801D8
:10702000BE51D8B471D0006EC251D8B46DD0002614
:1070300004E3810E002668E204D07F0E005E64E364
:1070400063E0BFC8C6F8C351C61BBF8FC38FC15111
:10705000C503F4CFC8F8C051C403F4CF03F0F3CF95
:10706000C7F8C503F350C827F450C723000E032206
:10707000C151C403F350C827F450C723000E026A5D
:1070800003220222BF51C503F350C727F450032245
:10709000000E0222BF51C403F3500326F450022213
:1070A000000E016A0122C151C303F350C727F450F7
:1070B0000322000E02220122C051C303F350032613
:1070C000F4500222000E0122BF51C303F3500226E6
:1070D000F4500122002A01BE05D0C737033602361C
:1070E00001360006000EC7AF0AD0032A0222012291
:1070F000015005E1025003E1035001E1002AC6BF3F
:10710000018EC6AF019E04D0006A016A026A036A5A
:107110000001000C8E0E006E0801BA51005EBBC863
:1071200002F0BCC801F0028E005209E0D890025271
:1071300002E1015204E002320132002EF7D7BBAF68
:1071400005D0011E021E012AD8B4022A0001000C3B
:107150000801D16BD26B010ED36FDA6AD96A080EBF
:10716000D66FC90ED56F080EEA6ECD0EE96ED6C881
:10717000E2FFD5C8E1FFD3C8D4F8D890E550EE02BD
:10718000F350D123F450D223D42FF7D7D1C8DEFF48
:10719000D2C8D1F8D26BD8B0D22BD52BD8B4D62B3D
:1071A000D32BD3510508DFE1000168EF39F0D8B2E5
:1071B00004D0080EEA6ED90EE96E0801D451D81930
:1071C000800BDE6FD4AF0BD0D11FD21FD31FD41FC3
:1071D000D12BD8B4D22BD8B4D32BD8B4D42BD8AF8E
:1071E0000BD0D51FD61FD71FD81FD52BD8B4D62B61
:1071F000D8B4D72BD8B4D82B006A016A026A036AC4
:10720000D96BDA6BDB6BDC6BD851D711D611D5118A
:107210002CE0200EDD6FD890D137D237D337D4375A
:10722000D937DA37DB37DC37D851DC5D08E1D751A5
:10723000DB5D05E1D651DA5D02E1D551D95D0FE3A1
:10724000D551D95FD651D8A0D63DDA5FD751D8A055
:10725000D73DDB5FD851D8A0D83DDC5FD880003661
:10726000013602360336DD2FD6D7DEAF0BD0001E37
:10727000011E021E031E002AD8B4012AD8B4022A15
:10728000D8B4032AD9C8EFFFDAC8ECFFDBC8ECFF9B
:10729000DCC8ECFF0001000C0801C46BC36BC26BBF
:1072A000010EC16FC66BC76BBDBF01D01AD0010EF6
:1072B000C66FBDC8CCF8BCC8CBF8BBC8CAF8BAC842
:1072C000C9F8FF0ED06FCF6FCE6FCD6F000140D7E2
:1072D00003C0BDF802C0BCF801C0BBF800C0BAF8DA
:1072E0000801C15306E1C25304E1C35302E1C45390
:1072F0006DE0D892BDC8D4F8BCC8D3F8BBC8D2F8EA
:10730000BAC8D1F8D86BD76BD66BBEC8D5F8000118
:107310004EDF03C0C4F802C0C3F801C0C2F800C009
:10732000C1F8036A0801C751BF25016EC05103228D
:1073300001C0C9F803C0CAF8EACFCCF8E9CFCBF84E
:10734000D882080EEA6ECD0EE96EBDC8D4F8BCC86E
:10735000D3F8BBC8D2F8BAC8D1F8D86BD76BD66B04
:10736000BEC8D5F8000123DFCCC8EAFFCBC8E9FFCF
:10737000300E0801CD25006E000ECE21000ECF216B
:10738000000ED021CAC8EAFFC9C8E9FF00C0EFFF5C
:10739000036AC751BF25E96EC0510320EA6EEF5062
:1073A00039080AE2036AC751BF25E96EC0510320BC
:1073B000EA6E070EEF24EF6EC72BC4C8BDF8C3C832
:1073C000BCF8C2C8BBF8C1C8BAF88BD7C62D0AD062
:1073D000036AC751BF25E96EC0510320EA6E2D0E26
:1073E000EF6EC72BC56BD890C731C55D2FE2036A1E
:1073F000C551BF25E96EC0510320EA6EEFCFC8F832
:10740000036AC551BF25016EC051032203C0CAF8EB
:10741000C551C75DFF0F036ABF25E96EC051032048
:10742000EA6EEFCFCBF8CAC8EAFF01C0E9FFCBC8CC
:10743000EFFFC551C75DFF0F036ABF25E96EC0515D
:107440000320EA6EC8C8EFFFC52BCDD7036AC7512A
:10745000BF25E96EC0510320EA6EEF6ABFC801F094
:10746000C0C802F00001000C0801A06B9F6B9E6B6E
:107470009D6B050EA16F230EA26F500EA36F300EF1
:10748000A46FA56F0D0EA66F050EA76F230EA86F34
:10749000540EA96F300EAA6FAB6F0D0EAC6F050EB8
:1074A000AD6F230EAE6F5A0EAF6F300EB06FB16F6F
:1074B0000D0EB26F9A517F0BB36FB35101084BE2BF
:1074C000BB6BB3C8BAF80001E0DC03C0A0F802C08F
:1074D0009FF801C09EF800C09DF8A0C8BDF89FC8E5
:1074E000BCF89EC8BBF89DC8BAF80801C16BC06B58
:1074F000400EBF6F830EBE6F0001E2DC00C0BAF821
:1075000001C0BBF802C0BCF803C0BDF803C0C1F89D
:1075100002C0C0F801C0BFF800C0BEF80801C56BCA
:10752000C46B440EC36F840EC26F000178DD03C0CC
:10753000A0F802C09FF801C09EF800C09DF8A0C846
:10754000BDF89FC8BCF89EC8BBF89DC8BAF8E2DD7C
:1075500001C0B3F808019B517F0BB46FB45101080F
:107560004BE2BB6BB4C8BAF800018FDC03C0A0F8D3
:1075700002C09FF801C09EF800C09DF8A0C8BDF8E9
:107580009FC8BCF89EC8BBF89DC8BAF80801C16B7B
:10759000C06B200EBF6F830EBE6F000191DC00C078
:1075A000BAF801C0BBF802C0BCF803C0BDF803C004
:1075B000C1F802C0C0F801C0BFF800C0BEF80801A1
:1075C000C56BC46B440EC36F840EC26F000127DD10
:1075D00003C0A0F802C09FF801C09EF800C09DF84B
:1075E000A0C8BDF89FC8BCF89EC8BBF89DC8BAF833
:1075F00091DD01C0B4F808019C51770BB56FB5510E
:10760000070B01084CE2B551070BBB6BBA6F0001C9
:107610003CDC03C0A0F802C09FF801C09EF800C087
:107620009DF8A0C8BDF89FC8BCF89EC8BBF89DC80F
:10763000BAF80801C16BC06B600EBF6F810EBE6FE0
:1076400000013EDC00C0BAF801C0BBF802C0BCF8C3
:1076500003C0BDF803C0C1F802C0C0F801C0BFF844
:1076600000C0BEF80801C56BC46B440EC36F840E26
:10767000C26F0001D4DC03C0A0F802C09FF801C0B3
:107680009EF800C09DF8A0C8BDF89FC8BCF89EC871
:10769000BBF89DC8BAF83EDD01C0B5F80801080E78
:1076A000EA6EB60EE96EE56BE76B040EE66F00015D
:1076B0006BEC25F00801B35305E1350EA46F300ED5
:1076C000A56F66D09A51800B800833E1320ED880C6
:1076D000B357BD6BBC6BBB6BB3C8BAF80A0EBE6FB9
:1076E000080EC06FB60EBF6F0001D6DD02C0BBF83A
:1076F00001C0BAF80801BA5302E1BB5313E0080E07
:10770000D36FB60ED26F0001EBEC20F001500108F0
:1077100005E2B6C8A4F8B7C8A5F802D0B6C8A5F85F
:1077200006D00801350EA46F300EA56F000131D0D0
:107730000801320EB327BD6BBC6BBB6BB3C8BAF884
:107740000A0EBE6F080EC06FB60EBF6F0001A4DD3B
:1077500002C0BBF801C0BAF80801BA5302E1BB533A
:1077600013E0080ED36FB60ED26F0001EBEC20F0E1
:107770000150010805E2B6C8A4F8B7C8A5F802D0C0
:10778000B6C8A5F806D00801350EA46F300EA56F57
:107790000001080E0801D36FA10ED26F0001EAECC0
:1077A00030F027EC33F00801B45305E1350EAA6F31
:1077B000300EAB6F66D09B51800B800832E1320EE9
:1077C000B427BD6BBC6BBB6BB4C8BAF80A0EBE6FF6
:1077D000080EC06FB60EBF6F00015EDD02C0BBF8C1
:1077E00001C0BAF80801BA5302E1BB5313E0080E16
:1077F000D36FB60ED26F0001EBEC20F00150010800
:1078000005E2B6C8AAF8B7C8ABF802D0B6C8ABF85C
:1078100006D00801350EAA6F300EAB6F000132D0D2
:107820000801320ED880B457BD6BBC6BBB6BB4C8BB
:10783000BAF80A0EBE6F080EC06FB60EBF6F000119
:107840002BDD02C0BBF801C0BAF80801BA5302E14F
:10785000BB5313E0080ED36FB60ED26F0001EBECF2
:1078600020F00150010805E2B6C8AAF8B7C8ABF885
:1078700002D0B6C8ABF806D00801350EAA6F300E9C
:10788000AB6F0001080E0801D36FA70ED26F000185
:10789000EAEC30F027EC33F00801B55305E1350E82
:1078A000B06F300EB16F66D09C51800B800832E112
:1078B000320EB527BD6BBC6BBB6BB5C8BAF80A0EF0
:1078C000BE6F080EC06FB60EBF6F0001E5DC02C0D0
:1078D000BBF801C0BAF80801BA5302E1BB5313E088
:1078E000080ED36FB60ED26F0001EBEC20F0015002
:1078F000010805E2B6C8B0F8B7C8B1F802D0B6C8FA
:10790000B1F806D00801350EB06F300EB16F00012E
:1079100032D00801320ED880B557BD6BBC6BBB6B43
:10792000B5C8BAF80A0EBE6F080EC06FB60EBF6FAC
:107930000001B2DC02C0BBF801C0BAF80801BA53BA
:1079400002E1BB5313E0080ED36FB60ED26F0001F5
:10795000EBEC20F00150010805E2B6C8B0F8B7C85A
:10796000B1F802D0B6C8B1F806D00801350EB06F34
:10797000300EB16F0001080E0801D36FAD0ED26F4B
:107980000001EAEC30F027EC33F0000C6B50060BF2
:1079900029E00101C4A11DD0460EF66E3E0EF76E21
:1079A000000EF86E160E0801E56F000169EC29F073
:1079B0006BCFE6F8570E0801E76F000182EC29F063
:1079C0000A0E9EA8FED7AD6E0D0E9EA8FED7AD6E18
:1079D00001016B6A010E0801D36F00012AEC20F04F
:1079E000900E6B6E3AEF3DF04990499C499E010123
:1079F000D339006E0F0E00160050FF0FF10F1EE27C
:107A00000F0F000164EF3DF008019A6B9B6B9C6BBC
:107A100000013BEC33F0010111D008019A6B9B6B24
:107A20009C6B000175EC35F0010108D008019A6BE0
:107A30009B6B9C6B000118DD010100D005010DB1AD
:107A400002D08D9601D08D8696960DB302D08D987A
:107A500001D08D8896980DB502D08D9A01D08D8A6F
:107A6000969A050E0801E56F00013FEC20F027EC27
:107A700033F08CD70DC510F2036A05010D51E30FE9
:107A8000E96E010E0320EA6EEFCFD3F10101D89029
:107A900005010D35036AF80FE96E010E0320EA6E49
:107AA000ECCF03F0ED52EFCFDDF1010103C0DEF1C9
:107AB000D46BD66BD56BD86BD76BDA6BD96BDC6BB1
:107AC000DB6BDF6B0001000CE824F76AF736E90F87
:107AD000F66E7A0EF722000EF86EFB6E0A00F55075
:107AE000FA6E0800F550F96E087A087A087A087A72
:107AF000087A087A087A087A087A087A087A1A7A64
:107B00002C7A087A087A070E0501716FFF0E726FE2
:107B1000300E736F746F756BA50E766F3C0E776FBA
:107B2000EF0E786F070E796FFF0E7A6F300E7B6F56
:107B30007C6F7D6BB40E7E6F300E7F6FEF0E806FAB
:107B4000060E816FFF0E826F300E836F846F856B20
:107B5000630E866FEF0E876F070E886FFF0E896FBB
:107B6000300E8A6F8B6F8C6BB10E8D6F300E8E6FF7
:107B7000EF0E8F6F070E906FFF0E916F300E926FAA
:107B8000936F946B900E956F300E966FEF0E976F0C
:107B9000070E986FFF0E996F300E9A6F9B6F9C6B5C
:107BA000A00E9D6F310E9E6FEF0E9F6F070EA06FA0
:107BB000FF0EA16F300EA26FA36FA46BA00EA56F76
:107BC000300EA66FEF0EA76F070EA86FFF0EA96FFE
:107BD000300EAA6FAB6FAC6BA50EAD6F310EAE6FF2
:107BE000EF0EAF6F070EB06FFF0EB16F300EB26FBA
:107BF000B36FB46BA50EB56F300EB66FEF0EB76FE7
:107C0000070EB86FFF0EB96F300EBA6FBB6FBC6B4B
:107C1000A70EBD6F300EBE6FEF0EBF6F070EC06FA9
:107C2000FF0EC16F300EC26FC36FC46BA70EC56F5E
:107C3000310EC66FEF0EC76F070EC86FFF0EC96F0C
:107C4000300ECA6FCB6FCC6BA70ECD6F310ECE6FDF
:107C5000EF0ECF6F070ED06FFF0ED16F300ED26FC9
:107C6000D36FD46BA50ED56F320ED66FEF0ED76FD4
:107C7000070ED86FFF0ED96F300EDA6FDB6FDC6B3B
:107C8000A50EDD6F320EDE6FEF0EDF6F090EE06FB7
:107C9000FF0EE16F300EE26FE36FE46BA50EE56F50
:107CA0003B0EE66FE76BE86BEF0EE96F080EEA6FCD
:107CB000FF0EEB6F300EEC6FED6FEE6BA50EEF6FFE
:107CC000340EF06F300EF16FEF0EF26F070EF36FA0
:107CD000FF0EF46F300EF56FF66FF76BA10EF86FB5
:107CE000300EF96FEF0EFA6F070EFB6FFF0EFC6F91
:107CF000300EFD6FFE6FFF6BA10E0601006F310E9F
:107D0000016FEF0E026F070E036FFF0E046F300E50
:107D1000056F066F076BA10E086F330E096FEF0E2C
:107D20000A6F070E0B6FFF0E0C6F300E0D6F0E6F8C
:107D30000F6BA10E106F320E116FEF0E126F070E48
:107D4000136FFF0E146F300E156F166F176BA10EA9
:107D5000186F310E196FEF0E1A6F060E1B6FFF0EA4
:107D60001C6F300E1D6F1E6F1F6B570E206FEF0EB6
:107D7000216F070E226FFF0E236F300E246F256FC9
:107D8000266B890E276F286BEF0E296F2B6B2A6BE2
:107D900005016F51340A0001D8B497D0350AD8B420
:107DA0009DD0030AD8B49BD0010AD8B499D0070A51
:107DB000D8B497D0010AD8B495D0030AD8B493D0D8
:107DC0000E0AD8B491D0010AD8B497D0030AD8B417
:107DD0009DD00D0AD8B4A3D00A0AD8B4A9D0030AFA
:107DE000D8B4AFD0010AD8B4B5D01F0AD8B4BBD02C
:107DF000010AD8B4C1D0030AD8B4C7D0010AD8B494
:107E0000CDD0250AD8B4D3D0030AD8B4E1D00C0A17
:107E1000D8B4EFD0230AD8B4EDD0030AD8B4F6D042
:107E20000D0AD8B4F4D0010AD8B4FAD0030AD8B4F1
:107E300011D1010AD8B414D10F0AD8B417D1040A49
:107E4000D8B451D1010AD8B457D1030AD8B45DD1FE
:107E5000010AD8B463D13F0AD8B469D1010AD8B4B1
:107E60006FD1050AD8B46DD1010AD8B477D1030A0D
:107E7000D8B481D1010AD8B486D10F0AD8B484D13C
:107E8000010AD8B48ED1030AD8B494D1010AD8B467
:107E90009FD1070AD8B4A5D1010AD8B4A3D1030A47
:107EA000D8B4A1D1010AD8B49FD11F0AD8B49DD1AA
:107EB000020AD8B4A2D1010AD8B4A8D1080AD8B409
:107EC000A6D1070AD8B4A4D1A4D1050E0801D36F56
:107ED000900ED26F0001EAEC30F09FD19ED19DD17F
:107EE0009CD19BD19AD199D1050E0801D36F710E07
:107EF000D26F0001EAEC30F090D1050E0801D36F8B
:107F0000790ED26F0001EAEC30F087D1050E08013E
:107F1000D36F810ED26F0001EAEC30F07ED1050EF6
:107F20000801D36F880ED26F0001EAEC30F075D1F2
:107F3000050E0801D36F980ED26F0001EAEC30F005
:107F40006CD1050E0801D36FA00ED26F0001EAECD0
:107F500030F063D1050E0801D36FA80ED26F000177
:107F6000EAEC30F05AD1050E0801D36FB00ED26F93
:107F70000001EAEC30F051D1050E0801D36FB80EC4
:107F8000D26F0001EAEC30F048D1050E0801D36F42
:107F9000C00ED26F0001EAEC30F03FD1050E0801AF
:107FA000D36FC80ED26F0001EAEC30F036D1020177
:107FB00011510F0B30090601286F8A0E276F060E2C
:107FC0000801D36F220ED26F0001EAEC30F025D108
:107FD000020111510F0B30090601286F890E276F1E
:107FE000060E0801D36F220ED26F0001EAEC30F0CA
:107FF00014D113D1300E0501F16F050E0801D36FB6
:10800000EA0ED26F0001EAEC30F007D106D1050E7E
:108010000801D36FD80ED26F0001EAEC30F0FDD02A
:10802000050E0801D36FD00ED26F0001EAEC30F0DC
:10803000640E0801E56F00013FEC20F0300E0501F1
:10804000F16F050E0801D36FEA0ED26F0001EAEC62
:1080500030F0E3D0020E0101DD27000EDE23000127
:108060000101DD51D8B4DE07DD0700010101DE5357
:1080700007E1DD510F0804E3DE6B100EDD6F06D063
:10808000DE51000803E2DE6BFF0EDD6FDEC12BF672
:10809000DDC12AF606012B312D6F2A312C6F2D33CD
:1080A0002C332D332C332D332C330F0E2D172CC6A0
:1080B000D3F8000171EC34F001C0E7F506012A5154
:1080C0000F0B2C6F2D6BE8CFD3F8000171EC34F05F
:1080D00001C0E8F5050E0801D36FE00ED26F000174
:1080E000EAEC30F09AD0050E0801D36FF30ED26F90
:1080F0000001EAEC30F091D0050E0801D36FFB0EC1
:10810000D26F0001EAEC30F088D0060E0801D36F80
:10811000030ED26F0001EAEC30F07FD0060E0801AA
:10812000D36F0B0ED26F0001EAEC30F076D0060E62
:108130000801D36F130ED26F0001EAEC30F06DD05E
:108140006CD00101CC51880906012C6F08019A6B93
:108150009B6B9C6F000175EC35F05FD00101CC5139
:10816000080906012C6F08019A6B9B6B9C6F00013C
:1081700075EC35F052D008019A6B9B6B9C6B00013B
:1081800075EC35F04AD049D00101C851800906018B
:108190002C6F08019A6B9B6F9C6B000175EC35F09E
:1081A0003CD008019A6BC8C19BF89C6B000175EC30
:1081B00035F033D00101C951800906012C6FE8CF99
:1081C0009AF808019B6B9C6B000175EC35F025D08B
:1081D000C9C19AF808019B6B9C6B000175EC35F0E6
:1081E0001CD01BD01AD019D018D008019A6B9B6BE9
:1081F0009C6B000175EC35F010D0060E0801D36FB2
:108200001B0ED26F0001EAEC30F007D006D005D08B
:1082100004D0000E016E0FD000D00501702D09D0E2
:10822000070E0801D36FD00ED26F000180EC34F03E
:108230000501010E016E0001000C05010F6B206BA2
:10824000FE0E216F236B226B010169B134D023C56F
:10825000E2FC22C5E1FC0C01E46B320EE36F00018D
:1082600058EC29F002C025F501C024F505010250A3
:10827000060815E2FF0A03E12451CF0810E20101CC
:10828000C4A10AD04E0EF66E240EF76E000EF86EE4
:108290000001B9EC2DF00101000E016E7ED0320E0E
:1082A0000801E56F00013FEC20F00501222BD8B456
:1082B000232BCAD70101050EEA6E100EE96E0801E4
:1082C000E56BE76BE66F00016BEC25F00101C4A1E3
:1082D0000AD0720EF66E240EF76E000EF86E0001D4
:1082E000B9EC2DF0010169A13DD0050120510F0825
:1082F000D8B002D0010136D000011AEC30F001C034
:108300000FF50A0E0801E56F00013FEC20F00101B6
:10831000C4A10ED00FC5E6F8370E0801E76F0001C3
:1083200082EC29F0200E9EA8FED7AD6E07D0010189
:10833000320E0801E56F00013FEC20F005012151EC
:108340000F5D04E1206B0FC510F50AD0202B036AE6
:108350002051100FE96E050E0320EA6E0FC5EFFFE6
:108360000101C1D705011051FE0813E1036A205134
:10837000100FE96E050E0320EA6EEF50EF0809E1D9
:108380002051050806E1010E016E010106D005D05D
:108390000501000E016E010100D00001F3EF63F052
:1083A0000601446B456B476B466B4891489301014E
:1083B00069B14AD047C6E2FC46C6E1FC0C01E46B59
:1083C000320EE36F000158EC29F002C04AF601C0FA
:1083D00049F606013751025C2BE303E13651495D52
:1083E00027E30101C4A121D09E0EF66E260EF76E82
:1083F000000EF86E140E0801E56F000169EC29F01B
:10840000100EE96E37C6E6F836C6E5F875EC31F0C1
:10841000B50EF66E260EF76E000EF86E070E08010A
:10842000E56F000169EC29F00101000E016E08D230
:10843000320E0801E56F00013FEC20F00601462BEB
:10844000D8B4472BB4D70101060EEA6E380EE96E98
:108450000801E56BE76B0C0EE66F00016BEC25F095
:108460000101C4A10AD0BE0EF66E260EF76E000EF4
:10847000F86E0001B9EC2DF0010169A1E1D1000114
:108480001AEC30F001C044F6060148A381D1443D06
:108490001DD10101C4A10DD044C6E6F8370E080174
:1084A000E76F000182EC29F0200E9EA8FED7AD6E8A
:1084B000010106013851880803E03851810810E1B4
:1084C0000101C4A108D00D0E9EA8FED7AD6E0A0E04
:1084D0009EA8FED7AD6E010E016EB2D1F5D0060199
:1084E0003951510804E039515208D8A47ED0010115
:1084F000C4A108D00D0E9EA8FED7AD6E0A0E9EA890
:10850000FED7AD6E060148A106D0010E016E010135
:1085100097D169D006010101C4A10AD0CC0EF66E34
:10852000260EF76E000EF86E0001B9EC2DF0010179
:10853000060EEA6E380EE96E0801E56BE76B0C0E6D
:10854000E66F00016BEC25F006014893010169B16B
:108550004AD047C6E2FC46C6E1FC0C01E46B320E91
:10856000E36F000158EC29F002C04AF601C049F659
:1085700006013751025C2BE303E13651495D27E3E5
:108580000101C4A121D0DA0EF66E260EF76E000EA0
:10859000F86E090E0801E56F000169EC29F0100E74
:1085A000E96E37C6E6F836C6E5F875EC31F0E60E4A
:1085B000F66E260EF76E000EF86E070E0801E56FD8
:1085C000000169EC29F00101000E016E39D1320E73
:1085D0000801E56F00013FEC20F00601462BD8B4FE
:1085E000472BB4D7010170D006013951410803E08F
:1085F0003951420868E148810101C4A10AD0EE0E58
:10860000F66E260EF76E000EF86E0001B9EC2DF036
:108610000101060EEA6E380EE96E0801E56BE76BA4
:108620000C0EE66F00016BEC25F00601489301018A
:1086300069B14AD047C6E2FC46C6E1FC0C01E46BD6
:10864000320EE36F000158EC29F002C04AF601C077
:1086500049F606013751025C2BE303E13651495DCF
:1086600027E30101C4A121D0FC0EF66E260EF76EA1
:10867000000EF86E090E0801E56F000169EC29F0A3
:10868000100EE96E37C6E6F836C6E5F875EC31F03F
:10869000080EF66E270EF76E000EF86E070E080134
:1086A000E56F000169EC29F00101000E016EC8D0F0
:1086B000320E0801E56F00013FEC20F00601462B69
:1086C000D8B4472BB4D7010161D00601036A4551E4
:1086D000380FE96E060E0320EA6E44C6EFFF010173
:1086E000C4A118D0036A06014551380FE96E060E81
:1086F0000320EA6EEFCF49F649C6E6F8370E0801C7
:10870000E76F000182EC29F0200E9EA8FED7AD6E27
:1087100007D00101320E0801E56F00013FEC20F0A7
:108720000601452B45510B0802E248932ED03851E3
:1087300090082BE14551020828E13951410A000116
:108740000FE0030A0DE0120A0BE0010A09E0030A38
:1087500007E0320A05E0010A03E0030A01E001D064
:1087600013D0060148930101C4A109D0100EF66E82
:10877000270EF76E000EF86E0001B9EC2DF0060121
:10878000476B466B000100D00601010151D0060184
:108790004451900806E04451810803E044518808A0
:1087A00027E1456B036A4551380FE96E060E032039
:1087B000EA6E44C6EFFF0101C4A116D0036A0601A8
:1087C0004551380FE96E060E0320EA6EEFCF49F6E9
:1087D00049C6E6F8370E0801E76F000182EC29F080
:1087E000200E9EA8FED7AD6E0601452B488320D0F3
:1087F0000101C4A116D05B0E9EA8FED7AD6E44C683
:10880000E6F8370E0801E76F000182EC29F05D0EF3
:108810009EA8FED7AD6E200E9EA8FED7AD6E07D0E7
:108820000101320E0801E56F00013FEC20F0060166
:10883000320E0801E56F00013FEC20F001011DD66A
:108840000001000C050E0501716F810E726F090E9B
:10885000736F746B020E756FFF0E766F050E776F78
:10886000810E786F090E796F040E7A6F4E0E7B6F52
:10887000FF0E7C6F050E7D6F810E7E6F090E7F6F80
:10888000040E806F470E816FFF0E826F050E836F9F
:10889000810E846F090E856F060E866F120E876F2C
:1088A000FF0E886F050E896F810E8A6F090E8B6F20
:1088B000040E8C6F480E8D6FFF0E8E6F090E8F6F3A
:1088C000810E906F010E916F040E926F4E0E936F9A
:1088D000946B956B966B976BFF0E986F060E996F66
:1088E000FF0E9A6F880E9B6F010E9C6F9D6B9E6FA3
:1088F000FF0E9F6F060EA06F810EA16F010EA26F7B
:10890000060EA36FA46F020EA56FFF0EA66F060ED4
:10891000A76F810EA86F010EA96F060EAA6FAB6F2D
:10892000030EAC6FFF0EAD6F060EAE6F810EAF6F14
:10893000010EB06F040EB16FB26B020EB36FFF0E7B
:10894000B46F060EB56F810EB66F010EB76F040ED1
:10895000B86FB96B030EBA6FFF0EBB6F060EBC6F1C
:10896000810EBD6F010EBE6F040EBF6F390EC06F5A
:10897000C16BFF0EC26F060EC36F810EC46F010E76
:10898000C56F040EC66F330EC76F020EC86FFF0EA1
:10899000C96F060ECA6F810ECB6F010ECC6F040E2D
:1089A000CD6F330ECE6F030ECF6FFF0ED06F060E5E
:1089B000D16F810ED26F010ED36F040ED46F350EBE
:1089C000D56FD66BFF0ED76F060ED86F810ED96F9D
:1089D000010EDA6F040EDB6F350EDC6F030EDD6FF8
:1089E000FF0EDE6F060EDF6F810EE06F010EE16F8E
:1089F000040EE26F3E0EE36F020EE46FFF0EE56FB2
:108A0000060EE66F810EE76F010EE86F040EE96F48
:108A10003E0EEA6F030EEB6FFF0EEC6F060EED6F6E
:108A2000810EEE6F010EEF6F040EF06F380EF16FD6
:108A3000020EF26FFF0EF36F060EF46F810EF56FEC
:108A4000010EF66F040EF76F380EF86F030EF96F14
:108A5000FF0EFA6F060EFB6F810EFC6F010EFD6FAD
:108A6000040EFE6F080EFF6F210E0601006FFF0E51
:108A7000016F060E026F810E036F010E046F040E6C
:108A8000056F080E066F310E076FFF0E086F060E9A
:108A9000096F810E0A6F010E0B6F040E0C6F080E2A
:108AA0000D6F0E6BFF0E0F6F050E106F810E116FA5
:108AB000010E126F060E136F040E146FFF0E156F6A
:108AC000050E166F810E176F010E186F060E196FC7
:108AD000050E1A6FFF0E1B6F070E1C6F810E1D6FA8
:108AE000010E1E6F040E1F6F3F0E206F010E216FCF
:108AF000226BFF0E236F050E246F810E256F010E72
:108B0000266F040E276F480E286FFF0E296F050E83
:108B10002A6F890E2B6F010E2C6F2D6F030E2E6F97
:108B2000FF0E2F6F050E306F810E316F090E326F01
:108B3000070E336F220E346FFF0E356F05016F5134
:108B4000010A0001D8B4A9D0030AD8B4A7D0400ABA
:108B5000D8B4ADD0410AD8B4B8D0070AD8B4B6D08A
:108B6000010AD8B4B4D0030AD8B4B2D00E0AD8B42B
:108B7000B0D0010AD8B4B6D0030AD8B4BCD00D0A1C
:108B8000D8B4C2D00C0AD8B4C8D0070AD8B4CED052
:108B90000C0AD8B4D4D00D0AD8B4DAD0030AD8B4A9
:108BA000E0D0150AD8B4E6D0140AD8B4ECD01F0A25
:108BB000D8B4F2D0010AD8B4F8D0020AD8B4FED0A2
:108BC000070AD8B40FD1010AD8B415D1030AD8B412
:108BD0001BD1010AD8B41ED10F0AD8B421D1040A7E
:108BE000D8B4D0D1010AD8B4D6D1030AD8B4DCD1D4
:108BF000010AD8B4F1D13F0AD8B406D2010AD8B4D8
:108C00000CD21B0AD8B40AD20C0AD8B410D2030A68
:108C1000D8B41ED20D0AD8B42CD20F0AD8B43AD286
:108C20000E0AD8B448D2020AD8B446D2070AD8B439
:108C300047D2180AD8B448D2010AD8B452D2030A8B
:108C4000D8B45CD2010AD8B461D20F0AD8B467D2C2
:108C5000010AD8B471D2030AD8B477D2010AD8B4C1
:108C600082D2070AD8B488D2010AD8B499D2030AAA
:108C7000D8B4A5D2010AD8B4B1D21F0AD8B4B8D298
:108C8000010AD8B4BDD2030AD8B4C3D2010AD8B4F9
:108C9000C9D20E0AD8B4CFD2D7D2DAD2050E080183
:108CA000D36F710ED26F0001EAEC30F0D1D2080E12
:108CB0000501746F0E0E756F050E0801D36F710EEE
:108CC000D26F0001EAEC30F0C3D2C2D2C1D2C0D21E
:108CD000BFD2050E0801D36F770ED26F0001EAEC08
:108CE00030F0B6D2050E0801D36F7D0ED26F0001B1
:108CF000EAEC30F0ADD2050E0801D36F830ED26FCF
:108D00000001EAEC30F0A4D2050E0801D36F890E01
:108D1000D26F0001EAEC30F09BD2050E0801D36F50
:108D2000A00ED26F0001EAEC30F092D2050E0801DD
:108D3000D36FA70ED26F0001EAEC30F089D2050E96
:108D40000801D36F990ED26F0001EAEC30F080D2A7
:108D5000050E0801D36FAE0ED26F0001EAEC30F0C1
:108D600077D2050E0801D36FB50ED26F0001EAEC81
:108D700030F06ED2050E0801D36FBC0ED26F000129
:108D8000EAEC30F065D2050E0801D36FC30ED26F46
:108D90000001EAEC30F05CD2050E0801D36FCA0E78
:108DA000D26F0001EAEC30F053D2050E0801D36F08
:108DB000D10ED26F0001EAEC30F04AD20101D33972
:108DC000006E0F0E001600500B0803E1050E0501A2
:108DD000DD6F050E0801D36FD80ED26F0001EAECEB
:108DE00030F036D2050E0801D36FDF0ED26F0001CE
:108DF000EAEC30F02DD2050E0801D36FE60ED26FEB
:108E00000001EAEC30F024D2020E0101DD27000E51
:108E1000DE2300010101DD51D8B4DE07DD070001CA
:108E20000101D339006E0F0E001600500B08D8A4B4
:108E30007AD0D89002011035036AEA0FE96E010E6C
:108E40000320EA6EEF50006EE92AEF50E906036E48
:108E5000020E035C05E1010E005C000127E0020147
:108E6000020E035C04E10052000134E00201030E33
:108E7000035C04E10052000141E00201010E035CC9
:108E800004E1005200013AE00201010E035C05E139
:108E9000010E005C000132E00201010E035C05E1FD
:108EA000020E005C00012AE0020128D00101DEBFB1
:108EB00005D0DE5306E1DD51000803E3DE6BDD6B18
:108EC00008D0DE5303E1DD51130803E2DE6B140E1C
:108ED000DD6F28D00101DEBF05D0DE5306E1DD5194
:108EE000000803E3DE6BDD6B08D0DE5303E1DD51E8
:108EF0000A0803E2DE6B0B0EDD6F14D00101DEBF4A
:108F000005D0DE5306E1DD51000803E3DE6BDD6BC7
:108F100008D0DE5303E1DD51100803E2DE6B110ED1
:108F2000DD6F00D011D0DE5307E1DD51010804E30D
:108F3000DE6B010EDD6F08D0DE5303E1DD510D085D
:108F400003E2DE6B0E0EDD6FDE31036EDD31026E8D
:108F50000332023203320232033202320F0E0316A0
:108F600002C096F505010101DD510F0BE8CF97F521
:108F70000501050E0801D36F8F0ED26F0001EAECD8
:108F800030F066D1050E0801D36FED0ED26F0001EF
:108F9000EAEC30F05DD1050E0801D36FF40ED26F0C
:108FA0000001EAEC30F054D10101D339006E0F0E0C
:108FB00000160050060804E1020E0601006F03D0FF
:108FC000200E0601006F050E0801D36FFB0ED26F55
:108FD0000001EAEC30F03CD10101D339006E0F0EF4
:108FE00000160050060804E1030E0601076F03D0C7
:108FF000300E0601076F060E0801D36F020ED26F06
:109000000001EAEC30F024D1060E0801D36F090EFE
:10901000D26F0001EAEC30F01BD11AD1060E080124
:10902000D36F2A0ED26F0001EAEC30F011D1010E9D
:109030000201115D0F0B0601226F020E216F060E59
:109040000801D36F1C0ED26F0001EAEC30F000D1A2
:10905000010E0201115D0F0B0601226F010E216F3F
:10906000060E0801D36F1C0ED26F0001EAEC30F03F
:10907000EFD0010E0201115D0F0B0601226F040EED
:10908000216F060E0801D36F1C0ED26F0001EAECAF
:1090900030F0DED0010E0201115D0F0B0601226FD0
:1090A000030E216F060E0801D36F1C0ED26F000154
:1090B000EAEC30F0CDD0CCD0010E016ED7D0C8D0C4
:1090C000010E016ED3D0C4D00101CC518809060134
:1090D000366F08019A6B9B6B9C6F00013BEC33F081
:1090E000B7D00101CC5108090601366F08019A6B0F
:1090F0009B6B9C6F00013BEC33F0AAD008019A6B8C
:109100009B6B9C6B00013BEC33F0A2D008019A6B87
:109110009B6BCCC19CF800013BEC33F099D0010172
:10912000C85180090601366F08019A6B9B6F9C6BD2
:1091300000013BEC33F08CD008019A6BC8C19BF85E
:109140009C6B00013BEC33F083D00101C9518009D5
:109150000601366FE8CF9AF808019B6B9C6B000103
:109160003BEC33F075D0C9C19AF808019B6B9C6B3E
:1091700000013BEC33F06CD00101C95180090601BC
:10918000366F0101C85180090601376F36C69AF85B
:10919000E8CF9BF808019C6B00013BEC33F058D002
:1091A0000101C85180090601366FC9C19AF8E8CF9C
:1091B0009BF808019C6B00013BEC33F049D00101A6
:1091C000C95180090601366FE8CF9AF8C8C19BF8EB
:1091D00008019C6B00013BEC33F03AD0C9C19AF80E
:1091E000C8C19BF808019C6B00013BEC33F030D008
:1091F00008019A6B9B6B9C6B00013BEC33F028D011
:10920000060E0801D36F240ED26F0001EAEC30F095
:109210001FD0060E0801D36F100ED26F0001EAECCA
:1092200030F016D0060E0801D36F160ED26F000173
:10923000EAEC30F00DD0060E0801D36F300ED26F7D
:109240000001EAEC30F004D0000E016E0FD000D027
:109250000501702D09D0070E0601376FD00E366F4D
:109260000001D0EC41F00501010E016E0001000C7F
:109270000501E96BEB6BEA6B020EEC6F030EED6F11
:10928000EE91DB2D04D0230EEC6F0D0EED6F050E6D
:10929000EA6EDC0EE96E0801E56BE76B0D0EE66F1A
:1092A00000016BEC25F0010169B14BD0EBC5E2FC8C
:1092B000EAC5E1FC0C01E46B190EE36F000158EC08
:1092C00029F002C0F0F501C0EFF50501DA51025CAA
:1092D0002BE303E1D951EF5D27E30101C4A121D0C4
:1092E000A00EF66E280EF76E000EF86E190E08012D
:1092F000E56F000169EC29F0100EE96EDAC5E6F8B9
:10930000D9C5E5F875EC31F0BC0EF66E280EF76E97
:10931000000EF86E070E0801E56F000169EC29F0F8
:109320000101000E016ECCD0190E0801E56F00019D
:109330003FEC20F00501EA2BD8B4EB2B0001B3D7AA
:109340000101C4A10AD0C40EF66E280EF76E000EFD
:10935000F86E0001B9EC2DF0010169A1AFD0036AEC
:109360000501E951DC0F016E050E032201C0EFF586
:1093700003C0F0F500011AEC30F0F0C5EAFFEFC5CC
:10938000E9FF01C0EFFF0101C4A133D0036A050169
:10939000E951DC0FE96E050E0320EA6EEF501F085D
:1093A00012E2036AE951DC0FE96E050E0320EA6E52
:1093B000EFCFEFF5EF519EA8FED7AD6E200E9EA821
:1093C000FED7AD6E16D0036AE951DC0FE96E050ECB
:1093D0000320EA6EEFCFEFF5EFC5E6F8370E080190
:1093E000E76F000182EC29F0200E9EA8FED7AD6E3B
:1093F00005010501DB5341E1EEB117D0036AE951E4
:10940000DC0FE96E050E0320EA6EEF5002080CE156
:10941000036AE951DC0FE96E050E0320EA6EEFCF17
:10942000DCF5EE81010EE96F27D0036AE951DC0F0C
:10943000E96E050E0320EA6EEF5003081DE10101FD
:10944000C4A108D00D0E9EA8FED7AD6E0A0E9EA830
:10945000FED7AD6E0501DD51450809E0DD51650817
:1094600006E0010E016E01012BD005D00501FF0EB3
:10947000016E010125D005010FD0036AE951DC0F0F
:10948000E96E050E0320EA6EEF500D0805E1010EAE
:10949000016E010115D00501E9510B0802E3E92B2A
:1094A00002D0E96BEE91010169B107D0320E0801DB
:1094B000E56F00013FEC20F001014FD7000E016E77
:1094C0000001000C05017691040E776F230E786F72
:1094D0004F0E796F310E7A6F0D0E7B6F0C0E7C6F15
:1094E000230E7D6F550E7E6F380E7F6F300E806FAE
:1094F000816F826F380E836F300E846F856F866F39
:10950000080E876F0D0E886F080E896F230E8A6F05
:10951000410E8B6F580E8C6F5A0E8D6F380E8E6FFA
:10952000300E8F6F906F0D0E916F050E926F230EA0
:10953000936F520E946F956B966B0D0E976F050E91
:10954000986F020E996F510E9A6F520E9B6F530EC9
:109550009C6F030E9D6F070E9E6F020E9F6F4F0E46
:10956000A06F520EA16F530EA26F3A0EA36F310E71
:10957000A46F030EA56F050EA66F020EA76F510E06
:10958000A86F520EA96F560EAA6F030EAB6F090E8D
:10959000AC6F020EAD6F4F0EAE6F520EAF6F560E28
:1095A000B06F3A0EB16F300EB26FB36FB46F030E7F
:1095B000B56F050EB66F020EB76F510EB86F410E44
:1095C000B96F460EBA6F030EBB6F070EBC6F020E6B
:1095D000BD6F4F0EBE6F410EBF6F460EC06F3A0E8D
:1095E000C16F310EC26F030EC36F050EC46F230E21
:1095F000C56F460EC66FC76BC86B0D0EC96F040EE4
:10960000CA6F230ECB6F470ECC6F460ECD6F0D0E7B
:10961000CE6F080ECF6F230ED06F410ED16F580E54
:10962000D26F460ED36FD46BD56BD66B0D0ED76F42
:109630006F51010A0001D8B4A0D0030AD8B4A1D058
:10964000010AD8B4A2D0070AD8B4A3D0010AD8B46A
:10965000A1D0030AD8B4A7D00E0AD8B4ADD0010A5D
:10966000D8B4B3D0030AD8B4B1D04A0AD8B4AFD072
:10967000010AD8B4ADD0460AD8B4ABD0070AD8B4E2
:10968000B1D00D0AD8B4AFD0030AD8B4B8D0010A0B
:10969000D8B4C1D01F0AD8B4BED0010AD8B4BCD047
:1096A000020AD8B4B9D0070AD8B4B7D0010AD8B4DE
:1096B000C0D0030AD8B4C9D0010AD8B40FD10F0A58
:1096C000D8B416D1040AD8B450D1010AD8B459D1AB
:1096D000030AD8B462D1010AD8B470D13F0AD8B411
:1096E0007ED1010AD8B48CD11B0AD8B4C6D10C0AD9
:1096F000D8B4C4D1030AD8B400D20C0AD8B4FDD16E
:10970000020AD8B439D2070AD8B437D2180AD8B462
:1097100035D2010AD8B433D2030AD8B431D2010AFF
:10972000D8B42FD20F0AD8B42DD2010AD8B42BD274
:10973000030AD8B429D2010AD8B427D2070AD8B468
:1097400025D2010AD8B423D2030AD8B421D2010AFF
:10975000D8B41FD21F0AD8B41DD2010AD8B41BD264
:109760000E0AD8B419D20D0AD8B424D2010AD8B43A
:109770002FD20D0AD8B42DD22DD2010E016E41D2B6
:109780002DD2010E016E3DD229D2010E016E39D2C9
:1097900025D224D2050E0801D36F980ED26F000196
:1097A000EAEC30F01BD2050E0801D36FB60ED26F73
:1097B0000001EAEC30F012D2050E0801D36FA60EBC
:1097C000D26F0001EAEC30F009D208D207D206D2FB
:1097D00005D2050E0801D36FCA0ED26F0001EAEC64
:1097E00030F0FCD1FBD1310E05017A6F050E080176
:1097F000D36F770ED26F0001EAEC30F0EFD1300E6C
:1098000005017A6F050E0801D36F770ED26F000144
:10981000EAEC30F0E3D1E2D1E1D1300E0501A46FE2
:10982000050E0801D36F9E0ED26F0001EAEC30F0F6
:10983000D5D1310E0501A46F050E0801D36F9E0E20
:10984000D26F0001EAEC30F0C9D10101DE5103080A
:1098500008E303E1DD51FE0804E3080EDD27000EF6
:10986000DE230501D86B0101DE510F0B0501D96F15
:10987000D86FD96BE8CFD3F8000171EC34F001C098
:10988000B2F50101DD51F00B0501D86FD96BD93369
:10989000D833D933D833D933D833D933D8330F0E5B
:1098A000D917D8C5D3F8000171EC34F001C0B3F575
:1098B0000101DD510F0B0501D86FD96BE8CFD3F84B
:1098C000000171EC34F001C0B4F5050E0801D36F4E
:1098D000AC0ED26F0001EAEC30F080D10101DD5313
:1098E00002E1DE5304E0080EDD5F000EDE5B0001E6
:1098F0000501D86B0101DE510F0B0501D96FD86F3F
:10990000D96BE8CFD3F8000171EC34F001C0B2F5A7
:109910000101DD51F00B0501D86FD96BD933D83374
:10992000D933D833D933D833D933D8330F0ED917E5
:10993000D8C5D3F8000171EC34F001C0B3F50101D2
:10994000DD510F0B0501D86FD96BE8CFD3F80001BB
:1099500071EC34F001C0B4F5050E0801D36FAC0E04
:10996000D26F0001EAEC30F039D1310E0501C26F3F
:10997000050E0801D36FBC0ED26F0001EAEC30F087
:109980002DD1300E0501C26F050E0801D36FBC0E3C
:10999000D26F0001EAEC30F021D1380E0501C76F1B
:1099A000300EC86F050E0801D36FC40ED26F0001D0
:1099B000EAEC30F00501706B000110D1320E0501A8
:1099C000C76F300EC86F050E0801D36FC40ED26F7B
:1099D0000001EAEC30F00501706B0001FFD0350E9C
:1099E0000501C76F300EC86F050E0801D36FC40E96
:1099F000D26F0001EAEC30F00501706B0001EED08F
:109A00000501D86B0101DC510F0B0501D96FD86F2F
:109A1000D96BE8CFD3F8000171EC34F001C0D4F574
:109A20000101DB51F00B0501D86FD96BD933D83365
:109A3000D933D833D933D833D933D8330F0ED917D4
:109A4000D8C5D3F8000171EC34F001C0D5F501019F
:109A5000DB510F0B0501D86FD96BE8CFD3F80001AC
:109A600071EC34F001C0D6F5050E0801D36FCF0EAE
:109A7000D26F0001EAEC30F0B1D0B0D0520E050147
:109A8000946F050EEA6E710EE96E0801E56BE76BE7
:109A9000050EE66F00016BEC25F00801BD6BBC6B99
:109AA000BB6B11C2BAF80A0EBE6F050EC06F710E05
:109AB000BF6F00014CEC39F0015002101DE0050EA3
:109AC0000801D36F710ED26F0001EBEC20F0015052
:109AD000010805E271C595F572C596F505D0300E01
:109AE0000501956F71C596F5050E0801D36F920EAD
:109AF000D26F0001EAEC30F071D04D0E0501946F89
:109B0000050EEA6E710EE96E0801E56BE76B050E56
:109B1000E66F00016BEC25F00801BD6BBC6BBB6B05
:109B200011C2BAF80A0EBE6F050EC06F710EBF6F7C
:109B300000014CEC39F0015002101DE0050E080147
:109B4000D36F710ED26F0001EBEC20F001500108D1
:109B500005E271C595F572C596F505D0300E050183
:109B6000956F71C596F5050E0801D36F920ED26FF1
:109B70000001EAEC30F032D031D030D02FD02ED0EE
:109B80002DD02CD02BD02AD029D028D027D026D009
:109B900025D024D023D022D005017681000127ECE6
:109BA00033F0050E0801D36F890ED26F0001EAEC85
:109BB00030F014D005017681000127EC33F0050E5A
:109BC0000801D36F7C0ED26F0001EAEC30F006D0B2
:109BD00005D004D0000E016E14D000D00501702D08
:109BE0000ED0000E76B1010ED86F070EDA6FD00ED0
:109BF000D96FD8C5DBF5000138EC49F00501010E3D
:109C0000016E0001000C0501296B2B6B2A6B2C9156
:109C100024C5EAFF23C5E9FF0801E56BE76B25C50D
:109C2000E6F800016BEC25F0010169B14BD02BC5C2
:109C3000E2FC2AC5E1FC0C01E46B190EE36F0001A4
:109C400058EC29F002C02EF501C02DF50501275171
:109C5000025C2BE303E126512D5D27E30101C4A142
:109C600021D0D60EF66E280EF76E000EF86E1D0E81
:109C70000801E56F000169EC29F0100EE96E27C5B7
:109C8000E6F826C5E5F875EC31F0F60EF66E280E0E
:109C9000F76E000EF86E070E0801E56F000169EC23
:109CA00029F00101000E016EE1D0190E0801E56FE7
:109CB00000013FEC20F005012A2BD8B42B2B00012A
:109CC000B3D70101C4A10AD0FE0EF66E280EF76EBE
:109CD000000EF86E0001B9EC2DF0010169A1C4D0AD
:109CE000036A050129512325016E2451032201C075
:109CF0002DF503C02EF500011AEC30F02EC5EAFF59
:109D00002DC5E9FF01C0EFFF0101C4A133D0036AF3
:109D1000050129512325E96E24510320EA6EEF50F5
:109D20001F0812E2036A29512325E96E24510320FA
:109D3000EA6EEFCF2DF52D519EA8FED7AD6E200E09
:109D40009EA8FED7AD6E16D0036A29512325E96E71
:109D500024510320EA6EEFCF2DF52DC5E6F8370E1E
:109D60000801E76F000182EC29F0200E9EA8FED7C3
:109D7000AD6E05010501285355E12CB11FD0036AD2
:109D800029512325E96E24510320EA6EEF50020881
:109D900014E124C503F0036A29512325E96E2451F7
:109DA0000320EA6EEFCF2FF524C5EAFF23C5E9FFB4
:109DB0002FC5EFFF2C81010E296F33D0036A295183
:109DC0002325E96E24510320EA6EEF50030829E1B0
:109DD0000101C4A108D00D0E9EA8FED7AD6E0A0EDB
:109DE0009EA8FED7AD6E010E05012325E96E000E7B
:109DF0002421EA6EEF5045080FE0010E2325E96E9D
:109E0000000E2421EA6EEF50650806E0010E016E97
:109E100001012CD005D00501FF0E016E010126D0F5
:109E200005010FD0036A29512325E96E245103202F
:109E3000EA6EEF500D0805E1010E016E010116D02A
:109E40000501010E255D295D02E2292B02D0296B57
:109E50002C91010169B107D0320E0801E56F0001B4
:109E60003FEC20F001013AD7000E016E0001000C1A
:109E70000801A96BA86BAB6BAA6BAC6BA75303E093
:109E8000A751060823E2B80EF66E230EF76E000EF9
:109E9000F86E190EE56F000169EC29F0A7C8ADF85E
:109EA0001F0E0801AE6F000168EC30F0D30EF66EA5
:109EB000230EF76E000EF86E060E0801E56F000126
:109EC00069EC29F0000E016ECBD00801A7C84FF253
:109ED000AB6B010EAA6FAB53D8A4B7D0AA510C0834
:109EE000D8A0B3D0A96B900EA86F010EA75D036A2E
:109EF000AD6F03C0AEF8A9C8E2FCA8C8E1FC03C07E
:109F0000E4FCE8CFE3FC000158EC29F002C0A9F81A
:109F100001C0A8F8200E0801A827000EA923010EF1
:109F2000AA5DAD6F000EAB59AE6FE8CFE2FCADC8D5
:109F3000E1FC0C01E46B0C0EE36F000158EC29F01E
:109F400001500801A8270250A9230101C4A13ED055
:109F50000801AA2D3AD0AB5338E1DA0EF66E230E83
:109F6000F76E000EF86E050EE56F000169EC29F042
:109F7000A7C8ADF81F0E0801AE6F000168EC30F005
:109F8000E10EF66E230EF76E000EF86E100E08014D
:109F9000E56F000169EC29F0A9C8E6F8370E080161
:109FA000E76F000182EC29F0A8C8E6F8370E080137
:109FB000E76F000182EC29F00A0E9EA8FED7AD6E75
:109FC0000D0E9EA8FED7AD6E08010101F2CFADF8CF
:109FD000F29EA9C8AAFFA8C8A9FFA69CA69EA68013
:109FE000A8500801ADBFF28EAC6FAC51F00B09E088
:109FF0004F0EAA25E96E020EAB21EA6EFF0EEF6E40
:10A0000007D04F0EAA25E96E020EAB21EA6EEF6A69
:10A010000101C4A115D04F0E0801AA25E96E020E58
:10A02000AB21EA6EEFCFADF8ADC8E6F8570EE76F9B
:10A03000000182EC29F0200E9EA8FED7AD6E010132
:10A040000801AA2BD8B4AB2B46D70101C4A108D074
:10A050000A0E9EA8FED7AD6E0D0E9EA8FED7AD6E61
:10A060000001000C0101D33905016E6F0F0E6E1750
:10A07000010E6E5DF10F1DE20F0F00015BEF50F05E
:10A080006CC56FF56DC570F522EC44F0050111D07B
:10A090006CC56FF56DC570F583EC3DF0050109D019
:10A0A0006CC56FF56DC570F562EC4AF0050101D025
:10A0B00005010001000CE824F76AF736D70FF66EA9
:10A0C000A00EF722000EF86EFB6E0A00F550FA6E35
:10A0D0000800F550F96E80A080A080A080A080A02C
:10A0E00080A080A080A080A080A080A090A0A0A040
:10A0F00080A080A00F0E0501246F810E256F010E38
:10A10000266F060E276F020E286F296B2A6B2B6BAA
:10A110002C6B2D6B2E6B2F6B306B316B326BFF0EFC
:10A12000336F346F090E356F810E366F010E376F46
:10A13000040E386F470E396F3A6B3B6B3C6B3D6BCF
:10A14000FF0E3E6F090E3F6F810E406F010E416F93
:10A15000040E426F480E436F446B456B466B476B72
:10A16000FF0E486F090E496F810E4A6F010E4B6F4B
:10A17000040E4C6F4E0E4D6F4E6B4F6B506B516B10
:10A18000FF0E526F070E536F0101D339006E0F0E91
:10A19000001600500A0807E0D339006E0F0E0016B3
:10A1A00000500B0824E1D339006E0F0E001600504A
:10A1B0000B08D8A4EFD0D89002011035036AEA0F3B
:10A1C000E96E010E0320EA6EECCF55F5ED52EFCFAC
:10A1D00054F5050154510208D8B402D0010107D04A
:10A1E000552D01D002D0010102D00101D3D0C9C147
:10A1F00029F5C8C12AF5D339006E0F0E001600509C
:10A20000080815E0D339006E0F0E001600500F0835
:10A210000EE0D339006E0F0E00160050070807E05D
:10A22000D339006E0F0E00160050090811E1050128
:10A23000242B036A5351240FE96E050E0320EA6EA6
:10A240000101D4510F0BEF6E0501532B2A6B010155
:10A25000036A05015351240FE96E050E0320EA6ECF
:10A260000101D6390501566F0F0E561756510F0BC7
:10A27000EF6E010E5325036A240FE96E050E0320CD
:10A28000EA6ED6C156F556510F0BEF6E020E5325EE
:10A29000036A240FE96E050E0320EA6E0101D63130
:10A2A0000501576F0101D5310501566F57335633FC
:10A2B00057335633573356330F0E571756510F0B2C
:10A2C000EF6E030E5325036A240FE96E050E03207B
:10A2D000EA6E0101D5510F0BEF6E040E05015325F7
:10A2E000036A240FE96E050E0320EA6E0101D839D6
:10A2F0000501566F0F0E561756510F0BEF6E050ED8
:10A300005325036A240FE96E050E0320EA6ED8C1B7
:10A3100056F556510F0BEF6E060E5325036A240FA8
:10A32000E96E050E0320EA6E0101D8310501576F71
:10A330000101D7310501566F573356335733563322
:10A34000573356330F0E571756510F0BEF6E070E3C
:10A350005325036A240FE96E050E0320EA6E0101FE
:10A36000D7510F0BEF6E050E0801D36F240ED26F7D
:10A370000001EAEC30F04E0E0601376F200E366F0A
:10A380000001D0EC41F0012C01D003D0000E016E91
:10A39000CDD10101D339006E0F0E00160050050813
:10A3A00005E1010E016E0001C1D10101DA3905019B
:10A3B000546F0F0E541754510F0B3A6FDAC154F506
:10A3C00054510F0B3B6F0101DA310501556F01014B
:10A3D000D9310501546F5533543355335433553304
:10A3E00054330F0E551754510F0B3C6F0101D951C7
:10A3F0000F0BE8CF3DF50501050E0801D36F350EB3
:10A40000D26F0001EAEC30F00F0E0601376FA00E9C
:10A41000366F0001D0EC41F0012C01D003D0000ECA
:10A42000016E84D10101D3A709D01C0E05016C6F08
:10A43000010E6D6F000116DED6D001011D0E050163
:10A440006C6F010E6D6F00010DDE0101D339006EDE
:10A450000F0E001600500B08D8A489D0D890020126
:10A460001035036AEA0FE96E010E0320EA6EEF5021
:10A47000006EE92AEF50E906036E030E035C04E167
:10A480000052000128E00201020E035C05E1010E0A
:10A49000005C000120E00201020E035C04E10052B6
:10A4A000000119E00201010E035C04E10052000109
:10A4B00050E00201010E035C05E1010E005C0001A9
:10A4C00048E00201010E035C05E1020E005C0001A0
:10A4D00040E002013FD00101DC390501546F0F0E4D
:10A4E000541754510F0B446FDCC154F554510F0BEA
:10A4F000456F0101DC310501556F0101DB310501BB
:10A50000546F5533543355335433553354330F0E3E
:10A51000551754510F0B466F0101DB510F0BE8CF5C
:10A5200047F50501050E0801D36F3F0ED26F0001FC
:10A53000EAEC30F0030E0601376FE80E366F0001CB
:10A54000D0EC41F0012C01D003D0000E016EEED012
:10A550000CD0020132B907D0380E05016C6F010E24
:10A560006D6F00017FDD000100D03DD00101DC39BD
:10A570000501546F0F0E541754510F0B446FDCC17B
:10A5800054F554510F0B456F0101DC310501556F36
:10A590000101DB310501546F5533543355335433C6
:10A5A000553354330F0E551754510F0B466F01019D
:10A5B000DB510F0BE8CF47F50501050E0801D36FFE
:10A5C0003F0ED26F0001EAEC30F0030E0601376F48
:10A5D000E80E366F0001D0EC41F0012C01D003D021
:10A5E000000E016EA3D00101D3A548D0D339006E6F
:10A5F0000F0E001600500B0835E0140E05016C6FAD
:10A60000010E6D6F00012EDD0101DE6B070EDD6FA7
:10A61000D89002011035036AF80FE96E010E03208D
:10A62000EA6EDEC1ECFFED52DDC1EFFF05014E6BBE
:10A630004F6B506B0101DD510F0BE8CF51F5050158
:10A64000050E0801D36F490ED26F0001EAEC30F01D
:10A65000030E0601376FE80E366F0001D0EC41F0B3
:10A6600004D00101DE6B110EDD6F150E05016C6F5C
:10A67000010E6D6F0001F6DC45D00101140E0501DD
:10A680006C6F010E6D6F0001EDDC0101DE3905011B
:10A69000546F0F0E541754510F0B4E6FDEC154F50B
:10A6A00054510F0B4F6F0101DE310501556F010150
:10A6B000DD310501546F553354335533543355331D
:10A6C00054330F0E551754510F0B506F0101DD51CC
:10A6D0000F0BE8CF51F50501050E0801D36F490EA8
:10A6E000D26F0001EAEC30F0030E0601376FE80E7E
:10A6F000366F0001D0EC41F0012C01D003D0000EE8
:10A70000016E14D00101D3A108D00F0E05016C6FAA
:10A71000010E6D6F0001A6DC07D0100E05016C6FF5
:10A72000010E6D6F00019EDC010E016EFAEF59F013
:10A7300005017B6B7D6B7C6B7E91050EEA6E6E0E68
:10A74000E96E0801E56BE76B0D0EE66F00016BEC3F
:10A7500025F0010169B14BD07DC5E2FC7CC5E1FC6F
:10A760000C01E46B190EE36F000158EC29F002C0F4
:10A7700080F501C07FF505016D51025C2BE303E11B
:10A780006C517F5D27E30101C4A121D0500EF66E0C
:10A79000270EF76E000EF86E180E0801E56F000127
:10A7A00069EC29F0100EE96E6DC5E6F86CC5E5F8A8
:10A7B00075EC31F06B0EF66E270EF76E000EF86E2C
:10A7C000070E0801E56F000169EC29F00101FF0E99
:10A7D000016EEBD0190E0801E56F00013FEC20F08F
:10A7E00005017C2BD8B47D2B0001B3D70101C4A196
:10A7F0000AD0740EF66E270EF76E000EF86E00018A
:10A80000B9EC2DF0010169A1CED0036A05017B519D
:10A810006E0F016E050E032201C07FF503C080F5A7
:10A8200000011AEC30F080C5EAFF7FC5E9FF01C0E6
:10A83000EFFF0101C4A116D0036A05017B516E0F21
:10A84000E96E050E0320EA6EEFCF7FF57FC5E6F8CF
:10A85000370E0801E76F000182EC29F0200E9EA858
:10A86000FED7AD6E05017EB117D0036A7B516E0F26
:10A87000E96E050E0320EA6EEF50FE080CE1036A54
:10A880007B516E0FE96E050E0320EA6EEFCF6EF579
:10A890007E81010E7B6F7CD0036A7B516E0FE96E67
:10A8A000050E0320EA6EEF50EF0864E10101C4A138
:10A8B00008D00D0E9EA8FED7AD6E0A0E9EA8FED73C
:10A8C000AD6EC4A147D0050171510F0B006E003869
:10A8D0007F6FF00E7F1772510F0B7F13860EF66E8F
:10A8E000270EF76E000EF86E0D0E0801E56F0001E1
:10A8F00069EC29F071C5E6F8570E0801E76F000111
:10A9000082EC29F02C0E9EA8FED7AD6E72C5E6F83B
:10A91000570E0801E76F000182EC29F0200E9EA877
:10A92000FED7AD6E280E9EA8FED7AD6E7FC5E6F8A9
:10A93000570E0801E76F000182EC29F0290E9EA84E
:10A94000FED7AD6E0D0E9EA8FED7AD6E0A0E9EA868
:10A95000FED7AD6E050171510F0B006E00387F6F91
:10A96000F00E7F1772510F0B7F11016E01011DD088
:10A9700007D00501320E0801E56F00013FEC20F021
:10A9800005017B510B0802E37B2B02D07B6B7E9190
:10A99000010169B107D0320E0801E56F00013FECFB
:10A9A00020F0010130D7EE0E016E0001000C0E0EFA
:10A9B0000501246FFF0E256F300E266F276F286B61
:10A9C000620E296F2A6B2B6B2C6B2D6B2E6B2F6BF2
:10A9D000306B316BEF0E326F0A0E336FFF0E346F38
:10A9E000300E356F366F376BB30E386F396B3A6B8D
:10A9F0003B6B3C6BEF0E3D6F0A0E3E6FFF0E3F6FE1
:10AA0000300E406F416F426BB00E436F446B456B2D
:10AA1000466B476BEF0E486F090E496FFF0E4A6F8A
:10AA2000300E4B6F4C6F4D6B500E4E6F4F6B506B2B
:10AA3000516BEF0E526F090E536FFF0E546F300EB5
:10AA4000556F566F576B510E586F596B5A6B5B6B46
:10AA5000EF0E5C6F080E5D6FFF0E5E6F300E5F6F66
:10AA6000606F616BB40E626F310E636F646BEF0EDB
:10AA7000656F676B666B696B686B6A6B6B6B036AA0
:10AA8000C9C16CF503C06DF50C01E26B210EE16FDD
:10AA900003C0E4FCC9C1E3FC000158EC29F0080E36
:10AAA00005010124686F000E0220696F695306E1F9
:10AAB0006851070803E3696B080E686F6951020863
:10AAC00009E2FF0A03E16851200804E2030E696FFE
:10AAD000200E686F69510F0B6C6FE8CFD3F800013F
:10AAE00071EC34F001C04FF5050168C500F0003A83
:10AAF0000F0E001600500F0B6C6FE8CFD3F800015B
:10AB000071EC34F001C050F5050168510F0B6C6F0A
:10AB1000E8CFD3F8000171EC34F001C051F5050E17
:10AB20000801D36F490ED26F0001EAEC30F0030E3A
:10AB300005016D6FE80E6C6F0001FADD01C06BF569
:10AB400005016B5330E06B51100803E06B51500866
:10AB500024E1020E6C6FFA0E0801E56F00013FEC74
:10AB600020F005016C2FF7D7050E0801D36F490EB1
:10AB7000D26F0001EAEC30F0030E0801D36FE80E4B
:10AB8000D26F000180EC34F0012C01D004D0000E13
:10AB9000016ECEEF59F006D00501000E016E0001E6
:10ABA000CEEF59F00501036AC8C16CF503C06DF51D
:10ABB0000C01E26B1E0EE16F03C0E4FCC8C1E3FCB4
:10ABC000000158EC29F0080E05010124666F000E03
:10ABD0000220676F675306E16651070803E3676B5E
:10ABE000080E666F6751010809E2FF0A03E166512A
:10ABF0006E0804E2020E676F6E0E666F67510F0BF0
:10AC00006C6FE8CFD3F8000171EC34F001C059F556
:10AC1000050166C500F0003A0F0E001600500F0B3C
:10AC20006C6FE8CFD3F8000171EC34F001C05AF535
:10AC3000050166510F0B6C6FE8CFD3F8000171EC82
:10AC400034F001C05BF5050E0801D36F530ED26FCF
:10AC50000001EAEC30F0030E05016D6FE80E6C6F39
:10AC6000000166DD01C06BF505016B532DE06B51F2
:10AC7000100803E06B51500823E1020E6C6FFA0ECE
:10AC80000801E56F00013FEC20F005016C2FF7D7BC
:10AC9000050E0801D36F530ED26F0001EAEC30F0BD
:10ACA000030E0801D36FE80ED26F000180EC34F080
:10ACB000012C01D003D0000E016E70D305D0050128
:10ACC000000E016E00016AD30101D63905016C6FD7
:10ACD0006D6B0F0E6C176C510F0B006E036A6C6F6F
:10ACE000E8CFD3F8000171EC34F001C02AF5D6C1E9
:10ACF0006CF505016D6B6C510F0B006E036A6C6F88
:10AD0000E8CFD3F8000171EC34F001C02BF501015C
:10AD1000D63105016D6F0101D53105016C6F6D33C1
:10AD20006C336D336C336D336C330F0E6D176C51A8
:10AD30000F0B006E036A6C6FE8CFD3F8000171EC63
:10AD400034F001C02CF50101D5510F0B006E036AE0
:10AD5000E8CF6CF5E8CFD3F8000171EC34F001C016
:10AD60002DF50101D83905016C6F6D6B0F0E6C1755
:10AD70006C510F0B006E036A6C6FE8CFD3F80001C3
:10AD800071EC34F001C02EF5D8C16CF505016D6B86
:10AD90006C510F0B006E036A6C6FE8CFD3F80001A3
:10ADA00071EC34F001C02FF50101D83105016D6F50
:10ADB0000101D73105016C6F6D336C336D336C332A
:10ADC0006D336C330F0E6D176C510F0B006E036AF1
:10ADD0006C6FE8CFD3F8000171EC34F001C030F5AE
:10ADE0000101D7510F0B006E036AE8CF6CF5E8CF75
:10ADF000D3F8000171EC34F001C031F5050E080103
:10AE0000D36F240ED26F0001EAEC30F0170E05016B
:10AE10006D6F700E6C6F00018BDC01C06BF505016E
:10AE20006B532EE06B51100803E06B51500823E187
:10AE3000080E6C6FFA0E0801E56F00013FEC20F080
:10AE400005016C2FF7D7050E0801D36F240ED26FC2
:10AE50000001EAEC30F0070E0801D36FD00ED26F7C
:10AE6000000180EC34F0012C01D003D0000E016E03
:10AE700095D205D00501000E016E00018FD20501AB
:10AE80006A5301E16A6B6A51070802E2070E6A6FB2
:10AE9000370E646F050E0801D36F5D0ED26F00018F
:10AEA000EAEC30F0030E05016D6FE80E6C6F0001E7
:10AEB0003FDC01C06BF505016B532DE06B511008B1
:10AEC00003E06B51500823E1020E6C6FFA0E08018B
:10AED000E56F00013FEC20F005016C2FF7D7050E60
:10AEE0000801D36F5D0ED26F0001EAEC30F0030E63
:10AEF0000801D36FE80ED26F000180EC34F0012C12
:10AF000001D003D0000E016E49D205D00501000E1C
:10AF1000016E000143D20101DA3905016C6F6D6BDE
:10AF20000F0E6C176C510F0B006E036A6C6FE8CF3D
:10AF3000D3F8000171EC34F001C039F5DAC16CF5D9
:10AF400005016D6B6C510F0B006E036A6C6FE8CFDF
:10AF5000D3F8000171EC34F001C03AF50101DA31A7
:10AF600005016D6F0101D93105016C6F6D336C33D3
:10AF70006D336C336D336C330F0E6D176C510F0BDB
:10AF8000006E036A6C6FE8CFD3F8000171EC34F007
:10AF900001C03BF50101D9510F0B006E036AE8CFE8
:10AFA0006CF5E8CFD3F8000171EC34F001C03CF54A
:10AFB000050E0801D36F330ED26F0001EAEC30F0BA
:10AFC000030E05016D6FE80E6C6F000198EC53F0F5
:10AFD00001C06BF505016B5328E06B51100803E0CD
:10AFE0006B51500822E1080E6C6FFA0E0801E56FF4
:10AFF00000013FEC20F005016C2FF7D7050E08018A
:10B00000D36F330ED26F0001EAEC30F0070E080167
:10B01000D36FD00ED26F000180EC34F0012C01D040
:10B0200003D0000E016EBAD105010101D3A742D0B1
:10B030001C0E05016C6F6D6B000132EC50F0030EBD
:10B0400005016D6FE80E6C6F000198EC53F001C0C4
:10B050006BF505016B532CE06B51100803E06B514D
:10B06000500821E1040E6C6FFA0E0801E56F000133
:10B070003FEC20F005016C2FF7D71C0E6C6F6D6B49
:10B08000000132EC50F0030E0801D36FE80ED26FCE
:10B09000000180EC34F0012C01D003D0000E016ED1
:10B0A0007DD105D00501000E016E000177D10501AB
:10B0B000FCD001011D0E05016C6F6D6B000132ECBF
:10B0C00050F0030E05016D6FE80E6C6F000198ECF7
:10B0D00053F001C06BF505016B532BE06B51100869
:10B0E00003E06B51500821E1040E6C6FFA0E080169
:10B0F000E56F00013FEC20F005016C2FF7D71D0E26
:10B100006C6F6D6B000132EC50F0030E0801D36FD1
:10B11000E80ED26F000180EC34F0012C01D003D096
:10B12000000E016E3BD105D00501000E016E00013D
:10B1300035D10101DC3905016C6F6D6B0F0E6C1799
:10B140006C510F0B006E036A6C6FE8CFD3F80001EF
:10B1500071EC34F001C044F5DCC16CF505016D6B98
:10B160006C510F0B006E036A6C6FE8CFD3F80001CF
:10B1700071EC34F001C045F50101DC3105016D6F62
:10B180000101DB3105016C6F6D336C336D336C3352
:10B190006D336C330F0E6D176C510F0B006E036A1D
:10B1A0006C6FE8CFD3F8000171EC34F001C046F5C4
:10B1B0000101DB510F0B006E036AE8CF6CF5E8CF9D
:10B1C000D3F8000171EC34F001C047F5050E080119
:10B1D000D36F3E0ED26F0001EAEC30F0070E05018E
:10B1E0006D6FD00E6C6F000198EC53F001C06BF5E1
:10B1F00005016B535AE06B51100803E06B51500886
:10B200004FE1080E6C6FFA0E0801E56F00013FEC8C
:10B2100020F005016C2FF7D7050E0801D36F3E0E05
:10B22000D26F0001EAEC30F0070E05016D6FD00E11
:10B230006C6F000198EC53F001C06BF505016B5386
:10B240002EE06B51100803E06B51500823E1080E0B
:10B250006C6FFA0E0801E56F00013FEC20F005016C
:10B260006C2FF7D7050E0801D36F3E0ED26F000189
:10B27000EAEC30F0070E0801D36FD00ED26F000158
:10B2800080EC34F0012C01D003D0000E016E86D08A
:10B2900005D00501000E016E000180D0050105D02A
:10B2A000000E016E00017AD005010101D3A309D07F
:10B2B000110E05016C6F010E6D6F000132EC50F044
:10B2C00008D0130E05016C6F010E6D6F000132EC9A
:10B2D00050F0640E0801E56F00013FEC20F0010121
:10B2E000D3B10AD0100E05016C6F010E6D6F000115
:10B2F00032EC50F009D001010F0E05016C6F010E08
:10B300006D6F000132EC50F0640E0801E56F000132
:10B310003FEC20F00101D3A52BD0DE6B480EDD6F92
:10B32000D89002011035036AF80FE96E010E032070
:10B33000EA6EDEC1ECFFED52DDC1EFFF140E050138
:10B340006F6F010E706F000183EC3DF0180E050168
:10B350006F6F010E706F000183EC3DF0150E05015B
:10B360006F6F010E706F000183EC3DF011D0010191
:10B37000140E05016F6F010E706F000183EC3DF03C
:10B38000180E05016F6F010E706F000183EC3DF028
:10B39000640E0801E56F00013FEC20F0FFEF59F06B
:10B3A000010E016E03EF5AF00101D339006E0F0E4A
:10B3B00000160050020A00011BE0010A19E0060A0B
:10B3C00017E00D0A15E0010A13E00E0A11E0080A61
:10B3D0000FE00B0A0DE00F0A0BE00A0A09E0070A6A
:10B3E00007E00C0A05E0060A08E0010A0BE00ED0AF
:10B3F0007AEF50F001500ED00DD0D7EF54F001503D
:10B4000009D008D0CDD7015005D004D0000E016E70
:10B4100001D000D0000C0FC5A7F838EC4FF00201A6
:10B420005B3D76D00FC524F50C0E0501256F00019C
:10B43000A5EC29F0012C6BD0050EEA6E100EE96E1A
:10B44000000EBFEC0FF00A000900F550EE6E000987
:10B45000FBE1050E0801A86F100EA76F0001C3ECF9
:10B4600025F00101D339006E0F0E001600500D08B3
:10B4700049E1D3A70AD01C0E05016F6F010E706F52
:10B48000000162EC4AF009D001011D0E05016F6F49
:10B49000010E706F000162EC4AF00101D3A50AD0E1
:10B4A000150E05016F6F010E706F000162EC4AF01E
:10B4B00009D00101140E05016F6F010E706F0001BC
:10B4C00062EC4AF00C0E0201116F360E05016F6F2F
:10B4D000706B000162EC4AF0070E0501DA6FD00EC6
:10B4E000D96F010EDB6F000138EC49F03A0E05010F
:10B4F000DA6F980ED96F010EDB6F000138EC49F05E
:10B5000003D00101000150DF010E016E25D00201C0
:10B51000050EEA6E100EE96E000E0001D2EC0FF07F
:10B520000A000900F550EE6E0009FBE1050E080166
:10B53000A86F100EA76F0001C3EC25F0080E0501DF
:10B54000246FFA0E0801D36F00012AEC20F00501E8
:10B55000242FF7D7000E016E0001000C05015B518E
:10B56000390805E2370E5B5D016E05D004D0300E60
:10B570005B5D016E00D00001000C0501536B546B44
:10B58000556B020E566F900E576F41C5E9FF42C5CD
:10B59000EAFFEC6AED52EF6A050EEA6E430EE96EC1
:10B5A0000801E56BE76B100EE66F00016BEC25F010
:10B5B0000101D339006E0F0E001600500C0805E192
:10B5C000050E0501566FFE0E576F020E0501586FEE
:10B5D000C80E0801E56F00013FEC20F00501582F6F
:10B5E000F7D7010169A13CD0050153510F08D8B02C
:10B5F00002D0010135D000011AEC30F001C054F541
:10B600000A0E0801E56F00013FEC20F00101C4A122
:10B610000ED054C5E6F8570E0801E76F000182EC22
:10B6200029F0200E9EA8FED7AD6E07D001010A0EAC
:10B630000801E56F00013FEC20F005015751545D12
:10B6400004E1536B54C543F50AD0532B036A53519D
:10B65000430FE96E050E0320EA6E54C5EFFFC1D714
:10B66000030E05015625535D03E2000E016E6FD0F7
:10B670000101D339006E0F0E001600500C0829E1AD
:10B6800056C555F5030E05015625555D01E022E22C
:10B69000036A5551430F016E050E032201C058F590
:10B6A00003C059F5036A5551430FE96E050E032097
:10B6B000EA6EEFCF5AF55AC55BF500014FDF59C569
:10B6C000EAFF58C5E9FF01C0EFFF0501552B010155
:10B6D000D9D70501556B5551030837E341C5E9FF3B
:10B6E00042C5EAFFEF34026EEC34036E02360336D5
:10B6F0000236033602360336F00E02160250ED52C1
:10B70000EF6E03C0ECFF42C503F042C5EAFF41C53E
:10B71000E9FFECCF5BF5ED52EFCF5AF555515625C9
:10B72000036A430FE96E050E0320EA6EEF500F0B1C
:10B730005A115BC503F042C5EAFF41C5E9FF5BC58D
:10B74000ECFFED52EF6E552BC6D7010E016E0001D6
:10B75000000C0501356B366B020E376F900E386F9B
:10B7600023C5E9FF24C5EAFFEF6A050EEA6E250E40
:10B77000E96E0801E56BE76B100EE66F00016BECFC
:10B7800025F00101D339006E0F0E001600500C0891
:10B7900005E1050E0501376FFE0E386F020E05013B
:10B7A000396FC80E0801E56F00013FEC20F005017C
:10B7B000392FF7D7010169A13CD0050135510F0898
:10B7C000D8B002D0010135D000011AEC30F001C030
:10B7D00036F50A0E0801E56F00013FEC20F001018B
:10B7E000C4A10ED036C5E6F8570E0801E76F000178
:10B7F00082EC29F0200E9EA8FED7AD6E07D0010185
:10B800000A0E0801E56F00013FEC20F005013851F8
:10B81000365D04E1356B36C525F50AD0352B036A54
:10B820003551250FE96E050E0320EA6E36C5EFFF90
:10B83000C1D7020E05013725355D03E2000E016E0A
:10B840007CD00101D339006E0F0E001600500C0899
:10B850003EE1036A05013751250F016E050E0322F3
:10B8600001C039F503C03AF5036A3751250FE96E77
:10B87000050E0320EA6EEFCF3BF53BC55BF50001FB
:10B880006DDE3AC5EAFF39C5E9FF01C0EFFF010EE1
:10B8900005013725036A250F016E050E032201C03D
:10B8A00039F503C03AF5010E3725036A250FE96E15
:10B8B000050E0320EA6EEFCF3BF53BC55BF50001BB
:10B8C0004DDE3AC5EAFF39C5E9FF01C0EFFF24C5E7
:10B8D00003F00501036A3751250FE96E050E0320B9
:10B8E000EA6EEFCF3BF524C5EAFF23C5E9FF3BC570
:10B8F000EFFF23C5E9FF24C5EAFFEF38006EF00E25
:10B90000001600C0EFFF24C503F024C5EAFF23C5DD
:10B91000E9FFEFCF3BF5010E3725036A250FE96EEE
:10B92000050E0320EA6EEF500F0B3B1124C5EAFF12
:10B9300023C5E9FFEF6E010E016E0001000C050149
:10B940000F6B116B106B000127EC33F00101D33941
:10B95000006E0F0E001600500C081DE0D339006E6B
:10B960000F0E001600500D0816E0080E05016F6F4F
:10B97000706B000122EC44F0050E0501426F100EC1
:10B98000416F0001FADD012C04D011C5DEF110C5B4
:10B99000DDF15DD00101D339006E0F0E00160050AD
:10B9A0000C0818E1080E05016F6F706B000183EC45
:10B9B0003DF0050E0501246F0F0E236F0001C9DE57
:10B9C000012C06D005010F510101DE6BDD6F000176
:10B9D0003ED00101D339006E0F0E001600500D0845
:10B9E00037E1080E05016F6F706B000162EC4AF0E1
:10B9F000050E0501246F120E236F0F0E256F070E23
:10BA0000276FD00E266F286B000103EC4EF0012C3F
:10BA10001ED018C55BF5A2DD01C021F519C55BF587
:10BA20009DDD01380501236FF00E23171AC55BF564
:10BA3000000194DD050123510110226F21C511F58C
:10BA400022C510F511C5DEF110C5DDF100010101BF
:10BA50000001000C0501446B436B466B456B476B63
:10BA6000586B900E596F000127EC33F0420E050120
:10BA70006F6F706B000122EC44F0010169B134D0AA
:10BA800046C5E2FC45C5E1FC0C01E46B320EE36FF8
:10BA9000000158EC29F002C05BF501C05AF5050120
:10BAA0005B5303E15A51C70812E20101C4A109D056
:10BAB0003C0EF66E260EF76E000EF86E0001B9EC25
:10BAC0002DF0050143C501F044C502F059D0320EF6
:10BAD0000801E56F00013FEC20F00501452BD8B4CB
:10BAE000462B0001CAD7010169A135D00501585183
:10BAF0000F08D8B002D001012ED000011AEC30F0AE
:10BB000001C047F50A0E0801E56F00013FEC20F087
:10BB100005015951475D04E1586B47C548F50AD006
:10BB2000582B036A5851480FE96E050E0320EA6E40
:10BB300047C5EFFF0101C4A10DD047C5E6F8570E78
:10BB40000801E76F000182EC29F0200E9EA8FED7C5
:10BB5000AD6E0101C9D7C4A108D00A0E9EA8FED7B8
:10BB6000AD6E0D0E9EA8FED7AD6E05014F3D04D003
:10BB70004AC544F54BC543F543C501F044C502F041
:10BB8000000160EF5FF00501436B426B446B556B46
:10BB9000900E566F0D0E6F6F010E706F000122EC4C
:10BBA00044F0050EEA6E450EE96E0801E56BE76BA1
:10BBB000100EE66F00016BEC25F03D0E05016F6F76
:10BBC000706B000122EC44F00101C4A10AD0480EC0
:10BBD000F66E260EF76E000EF86E0001B9EC2DF031
:10BBE000010169B13BD043C5E2FC42C5E1FC0C0157
:10BBF000E46B320EE36F000158EC29F002C058F5F7
:10BC000001C057F50501585303E15751C7081AE21F
:10BC10000101C4A109D05A0EF66E260EF76E000E71
:10BC2000F86E0001B9EC2DF00501415308E10E0E4C
:10BC30006F6F010E706F000122EC44F00501000EE1
:10BC4000016E68D0320E0801E56F00013FEC20F074
:10BC50000501422BD8B4432B0101C3D769A135D0CC
:10BC6000050155510308D8B002D001012ED00001C2
:10BC70001AEC30F001C044F50A0E0801E56F00012E
:10BC80003FEC20F005015651445D04E1556B44C57D
:10BC900045F50AD0552B036A5551450FE96E050E3F
:10BCA0000320EA6E44C5EFFF0101C4A10DD044C5D5
:10BCB000E6F8570E0801E76F000182EC29F0200E2C
:10BCC0009EA8FED7AD6E0101C9D7C4A108D00A0E47
:10BCD0009EA8FED7AD6E0D0E9EA8FED7AD6E0501D7
:10BCE000555103080BE1483D09D04651500806E183
:10BCF0004751020803E3010E016E0CD0415308E1E5
:10BD00000E0E6F6F010E706F000122EC44F0050102
:10BD1000000E016E0001000C0501176B166B196B0C
:10BD2000186B1A6B2B6B900E2C6F050EEA6E2D0E96
:10BD3000E96E0801E56BE76B140EE66F00016BEC32
:10BD400025F0050EEA6E1B0EE96E0801E56BE76B48
:10BD5000100EE66F00016BEC25F0020E05016F6F0F
:10BD6000706B000122EC44F00101C4A10AD0840EE2
:10BD7000F66E240EF76E000EF86E0001B9EC2DF091
:10BD8000010169B130D019C5E2FC18C5E1FC0C0114
:10BD9000E46B320EE36F000158EC29F002C042F56B
:10BDA00001C041F50501425303E14151C7080FE2CB
:10BDB0000101C4A10AD0940EF66E240EF76E000E97
:10BDC000F86E0001B9EC2DF00101DBEF63F0320EEB
:10BDD0000801E56F00013FEC20F00501182BD8B4F5
:10BDE000192B0101CED769A135D005012B510F08C0
:10BDF000D8B002D001012ED000011AEC30F001C001
:10BE00001AF50A0E0801E56F00013FEC20F005016C
:10BE10002C511A5D04E12B6B1AC51BF50AD02B2B94
:10BE2000036A2B511B0FE96E050E0320EA6E1AC53B
:10BE3000EFFF0101C4A10DD01AC5E6F8570E0801A5
:10BE4000E76F000182EC29F0200E9EA8FED7AD6EB0
:10BE50000101C9D7C4A108D00A0E9EA8FED7AD6EB5
:10BE60000D0E9EA8FED7AD6E05012B510408D8B06B
:10BE700078EF63F01DC511F51EC510F51FC513F54C
:10BE800020C512F521C515F522C514F514510E086B
:10BE9000D8A485D115510E08D8A481D10101D36B46
:10BEA000B00ED313D89005010F35036AEA0F016E67
:10BEB000010E032201C041F503C042F50001CAD5BD
:10BEC00042C5EAFF41C5E9FF02C0ECFFED5201C0E7
:10BED000EFFFD89005010F35036AEA0FE96E010EF6
:10BEE0000320EA6EECCF42F5ED52EFCF41F541531E
:10BEF0000FE142530DE1D8900F35036AEA0FE96E66
:10BF0000010E0320EA6E010EEC6EED52EF6A48D08E
:10BF1000D8900F35036AEA0FE96E010E0320EA6E2E
:10BF2000ECCF42F5ED52EFCF41F5415339E14251AB
:10BF3000020836E1150E6C6F010E6D6F000132ECD8
:10BF400050F027EC33F00101DE6B0B0EDD6F080EB5
:10BF500005016C6F6D6B000132EC50F0050E0501B0
:10BF6000426F160E416F0001BDEC5AF0012C04D057
:10BF700017C5DEF116C5DDF10101DE5303E1DD5128
:10BF80000B080FE2D89005010F35036AEA0FE96E3E
:10BF9000010E0320EA6E020EEC6EED52010EEF6E02
:10BFA0000101D89005010F35036AEA0FE96E010E11
:10BFB0000320EA6EEF50006EE92AEF50E906036EA7
:10BFC000010E035C04E10052000129E00501010EAD
:10BFD000035C05E1010E005C00013DE00501010E7E
:10BFE000035C05E1020E005C000151E00501020E58
:10BFF000035C05E1010E005C000165E00501020E35
:10C00000035C04E1005200015EE00501030E035CE5
:10C0100005E100520001D8B472D005018CD00101B5
:10C02000C4A10AD0A00EF66E240EF76E000EF86EB4
:10C030000001B9EC2DF00101050EEA6E2D0EE96E3E
:10C04000000E00016AEC0BF00A000900F550EE6EDC
:10C050000009FBE18CD00101C4A10AD0B20EF66E3A
:10C06000240EF76E000EF86E0001B9EC2DF0010100
:10C07000050EEA6E2D0EE96E000E00017DEC0BF050
:10C080000A000900F550EE6E0009FBE170D00101D5
:10C09000C4A10AD0CA0EF66E240EF76E000EF86E1A
:10C0A0000001B9EC2DF00101050EEA6E2D0EE96ECE
:10C0B000000E000190EC0BF00A000900F550EE6E46
:10C0C0000009FBE154D00101C4A10AD0E80EF66ECC
:10C0D000240EF76E000EF86E0001B9EC2DF0010190
:10C0E000050EEA6E2D0EE96E000E0001A3EC0BF0BA
:10C0F0000A000900F550EE6E0009FBE138D001019D
:10C10000C4A10AD0FA0EF66E240EF76E000EF86E79
:10C110000001B9EC2DF00101050EEA6E2D0EE96E5D
:10C12000000E0001B6EC0BF00A000900F550EE6EAF
:10C130000009FBE11CD00101C4A10AD00C0EF66E6F
:10C14000250EF76E000EF86E0001B9EC2DF001011E
:10C15000050EEA6E2D0EE96E000E0001C9EC0BF023
:10C160000A000900F550EE6E0009FBE100D0050160
:10C170000F5130093D6F036A0F51E30FE96E010E55
:10C180000320EA6ED3C1EFFF050E0801A86F2D0E44
:10C19000A76F0001C3EC25F001010DD30501125179
:10C1A000006E1351036E040E035C06E1020E005C88
:10C1B0000001D8B46DD00501080E035C05E1005202
:10C1C0000001D8B4B5D00501040E035C06E10D0EE4
:10C1D000005C0001D8B4DFD00501040E035C06E169
:10C1E0000E0E005C0001D8B400D10501050E035C01
:10C1F00006E1030E005C0001D8B422D10501050E52
:10C20000035C06E1010E005C0001D8B419D1050100
:10C21000040E035C06E10F0E005C0001D8B464D18B
:10C220000501050E035C06E1050E005C0001D8B4B3
:10C2300085D10501050E035C06E1070E005C0001D7
:10C24000D8B4A7D10501050E035C06E1040E005C1D
:10C250000001D8B4D1D10501040E035C06E12C0E17
:10C26000005C0001D8B4F2D10501200E035C06E1A8
:10C27000010E005C0001D8B4E9D10501040E035C95
:10C2800006E12D0E005C0001D8B4E0D1050109D211
:10C290000101D36B010E0501416F000174DC012C1B
:10C2A0001ED0600E0101D313C4A10AD0200EF66E79
:10C2B000250EF76E000EF86E0001B9EC2DF00101AD
:10C2C000050EEA6E2D0EE96E000E0001DCEC0BF09F
:10C2D0000A000900F550EE6E0009FBE11CD00101D7
:10C2E000D389C4A10AD0360EF66E250EF76E000E65
:10C2F000F86E0001B9EC2DF00101050EEA6E2D0E6D
:10C30000E96E000E0001EFEC0BF00A000900F55099
:10C31000EE6E0009FBE105010F5130093D6F050E7E
:10C320000801A86F2D0EA76F0001C3EC25F0DED128
:10C330000101D36B500ED313C4A10AD0480EF66E80
:10C34000250EF76E000EF86E0001B9EC2DF001011C
:10C35000050EEA6E2D0EE96E000E000102EC0CF0E7
:10C360000A000900F550EE6E0009FBE105010F51CE
:10C3700030093D6F050E0801A86F2D0EA76F000153
:10C38000C3EC25F03A0E05016C6F010E6D6F0001D4
:10C3900032EC50F0ABD10101D36BD38BC4A10AD0E6
:10C3A0005E0EF66E250EF76E000EF86E0001B9EC0B
:10C3B0002DF00101050EEA6E2D0EE96E000E000152
:10C3C00015EC0CF00A000900F550EE6E0009FBE1D7
:10C3D00005010F5130093D6F050E0801A86F2D0EA4
:10C3E000A76F0001C3EC25F081D10101D36B300EA2
:10C3F000D313C4A10AD0700EF66E250EF76E000E90
:10C40000F86E0001B9EC2DF00101050EEA6E2D0E5B
:10C41000E96E000E000128EC0CF00A000900F5504E
:10C42000EE6E0009FBE105010F5130093D6F050E6D
:10C430000801A86F2D0EA76F0001C3EC25F056D19F
:10C440000501122D27D01351050824E1102D22D00B
:10C45000115320E10101D36B900ED313C4A10AD074
:10C46000820EF66E250EF76E000EF86E0001B9EC26
:10C470002DF00101050EEA6E2D0EE96E000E000191
:10C480003BEC0CF00A000900F550EE6E0009FBE1F0
:10C490001ED005010101D36BD389C4A10AD0940E2B
:10C4A000F66E250EF76E000EF86E0001B9EC2DF059
:10C4B0000101050EEA6E2D0EE96E000E00014EEC34
:10C4C0000CF00A000900F550EE6E0009FBE10501D1
:10C4D0000F5130093D6F050E0801A86F2D0EA76F93
:10C4E0000001C3EC25F002D10101D36BD38FC4A1AD
:10C4F0000AD0A40EF66E250EF76E000EF86E00013F
:10C50000B9EC2DF00101050EEA6E2D0EE96E000E5C
:10C51000000161EC0CF00A000900F550EE6E000914
:10C52000FBE105010F5130093D6F050E0801A86FB1
:10C530002D0EA76F0001C3EC25F0D8D00101D36BFD
:10C54000700ED313C4A10AD0B60EF66E250EF76E88
:10C55000000EF86E0001B9EC2DF00101050EEA6E37
:10C560002D0EE96E000E000174EC0CF00A000900BB
:10C57000F550EE6E0009FBE105010F5130093D6FEA
:10C58000050E0801A86F2D0EA76F0001C3EC25F062
:10C59000ADD00101D36BF00ED313C4A10AD0C80EE5
:10C5A000F66E250EF76E000EF86E0001B9EC2DF058
:10C5B0000101050EEA6E2D0EE96E000E000187ECFA
:10C5C0000CF00A000900F550EE6E0009FBE10501D0
:10C5D0000F5130093D6F050E0801A86F2D0EA76F92
:10C5E0000001C3EC25F01B0E05016F6F010E706F8B
:10C5F000000122EC44F07AD00101D36BD38DC4A1A9
:10C600000AD0DA0EF66E250EF76E000EF86E0001F7
:10C61000B9EC2DF00101050EEA6E2D0EE96E000E4B
:10C6200000019AEC0CF00A000900F550EE6E0009CA
:10C63000FBE105010F5130093D6F050E0801A86FA0
:10C640002D0EA76F0001C3EC25F050D00101D36B74
:10C65000A00ED313C4A10AD0EC0EF66E250EF76E11
:10C66000000EF86E0001B9EC2DF00101050EEA6E26
:10C670002D0EE96E000E0001ADEC0CF00A00090071
:10C68000F550EE6E0009FBE105010F5130093D6FD9
:10C69000050E0801A86F2D0EA76F0001C3EC25F051
:10C6A00025D00101C4A10AD0040EF66E260EF76E45
:10C6B000000EF86E0001B9EC2DF00101D36B050EF0
:10C6C000EA6E2D0EE96E000E0001C0EC0CF00A00BF
:10C6D0000900F550EE6E0009FBE1050E0801A86F98
:10C6E0002D0EA76F0001C3EC25F000D063D005012B
:10C6F0002B5103083BE11E3D39D01C51600803E07B
:10C700001C51610833E1416B0001C3EC5DF0012C69
:10C710002DD00101D36B600ED313C4A10AD0160E25
:10C72000F66E260EF76E000EF86E0001B9EC2DF0D5
:10C730000101050EEA6E2D0EE96E000E0001D2EC2D
:10C740000CF00A000900F550EE6E0009FBE105014E
:10C750000F5130093D6F050E0801A86F2D0EA76F10
:10C760000001C3EC25F0010126D000010101C4A1A4
:10C770000AD02A0EF66E260EF76E000EF86E000135
:10C78000B9EC2DF00101D36B050EEA6E2D0EE96EAA
:10C79000000E0001C0EC0CF00A000900F550EE6E2E
:10C7A0000009FBE1050E0801A86F2D0EA76F00011F
:10C7B000C3EC25F0010100012FEF65F0040EEA6ED5
:10C7C000F10EE96E0801E56BE76B140EE66F0001F0
:10C7D0006BEC25F0340E05016F6F706B000183EC7C
:10C7E0003DF01DEF41F00152D8A467D105016F6BF8
:10C7F000706B000122EC44F0070E0601376FD00E7B
:10C80000366F0001D0EC41F00152D8A424D10501CB
:10C810006F6B706B000122EC44F0070E0601376F5E
:10C82000D00E366F0001D0EC41F00152D8A413D1E4
:10C830000101C3BB28D0040EEA6EF10EE96E000EB2
:10C84000000131EC0BF00A000900F550EE6E000912
:10C85000FBE10401F05130090501016F040E0801EC
:10C86000A86FF10EA76F0001C3EC25F0040E0501BF
:10C870000F6FFA0E0801E56F00013FEC20F0050193
:10C880000F2FF7D7C5D10D0E05016F6F706B00012B
:10C8900062EC4AF0320E0801E56F00013FEC20F037
:10C8A000050E0501246F236F0A0E256F3A0E276FC0
:10C8B000980E266F010E286F000103EC4EF0012C3C
:10C8C00001D029D0040EEA6EF10EE96E000E31ECB3
:10C8D0000BF00A000900F550EE6E0009FBE10401BF
:10C8E000F05130090501016F040E0801A86FF10E27
:10C8F000A76F0001C3EC25F0040E05010F6FFA0EBF
:10C900000801E56F00013FEC20F005010F2FF7D77C
:10C910007FD1A0D000010101D36BD00ED313040E40
:10C92000EA6EF10EE96E000E000144EC0BF00A0015
:10C930000900F550EE6E0009FBE10401F0513009E9
:10C940000501016F040E0801A86FF10EA76F000129
:10C95000C3EC25F00101C4A109D0260EF66E240E09
:10C96000F76E000EF86E0001B9EC2DF0040E050113
:10C970000F6FFA0E0801E56F00013FEC20F0050192
:10C980000F2FF7D7130EDA6F880ED96FDB6B00010C
:10C9900038EC49F027EC33F00101C3A307D0F0C411
:10C9A0000FF500010BEC5AF038D00101320E0501F1
:10C9B0006F6F706B000162EC4AF01F0E0501DA6FB9
:10C9C000400ED96F010EDB6F000138EC49F0200EEC
:10C9D00005010F6FFA0E0801E56F00013FEC20F032
:10C9E00005010F2FF7D7000127EC33F03F0E0501AB
:10C9F0006F6F706B000162EC4AF01F0E0501DA6F79
:10CA0000400ED96F010EDB6F000138EC49F00101D7
:10CA1000D383D385D387D3910001036A0401F051F6
:10CA2000E30FE96E010E0320EA6ED3C1EFFF0001B0
:10CA30009FEC5CF0D8900401F035036AF80FE96EC2
:10CA4000010E0320EA6EDEC1ECFFED52DDC1EFFF07
:10CA50000501DED00001F0C40FF58CEF5EF001019E
:10CA6000D35302E10501D4D00D0E05016F6F706B39
:10CA7000000122EC44F04E0E0601376F200E366F97
:10CA80000001D0EC41F00101C3A307D0F0C40FF5C1
:10CA900000010BEC5AF010D00101320E05016F6F4E
:10CAA000706B000122EC44F04E0E0601376F200E31
:10CAB000366F0001D0EC41F067D00101D36BC00E9E
:10CAC000D313040EEA6EF10EE96E000E000157EC6E
:10CAD0000BF00A000900F550EE6E0009FBE10401BD
:10CAE000F05130090501016F040E0801A86FF10E25
:10CAF000A76F0001C3EC25F00101C4A109D03C0ED1
:10CB0000F66E240EF76E000EF86E0001B9EC2DF0F3
:10CB1000000127EC33F00D0E05016F6F706B000103
:10CB200083EC3DF01F0E0801D36F400ED26F000161
:10CB300080EC34F027EC33F01A0E05016C6F6D6B4E
:10CB4000000132EC50F0030E0801D36FE80ED26FF3
:10CB5000000180EC34F00101C3A307D0F0C40FF54D
:10CB600000010BEC5AF010D00101320E05016F6F7D
:10CB7000706B000183EC3DF0170E0801D36F700E4F
:10CB8000D26F000180EC34F00101D383110E050156
:10CB90006C6F010E6D6F000132EC50F00101D38714
:10CBA0001C0E05016C6F010E6D6F000132EC50F030
:10CBB0000101D385150E05016C6F010E6D6F00012B
:10CBC00032EC50F00101D391100E05016C6F010E93
:10CBD0006D6F000132EC50F0036A02011051E30F57
:10CBE000E96E010E0320EA6ED3C1EFFF00019FEC56
:10CBF0005CF0D89002011035036AF80FE96E010E5F
:10CC00000320EA6EDEC1ECFFED52DDC1EFFF05014E
:10CC1000000163EF66F0010EEA6EE30EE96E0801B3
:10CC2000E56BE76B070EE66F00016BEC25F037EC68
:10CC300030F00101C4A109D0F80EF66E230EF76E94
:10CC4000000EF86E0001B9EC2DF0010E0401EF6F3B
:10CC5000EF5106083BE30101C4A122D01A0EF66E83
:10CC6000240EF76E000EF86E050E0801E56F000148
:10CC700069EC29F0EFC4ADF81F0E0801AE6F00019A
:10CC800068EC30F03A0E9EA8FED7AD6E200E9EA83E
:10CC9000FED7AD6E200E9EA8FED7AD6E07D0010167
:10CCA000320E0801E56F00013FEC20F0EFC40DF5F6
:10CCB000F4EC3CF00A0E0801E56F00013FEC20F0B7
:10CCC000EFC4F0F47BD50401EF2BC2D70001000CB8
:10CCD000040EEA6EFA0EE96E0801E56BE76B130EBF
:10CCE000E66F00016BEC25F0050EEA6E0D0EE96EA5
:10CCF0000801E56BE76B130EE66F00016BEC25F0A6
:10CD00000C01E26BF8C4E1FCE46B120EE36F00016E
:10CD100058EC29F002C003F001505C0F016E020EC6
:10CD2000032201C020F503C021F5040E0801D06FD5
:10CD3000FA0ECF6F03C0D2F801C0D1F8D46B120E37
:10CD4000D36F00017AEC25F00C0E0401FA6F036A30
:10CD50000301C451C50FE96E030E0320EA6EEF2CE8
:10CD600003D03E0E0401FB6F040E0801D06FFA0ED3
:10CD7000CF6F000149EC21F0050E0801E56F0001BD
:10CD80003FEC20F00C01E26BF9C4E1FCE46B120E05
:10CD9000E36F000158EC29F002C003F001505C0F72
:10CDA000016E020E032201C020F503C021F5050E1D
:10CDB0000801D06F0D0ECF6F03C0D2F801C0D1F8BB
:10CDC000D46B120ED36F00017AEC25F00A0E050128
:10CDD0000D6F036A0301C451C50FE96E030E0320F2
:10CDE000EA6EEF50020803E13E0E05010E6F050EDC
:10CDF0000801D06F0D0ECF6F000149EC21F0000C3F
:10CE00000401EF6BEF6BEF51020821E3036AEF516E
:10CE1000C50FE96E030E0320EA6EEF6A036AEF5155
:10CE2000C90F016E030E032203C0F1F4036AEF5130
:10CE3000D10FE96E030E0320EA6EEFCFF2F4F1C4D6
:10CE4000EAFF01C0E9FFF2C4EFFFEF2BDCD70301DB
:10CE5000C46B01016993699569970401656B65C4A9
:10CE600067F467C466F4036A0301C451C90FE96E2D
:10CE7000030E0320EA6EEFCFF0F4036AC451C90F2A
:10CE8000E96E030E0320EA6E010EEF240401F16F38
:10CE9000F0C4F8F4F96F00011BDF000C0401D86B3B
:10CEA000D76BD96BDA6BFA0E0801D36F00012AEC4D
:10CEB00020F0FF0E0401A86FA76FA96FAC6BAB6FDA
:10CEC000AA6F5D905A9E476A466A496A486A4E6AE6
:10CED0005D925D945D965E6A5F6A0001606B616B56
:10CEE0000401DA6BDA510C080AE3036ADA514F0FD6
:10CEF000E96E020E0320EA6EEF6ADA2BF3D7010E19
:10CF0000EA6EC10EE96E0801E56BE76B590EE66F3C
:10CF100000016BEC25F00401DA6BDA510108D8A0AE
:10CF200086D0DA51040DF350F06BEF6F6B0EEF25E6
:10CF3000E96E040EF021EA6EFF0EEC6EED52EF6E1C
:10CF4000DA51040DF350F06BEF6F020EEF25016E16
:10CF5000000EF021036E01506B0FE96E040E0320EA
:10CF6000EA6EEF6ADA51040DF350F06BEF6F770E53
:10CF7000EF25E96E040EF021EA6EFF0EEC6EED5225
:10CF8000EF6EDA51040DF350F06BEF6F020EEF25E8
:10CF9000016E000EF021036E0150770FE96E040E52
:10CFA0000320EA6EEF6ADA51040DF350F06BEF6F75
:10CFB000830EEF25E96E040EF021EA6EFF0EEC6E93
:10CFC000ED52EF6EDA51040DF350F06BEF6F020E7D
:10CFD000EF25016E000EF021036E0150830FE96E04
:10CFE000040E0320EA6EEF6ADA51040DF350F06B81
:10CFF000EF6F8F0EEF25E96E040EF021EA6EFF0E43
:10D00000EC6EED52EF6EDA51040DF350F06BEF6FF2
:10D01000020EEF25016E000EF021036E01508F0FFE
:10D02000E96E040E0320EA6EEF6ADA2B76D7040E5F
:10D03000EA6EC30EE96E000E000162EC10F00A0009
:10D040000900F550EE6E0009FBE1040E0801A86F1F
:10D05000C30EA76F0001C3EC25F05EEF2CF0040EA9
:10D060000401EF6FFA0E0801D36F00012AEC20F0E3
:10D070000401EF2FF7D79D80F28A070EB46E975008
:10D08000976E0D0E006E002EFED7B450A19CB56AAF
:10D09000FA0E0801D36F00012AEC20F013C26CF4E1
:10D0A00012C26BF413C270F412C26FF41B6AF2BEA8
:10D0B0001B8EF29E400E0C01E86FE96B000168ECDC
:10D0C0001AF01BBEF28E02C0D8F401C0D7F41B6A5E
:10D0D000F2BE1B8EF29E440E0C01E86FE96B00015C
:10D0E00068EC1AF01BBEF28E02C0D8F401C0D7F46F
:10D0F0001B6AF2BE1B8EF29E420E0C01E86FE96BBA
:10D10000000168EC1AF01BBEF28E02C0D8F401C018
:10D11000D7F41B6AF2BE1B8EF29E460E0C01E86F1E
:10D12000E96B000168EC1AF01BBEF28E02C0D8F465
:10D1300001C0D7F4010EEA6E6A0EE96E0801E56BD4
:10D14000E76B400EE66F00016BEC25F0666B66C086
:10D1500064F001016991040E0801A86FC30EA76F66
:10D160000001C3EC25F0676B0D0E686FEA6A6A0E6A
:10D17000E96E0801E56BE76BFF0EE66F00016BECF3
:10D1800025F0656B65C063F05D9EA38A9D8AC00E25
:10D19000F2120101C1A14BD1040EEA6EC30EE96E79
:10D1A000000E000175EC10F00A000900F550EE6E5B
:10D1B0000009FBE1040E0801A86FC30EA76F000170
:10D1C000C3EC25F0ACEC2DF04E0EF66E400EF76E73
:10D1D000000EF86EB9EC2DF0040E0401F06FDB0EBA
:10D1E000EF6F140EF16F0001FCEF2EF0012C23D035
:10D1F000040EEA6EC30EE96E000E87EC10F00A0012
:10D200000900F550EE6E0009FBE1040E0801A86F5D
:10D21000C30EA76F0001C3EC25F0080E0401EF6FE9
:10D22000FA0E0801D36F00012AEC20F00401EF2F61
:10D23000F7D7D4D00001F2CFEFF4F29EAA6A110E14
:10D24000A96EA69CA69EA680A8500401EFBFF28EF0
:10D25000D96FD9B1A1D0D981AA6A110EA96ED9C44A
:10D26000A8FFA69CA69EA684F250006EF29E0F0117
:10D27000550EA76EAA0EA76EA682A6B2FED7A694DA
:10D280000050F212040EEA6EC30EE96E000E0001A9
:10D2900099EC10F00A000900F550EE6E0009FBE170
:10D2A000040E0801A86FC30EA76F0001C3EC25F0A0
:10D2B000280E0401EF6FFA0E0801D36F00012AEC6B
:10D2C00020F00401EF2FF7D7040EEA6EC30EE96ECB
:10D2D000000E0001ACEC10F00A000900F550EE6EF3
:10D2E0000009FBE1040E0801A86FC30EA76F00013F
:10D2F000C3EC25F0280E0401EF6FFA0E0801D36F7E
:10D3000000012AEC20F00401EF2FF7D7040EEA6E9B
:10D31000C30EE96E000E0001BFEC10F00A00090018
:10D32000F550EE6E0009FBE1040E0801A86FC30E74
:10D33000A76F0001C3EC25F0280E0401EF6FFA0E71
:10D340000801D36F00012AEC20F00401EF2FF7D77A
:10D35000040EEA6EC30EE96E000E0001D2EC10F06E
:10D360000A000900F550EE6E0009FBE1040E080109
:10D37000A86FC30EA76F0001C3EC25F0040E0401D3
:10D38000EF6FFA0E0801D36F00012AEC20F00401C0
:10D39000EF2FF7D7FF0022D0040EEA6EC30EE96E1E
:10D3A000000E0001E4EC10F00A000900F550EE6EEA
:10D3B0000009FBE1040E0801A86FC30EA76F00016E
:10D3C000C3EC25F0080E0401EF6FFA0E0801D36FCD
:10D3D00000012AEC20F00401EF2FF7D7F2CFEFF491
:10D3E000F29EAA6A110EA96EA69CA69EA680A850BF
:10D3F000EFBFF28ED96FD9A118D0D991AA6A110EB8
:10D40000A96ED9C4A8FFA69CA69EA684F250006E61
:10D41000F29E0F01550EA76EAA0EA76EA682A6B2A7
:10D42000FED7A6940050F21204012CD10101C1A331
:10D430002AD1040EEA6EC30EE96E000E0001F7EC6D
:10D4400010F00A000900F550EE6E0009FBE1040E31
:10D450000801A86FC30EA76F0001C3EC25F0ACEC68
:10D460002DF0670E9EA8FED7AD6E040E0501276F46
:10D47000DB0E266F140E286F0001CEEC2DF0012C70
:10D480002ED00401DB51450828E1DC514F0825E18D
:10D49000DD514E0822E1040EEA6EC30EE96E000E65
:10D4A00000010AEC11F00A000900F550EE6E0009C7
:10D4B000FBE1040E0801A86FC30EA76F0001C3ECC7
:10D4C00025F0080E0401EF6FFA0E0801D36F00017A
:10D4D0002AEC20F00401EF2FF7D7D4D00001F2CFCF
:10D4E000EFF4F29EAA6A110EA96EA69CA69EA680D3
:10D4F000A8500401EFBFF28ED96FD9B1A1D0D98164
:10D50000AA6A110EA96ED9C4A8FFA69CA69EA684DD
:10D51000F250006EF29E0F01550EA76EAA0EA76E76
:10D52000A682A6B2FED7A6940050F212040EEA6EAE
:10D53000C30EE96E000E00011DEC11F00A00090097
:10D54000F550EE6E0009FBE1040E0801A86FC30E52
:10D55000A76F0001C3EC25F0280E0401EF6FFA0E4F
:10D560000801D36F00012AEC20F00401EF2FF7D758
:10D57000040EEA6EC30EE96E000E000130EC11F0ED
:10D580000A000900F550EE6E0009FBE1040E0801E7
:10D59000A86FC30EA76F0001C3EC25F0280E04018D
:10D5A000EF6FFA0E0801D36F00012AEC20F004019E
:10D5B000EF2FF7D7040EEA6EC30EE96E000E0001DE
:10D5C00043EC11F00A000900F550EE6E0009FBE192
:10D5D000040E0801A86FC30EA76F0001C3EC25F06D
:10D5E000280E0401EF6FFA0E0801D36F00012AEC38
:10D5F00020F00401EF2FF7D7040EEA6EC30EE96E98
:10D60000000E000156EC11F00A000900F550EE6E14
:10D610000009FBE1040E0801A86FC30EA76F00010B
:10D62000C3EC25F0040E0401EF6FFA0E0801D36F6E
:10D6300000012AEC20F00401EF2FF7D7FF0022D0E1
:10D64000040EEA6EC30EE96E000E000169EC11F0E3
:10D650000A000900F550EE6E0009FBE1040E080116
:10D66000A86FC30EA76F0001C3EC25F0080E0401DC
:10D67000EF6FFA0E0801D36F00012AEC20F00401CD
:10D68000EF2FF7D70101C1B102D0C1A329D0F2CF4A
:10D69000EFF4F29EAA6A110EA96EA69CA69EA68021
:10D6A000A8500401EFBFF28ED96FD9A118D0D9913B
:10D6B000AA6A110EA96ED9C4A8FFA69CA69EA6842C
:10D6C000F250006EF29E0F01550EA76EAA0EA76EC5
:10D6D000A682A6B2FED7A6940050F2120401010160
:10D6E000040EEA6EC30EE96E000E000116EC10F097
:10D6F0000A000900F550EE6E0009FBE1040E080176
:10D70000A86FC30EA76F0001C3EC25F00BEC66F009
:10D7100000EC67F0640E0801D36F00012AEC20F0E2
:10D720000401A9911B6AF2BE1B8EF29E480E0C01E9
:10D73000F16F010EF26FA9C4F3FC0001F5EC1BF0D0
:10D740001BBEF28E0A0E0801D36F00012AEC20F0F6
:10D75000468AC6C114F24B8A0101C4A506D0C48909
:10D76000010802E14B8401D04B820201106B116B66
:10D77000036A0101C651E30FE96E010E0320EA6E50
:10D78000EF50F00B08E0C6C116F24C80C3B303D0D3
:10D79000C7C117F24C82050E0801D36F00012AECB5
:10D7A00020F00101C5B701D09D9A0001ACEC2DF02D
:10D7B000CBEFF5F0020111530BE0080199517F0BFB
:10D7C00006E197517F0B03E198517F0B01E0488CF4
:10D7D0000101D339006E0F0E00160050FF0FF10F3C
:10D7E00023E20F0F000116EF6CF097C89AF898C863
:10D7F0009BF899C89CF83BEC33F0010115D097C811
:10D800009AF898C89BF899C89CF875EC35F0010116
:10D810000BD097C89AF898C89BF899C89CF834EC34
:10D820003AF0010101D001010001000CE824F76A7F
:10D83000F7364D0FF66ED80EF722000EF86EFB6E1F
:10D840000A00F550FA6E0800F550F96EEAD7EAD7EB
:10D85000EAD7EAD7EAD7EAD7EAD7EAD7EAD7EAD7C0
:10D86000EAD7FED712D826D8EAD70401C36BC46B17
:10D87000C56B140EC66F180EC76F070EC86FC96B45
:10D88000050ECA6F060ECB6F120ECC6F0101D33995
:10D89000006E0F0E00160050020A00011DE0070A7C
:10D8A00024E0010A2BE00E0A32E0020A30E0010A0D
:10D8B0002EE00E0A2CE0080A2AE0040A28E0070AF3
:10D8C0002FE0010A36E0030A3CE00F0A43E0070AB2
:10D8D00041E0050A49E052D0120E0401C76F0D0E57
:10D8E000C66F070EC86FC96B4BD00C0E0401C76F13
:10D8F0000A0EC66F070EC86FC96B42D0100E040126
:10D90000C76F0C0EC66F070EC86FC96B39D0180EE3
:10D910000401C76F140EC66F070EC86FC96B30D0F5
:10D92000180E0401C76F080EC66F070EC86FC96BCB
:10D9300027D0180E0401C76F140EC66F070EC86FEC
:10D940001FD0140E0401C76F0C0EC66F070EC86FF0
:10D95000C96B16D0180E0401C76F140EC66F070EE0
:10D96000C86F020EC96F0CD0100E0401C76F0A0EEB
:10D97000C66F070EC86FC96B03D000016BD20401DC
:10D98000C7510101CF5D02E2CFC1C7F40401C65106
:10D990000101D05D02E2D0C1C6F41B6AF2BE1B8E4B
:10D9A000F29E7F0E0C01E86FC7C4E9FC0001CFECCA
:10D9B0001AF01BBEF28E01C0CAF41B6AF2BE1B8EA7
:10D9C000F29E7F0E0C01E86FC6C4E9FC0001CFECAB
:10D9D0001AF01BBEF28E01C0CBF41B6AF2BE1B8E86
:10D9E000F29E7F0E0C01E86FC8C4E9FC0001CFEC89
:10D9F0001AF01BBEF28E01C0CCF40101D339006EC7
:10DA00000F0E001600500A0807E0D339006E0F0E03
:10DA1000001600500B0824E1D339006E0F0E0016DB
:10DA200000500B08D8A40ED1D89002011035036A1B
:10DA3000EA0FE96E010E0320EA6EECCFCEF4ED5250
:10DA4000EFCFCDF40401CD510208D8B402D00101CA
:10DA500007D0CE2D01D002D0010102D00101F2D0B9
:10DA6000D890D131FF0A800FC0533AE1BF5D38E250
:10DA7000800ED880BF550401CD6FD8900101D131FF
:10DA80000401CD5DCE6F1B6AF2BE1B8EF29EE8CF05
:10DA9000E8FCCAC4E9FC0001CFEC1AF01BBEF28E10
:10DAA00001C0C4F40401C451C75D03E2C7C4C4F497
:10DAB00004D0C45302E1010EC46FCAC100F00201D8
:10DAC0001051016E04E0D8900032012EFCD700A066
:10DAD00003D00401C49F02D00401C48F3ED00101D1
:10DAE000D890D1317F0FC05303E1BF5D37E036E3FB
:10DAF000800EBF5D0401CD6FD8900101D1310401CA
:10DB0000CD5DCE6F1B6AF2BE1B8EF29EE8CFE8FCA5
:10DB1000CAC4E9FC0001CFEC1AF01BBEF28E01C0B2
:10DB2000C4F40401C451C75D03E2C7C4C4F404D003
:10DB3000C45302E1010EC46FCAC100F002011051CA
:10DB4000016E04E0D8900032012EFCD700A003D073
:10DB50000401C48F02D00401C49F01017F0ED8804C
:10DB6000D155BE5336E1BD5D34E2800ED880BD553F
:10DB7000D880D1550401CE6F1B6AF2BE1B8EF29E77
:10DB8000E8CFE8FCCBC4E9FC0001CFEC1AF01BBEE7
:10DB9000F28E01C0C3F40401C351C65D03E2C6C4E2
:10DBA000C3F404D0C35302E1010EC36FCBC100F034
:10DBB00002011051016E04E0D8900032012EFCD712
:10DBC00000A003D00401C38F02D00401C39F39D049
:10DBD00001017F0ED125BE5303E1BD5D33E032E389
:10DBE000800EBD5DD880D1550401CE6F1B6AF2BE98
:10DBF0001B8EF29EE8CFE8FCCBC4E9FC0001CFEC21
:10DC00001AF01BBEF28E01C0C3F40401C351C65DFD
:10DC100003E2C6C4C3F404D0C35302E1010EC36FD0
:10DC2000CBC100F002011051016E04E0D890003227
:10DC3000012EFCD700A003D00401C39F02D0040131
:10DC4000C38F0101D890D131FF0A800FBC5343E14B
:10DC5000BB5D41E2800ED880BB550401CD6FD890EA
:10DC60000101D1310401CD5DCE6F1B6AF2BE1B8E66
:10DC7000F29EE8CFE8FCCCC4E9FC0001CFEC1AF03E
:10DC80001BBEF28E01C0C5F40401C551C85D03E29C
:10DC9000C8C4C5F405D0C551C95D02E3C9C4C5F403
:10DCA0000101D339006E0F0E001600500D0804E07C
:10DCB0000401C58706D001010401C55302E1010E2C
:10DCC000C56F0101C5A303D00401C58F02D00401B3
:10DCD000C59F47D00101D890D1317F0FBC5303E1DC
:10DCE000BB5D40E03FE3800EBB5D0401CD6FD8908B
:10DCF0000101D1310401CD5DCE6F1B6AF2BE1B8ED6
:10DD0000F29EE8CFE8FCCCC4E9FC0001CFEC1AF0AD
:10DD10001BBEF28E01C0C5F40401C551C85D03E20B
:10DD2000C8C4C5F405D0C551C95D02E3C9C4C5F472
:10DD30000101D339006E0F0E001600500D0804E0EB
:10DD40000401C58706D001010401C55302E1010E9B
:10DD5000C56F0101C5A303D00401C59F02D0040112
:10DD6000C58F0101AB510401C55D0DE10101AC514D
:10DD70000401C45D08E10101AD510401C35D03E18B
:10DD8000000168D00401C5C4ABF1C4C4ACF1C3C484
:10DD9000ADF10101D339006E0F0E001600500B08D3
:10DDA00051E10401C553D8A402D001014BD0D89051
:10DDB00002011035036AEA0FE96E010E0320EA6ED4
:10DDC000EF50006EE92AEF50E906036E030E035C84
:10DDD00004E10052000128E00201020E035C05E1AB
:10DDE000010E005C000120E00201020E035C04E170
:10DDF0000052000119E00201010E035C04E100522F
:10DE0000000113E00201010E035C05E1010E005C5C
:10DE100000010BE00201010E035C05E1020E005C53
:10DE2000000103E0020101D00DD00401C551800BB7
:10DE3000CD6F0101CC517F0B08090401CD11C56FD5
:10DE4000000100D0C4C497F8C3C498F8C5C499F8B9
:10DE50000001B0DCD3EFF5F00401C56BC691C693A9
:10DE60001B6AF2BE1B8EF29E460E0C01E86FE96B38
:10DE7000000168EC1AF01BBEF28E02C0C4F401C0AF
:10DE8000C3F4FF0E0401C31BC41BC4C494F4C3C475
:10DE900093F4A9A107D0C3518008D8A4B5D0C45326
:10DEA000D8A4B2D0C351006EC451036E035005E133
:10DEB00000520001D8B478D00401035006E1010EED
:10DEC000005C0001D8B478D00401200E035C05E1A9
:10DED00000520001D8B475D00401035006E1020ECF
:10DEE000005C0001D8B472D00401020E035C05E1AD
:10DEF00000520001D8B46AD00401040E035C05E1AD
:10DF000000520001D8B462D00401080E035C05E1A0
:10DF100000520001D8B45AD00401400E035C04E161
:10DF20000052000153E00401800E035C04E1005242
:10DF300000014CE00401035005E1400E005C0001CB
:10DF400049E00401035005E1200E005C000142E0BD
:10DF50000401035005E1800E005C000141E0040172
:10DF6000035005E1040E005C00013AE00401035097
:10DF700005E1080E005C000133E00401035005E1F7
:10DF8000100E005C00012CE00401010E035C04E1B2
:10DF90000052000125E00401100E035C04E1005270
:10DFA00000011EE004011ED05DB402D05DA601D0C8
:10DFB000488A5D945D9627D00401C6815D84000186
:10DFC00022D00401C6815D8600011DD00401C681F6
:10DFD000000119D0626B5D980401C691000113D055
:10DFE0000401C6815AB406D047BA04D05ABE02D042
:10DFF0005DA007D05D905A9E479A5AA402D04680F1
:10E000005A86000100D00401C6A105D0C5C495F40C
:10E01000958F5D9A4DD090C494F48FC493F4010110
:10E02000C4A147D00401C35302E1C45341E0C6B3C5
:10E030003FD0C351FF0AC76FC451FF0AC86F340EE7
:10E04000F66E320EF76E000EF86E100E0801E56FD8
:10E05000000169EC29F0C8C4E6F8370E0801E76F43
:10E06000000182EC29F0C7C4E6F8370E0801E76F1B
:10E07000000182EC29F0200E9EA8FED7AD6EC4C42C
:10E08000E6F8370E0801E76F000182EC29F0C3C4FF
:10E09000E6F8370E0801E76F000182EC29F00A0E5E
:10E0A0009EA8FED7AD6E0D0E9EA8FED7AD6E0401E4
:10E0B00001010001FBEFAAF00401F76B010EF76FFD
:10E0C000F75106081CE3F7C40DF50001F4EC3CF031
:10E0D0000401F62D09D00E0E05016C6F010E6D6F57
:10E0E000000132EC50F008D00D0E05016C6F010EEE
:10E0F0006D6F000132EC50F00401F72BE1D7000105
:10E1000086EF71F00401F66BF66BF651020821E31D
:10E11000036AF651C50FE96E030E0320EA6EEF6A3B
:10E12000036AF651C90F016E030E032203C0F8F40F
:10E13000036AF651D10FE96E030E0320EA6EEFCFAA
:10E14000F9F4F8C4EAFF01C0E9FFF9C4EFFFF62BC8
:10E15000DCD7F76B000137EC23F00301C46B01013E
:10E160006993699569970401656B65C467F467C431
:10E1700066F4036A0301C451C90FE96E030E03205C
:10E18000EA6EEFCFF7F4F7C4F8F4130E0401F96F59
:10E19000000168EC66F087EF71F00401E16BE06B61
:10E1A000DF2D1BD0A9A118D0040EEA6EE20EE96E95
:10E1B000000E00017CEC11F00A000900F550EE6E33
:10E1C0000009FBE1040E0801A86FE20EA76F000131
:10E1D000C3EC25F0FF0004019FD0DF53D8A49CD0EE
:10E1E000A9B19AD00301C46B036AC451C50FE96E8B
:10E1F000030E0320EA6E010EEF6E040EEA6EE20ECD
:10E20000E96E000E0001E6EC0FF00A000900F5507F
:10E21000EE6E0009FBE1040E0801D06FE20ECF6F35
:10E22000000149EC21F0040EEA6EE20EE96E000EE8
:10E230008FEC11F00A000900F550EE6E0009FBE1C9
:10E24000040E0801D06FE20ECF6F000149EC21F0FF
:10E25000FF0E0401A86FA76FA96FAB6FAA6F1B6AAF
:10E26000F2BE1B8EF29E480E0C01F16F010EF26F92
:10E27000A9C4F3FC0001F5EC1BF01BBEF28E1B6A77
:10E28000F2BE1B8EF29E4C0E0C01EA6FEB6BA8C423
:10E29000EDFCA7C4ECFC000121EC1CF01BBEF28ECF
:10E2A0001B6AF2BE1B8EF29E4A0E0C01EA6FEB6BEC
:10E2B000ABC4EDFCAAC4ECFC000121EC1CF01BBEBD
:10E2C000F28E0101C4A705D0800E0401E017E16BB6
:10E2D00005D07F0E0401E013FF0EE1131B6AF2BEAE
:10E2E0001B8EF29E400E0C01EA6FEB6BE1C4EDFC5D
:10E2F000E0C4ECFC000121EC1CF01BBEF28EBE6AF7
:10E300009D90010E0401F66F0001D6D6FBD60101E7
:10E31000C15301E09D9A04010001000C0401E06B6F
:10E32000DF6B020E0301C95DF00FD8B037D1100FBB
:10E330000001D1EF72F0040165530CE1468CD1C3AA
:10E34000C9F3036A0301C451C50FE96E030E03202C
:10E35000EA6EEF6A030122D10401652D04D00101A8
:10E36000C38B03D004010101C39B468E030116D168
:10E37000040165510101C65D03E065C4C6F1468E26
:10E3800003010CD1040165510101C75D03E065C4BF
:10E39000C7F1468E030102D1040165510101C95D37
:10E3A00003E065C4C9F1468E0301F8D0040165534A
:10E3B00005E10101C595468E06D00401652D03D007
:10E3C0000101C585468E0301E9D0040165510101B3
:10E3D000C85D03E065C4C8F1468E0301DFD00401C7
:10E3E000655305E10101C591468E06D00401652DF6
:10E3F00003D00101C581468E0301D0D004016551CF
:10E400000101CE5D04E065C4CEF1468E07D0CE5149
:10E41000030DF3CFE1F40401E1C4BEFF0301BED05C
:10E42000040165510101CD5D03E065C4CDF1468E67
:10E430000301B4D00401655305E10101C593468E83
:10E4400006D00401652D03D00101C583468E03016A
:10E45000A5D00101C16BC26B0401652D04D001017F
:10E46000C1812CD004016551020804E10101C1837E
:10E4700025D004016551030805E10101C185C2836E
:10E480001DD004016551040805E10101C185C28563
:10E4900015D004016551050805E10101C185C2815E
:10E4A0000DD004016551060804E10101C18706D0C1
:10E4B00004016551070803E10101C18904016553A5
:10E4C00004E00101C493C4910401468E030166D0A7
:10E4D0001B6AF2BE1B8EF29E400E0C01E86FE96BC8
:10E4E000000168EC1AF01BBEF28E02C0E0F401C01D
:10E4F000DFF40401655307E1800EDF17E06B0101D3
:10E50000C49709D00401652D07D07F0EDF13FF0EDD
:10E51000E0130101C48704011B6AF2BE1B8EF29E48
:10E52000400E0C01EA6FEB6BE0C4EDFCDFC4ECFCC9
:10E53000000121EC1CF01BBEF28E468E03012ED092
:10E54000040165510101CF5D03E065C4CFF1468E42
:10E55000030124D0040165510101D05D03E065C4CD
:10E56000D0F1468E03011AD004016551010A000161
:10E5700005E0030A07E0020A09E008D00101C58BA3
:10E58000C59D08D00101C58DC59B04D00101C59B67
:10E59000C59D00D0468E030101D00301030176EF33
:10E5A00074F0E824F76AF736C30FF66EE50EF7222B
:10E5B000000EF86EFB6E0A00F550FA6E0800F5507A
:10E5C000F96E36E358E370E384E340E554E598E3FD
:10E5D000ACE3CAE3DEE334E4FCE368E552E420E4C0
:10E5E000D0E4010E0301CA5DF90F52E2070F0001EA
:10E5F0004BEF73F00401655305E10101C587478EB8
:10E6000006D00401652D04D00101C597478E040191
:10E61000468E03013DD00401655304E10101C58923
:10E6200005D00401652D03D00101C5990401468E72
:10E6300003012ED00401655301E14782030128D074
:10E640000401655301E14784030122D00401652DD3
:10E6500003D00101C48302D00101C493468E03019B
:10E6600017D00401652D03D00101C38302D001013D
:10E67000C393468E03010CD00401652D03D0010124
:10E68000C38902D00101C399468E030101D0030161
:10E69000030176EF74F0E824F76AF736B70FF66EE9
:10E6A000E60EF722000EF86EFB6E0A00F550FA6EC9
:10E6B0000800F550F96EF4E516E634E640E64CE65F
:10E6C00062E678E60401DF6B036A0301C451C90FF7
:10E6D000E96E030E0320EA6E010EEF5CF90FD8B06D
:10E6E00079D0070F0001EDEF73F00401DF2B00017B
:10E6F0000401DF2B00010401DF2B00010401DF2BEB
:10E7000000010401DF2B00010401DF2B00010401E3
:10E7100065532FE10301C451020815E10401DF53E1
:10E7200004E10101CA6B0ED00401010E006EDF513D
:10E73000016E04E0D8900036012EFCD70050FF0A8D
:10E740000101CA1714D00401DF5304E10101CB6BAE
:10E750000ED00401010E006EDF51016E04E0D8906E
:10E760000036012EFCD70050FF0A0101CB172ED036
:10E7700004010301C451020815E10401DF5305E15E
:10E78000FF0E0101CA6F0DD00401010E006EDF51B2
:10E79000016E04E0D8900036012EFCD70050010134
:10E7A000CA1314D00401DF5305E1FF0E0101CB6F42
:10E7B0000DD00401010E006EDF51016E04E0D8900F
:10E7C0000036012EFCD700500101CB13468E030109
:10E7D00001D00301030176EF74F0E824F76AF736FD
:10E7E000FB0FF66EE70EF722000EF86EFB6E0A00C6
:10E7F000F550FA6E0800F550F96E0EE708E702E7EB
:10E80000FCE6F6E6F0E6EAE6036A0301C451C50F4A
:10E81000E96E030E0320EA6EEF5002081EE1036A60
:10E82000C451C90FE96E030E0320EA6E010EEF5CBE
:10E830000401E06F036A0301C451C90FE96E030EBE
:10E840000320EA6EEFCFE1F4E0C4F8F4E1C4F9F498
:10E85000000168EC66F01BD00301036AC451C90FC4
:10E86000E96E030E0320EA6EEFCFE0F4036AC451B1
:10E87000C90FE96E030E0320EA6E010EEF240401B6
:10E88000E16FE0C4F8F4F96F000168EC66F0000C89
:10E8900001016993699569970401656B65C467F423
:10E8A00067C466F4FF0E656F0301C4530BE1C951E1
:10E8B0000D0808E10101CE51030DF3CFE0F404018E
:10E8C000E0C4BEFF0001A0DF000C0301C451FC0F37
:10E8D0000DE2040F00017AEF74F020D5030106D099
:10E8E00080D6030103D0EED6030100D00001D0DFB3
:10E8F000FFEF7AF0E824F76AF736150FF66EE90EA7
:10E90000F722000EF86EFB6E0A00F550FA6E080052
:10E91000F550F96EDAE8E0E8E6E8E6E8010169B307
:10E920003CD00301C45324E1036AC451C50FE96E0E
:10E93000030E0320EA6EEF6A036AC451C90F016E29
:10E94000030E0322040103C0E0F4036A0301C4516F
:10E95000D10FE96E030E0320EA6EEFCFE1F404015C
:10E96000E0C4EAFF01C0E9FFE1C4EFFF13D00301F7
:10E97000036AC451C50FE96E030E0320EA6E020E4E
:10E98000EF6E036AC451C90FE96E030E0320EA6EED
:10E99000010EEF6E000138DF02D0000179DF000CBC
:10E9A0000301C951120A00012FE0100A49E0010ACF
:10E9B0005BE00A0AD8B47FD0020AD8B498D0070A1C
:10E9C000D8B4B1D0030AD8B4D6D0010AD8B476D11D
:10E9D0001F0AD8B4AFD1170AD8B4D4D1010AD8B419
:10E9E000D1D1030AD8B4E4D1010AD8B4ECD10D0ACC
:10E9F000D8B4F4D1020AD8B4FCD1070AD8B404D2EE
:10EA00001D0AD8B40BD215D2010E0401F76F000114
:10EA100037EC23F0036A0301C451C90FE96E030EFA
:10EA20000320EA6E010EEF6E036AC451C50FE96E52
:10EA3000030E0320EA6E020EEF6E00016FDF00D2BC
:10EA4000030EEA6ED50EE96E000E88EC09F00A009E
:10EA50000900F550EE6E0009FBE10401666B656B81
:10EA600065C467F40001ECD1030EEA6ED50EE96EC1
:10EA7000000E98EC09F00A000900F550EE6E00094E
:10EA8000FBE1030EEA6EE70EE96E000EA8EC09F05A
:10EA90000A000900F550EE6E0009FBE1010E0401C9
:10EAA000666F676B656B0101C3AB03D00401652B17
:10EAB00001010001C5D1020E0401F76F000137EC1E
:10EAC00023F0036A0301C451C90FE96E030E03204A
:10EAD000EA6E010EEF6E036AC451C50FE96E030EB4
:10EAE0000320EA6E020EEF6E000118DFA9D1030EBB
:10EAF0000401F76F000137EC23F0036A0301C451EE
:10EB0000C90FE96E030E0320EA6E010EEF6E036A71
:10EB1000C451C50FE96E030E0320EA6E020EEF6EBC
:10EB20000001FCDE8DD1030EEA6ED50EE96E000EFB
:10EB3000B8EC09F00A000900F550EE6E0009FBE19F
:10EB4000030EEA6EE70EE96E000EC9EC09F00A004A
:10EB50000900F550EE6E0009FBE10401656B01014F
:10EB6000C5A303D00401652B0101010E0401666FEA
:10EB7000676B000165D1030EEA6ED50EE96E000EDB
:10EB8000DAEC09F00A000900F550EE6E0009FBE12D
:10EB9000030EEA6EE70EE96E000EECEC09F00A00D7
:10EBA0000900F550EE6E0009FBE1030EEA6EF90E66
:10EBB000E96E000EFEEC09F00A000900F550EE6E59
:10EBC0000009FBE1040EEA6E0B0EE96E000E10EC7C
:10EBD0000AF00A000900F550EE6E0009FBE1040E90
:10EBE000EA6E1D0EE96E000E22EC0AF00A00090022
:10EBF000F550EE6E0009FBE1040EEA6E2F0EE96E91
:10EC0000000E34EC0AF00A000900F550EE6E00091F
:10EC1000FBE1040EEA6E410EE96E000E46EC0AF0CE
:10EC20000A000900F550EE6E0009FBE1040EEA6EE1
:10EC3000530EE96E000E58EC0AF00A000900F55078
:10EC4000EE6E0009FBE10101C1A105D0010E040136
:10EC5000656F2ED00101C1A305D0020E0401656FBE
:10EC600027D00101C1A515D0C2A305D0030E040110
:10EC7000656F0DD00101C2A505D0040E0401656FBA
:10EC800006D00101C2A104D0050E0401656F010187
:10EC90000FD0C1A705D0060E0401656F09D0010190
:10ECA000C1A904D0070E0401656F02D00401656B91
:10ECB000060E0401666F676B0001C2D0030EEA6E98
:10ECC000D50EE96E000E6AEC0AF00A000900F55054
:10ECD000EE6E0009FBE1030EEA6EE70EE96E000E30
:10ECE0007BEC0AF00A000900F550EE6E0009FBE12A
:10ECF000030EEA6EF90EE96E000E8EEC0AF00A00C1
:10ED00000900F550EE6E0009FBE10101C5AB05D02D
:10ED1000010E0401656F09D00101C5AD04D0020EDA
:10ED20000401656F02D00401656B020E666F676BAC
:10ED3000000186D0030EEA6ED50EE96E000EA1EC3E
:10ED40000AF00A000900F550EE6E0009FBE1030E1F
:10ED5000EA6EE70EE96E000EB3EC0AF00A00090055
:10ED6000F550EE6E0009FBE10401656B0101C4A7DB
:10ED700003D00401652B0101010E0401666F676B6E
:10ED800000015ED001016985180E0401666F010E55
:10ED9000676F0301C951060A000103E0010A04E09C
:10EDA00006D0CFC165F403D0D0C165F400D048D0FF
:10EDB00001016985060E0401666FC6C165F4010E86
:10EDC000676F00013DD0010169850C0E0401666F7B
:10EDD000C7C165F4010E676F000132D0010169857A
:10EDE000180E0401666F010E676FC9C165F400015A
:10EDF00027D001016985140E0401666F010E676F4B
:10EE0000C8C165F400011CD001016985320E0401FE
:10EE1000666F676BCEC165F4000112D00101698590
:10EE20006987280E0401666F676BCDC165F4000128
:10EE300007D001016993699569976997000100D02E
:10EE400019EF7BF00301CA51030A000112E0070A1F
:10EE500010E0010A21E0040A46E0030A44E0040A43
:10EE6000D8B485D0010AD8B4A9D00F0AD8B4CDD06F
:10EE7000D2D0030EEA6ED50EE96E000E88EC09F0D2
:10EE80000A000900F550EE6E0009FBE10401666B13
:10EE9000656B65C467F4C5D0030EEA6ED50EE96EE6
:10EEA000000E98EC09F00A000900F550EE6E00091A
:10EEB000FBE1030EEA6EE70EE96E000EA8EC09F026
:10EEC0000A000900F550EE6E0009FBE1010E040195
:10EED000666F676B656B0101C4A303D00401652BEA
:10EEE000010104019ED0030EEA6ED50EE96E000EFC
:10EEF000C5EC0AF00A000900F550EE6E0009FBE1CE
:10EF0000030EEA6EE70EE96E000ED5EC0AF00A0079
:10EF10000900F550EE6E0009FBE1036A0301C451DC
:10EF2000C90FE96E030E0320EA6EEF50010A0001DB
:10EF300003E0030A0AE012D00401656B0101C5B7C2
:10EF400003D00401652B01010DD00401656B0101A3
:10EF5000C5B903D00401652B010104D00401656B20
:10EF6000010100D0010E0401666F676B5AD0030ED9
:10EF7000EA6ED50EE96E000EE5EC0AF00A00090013
:10EF8000F550EE6E0009FBE1030EEA6EE70EE96E46
:10EF9000000EF8EC0AF00A000900F550EE6E0009C8
:10EFA000FBE1010E0401666F676B656B0101C3A392
:10EFB00003D00401652B0101040133D0030EEA6E76
:10EFC000D50EE96E000E0BEC0BF00A000900F550AF
:10EFD000EE6E0009FBE1030EEA6EE70EE96E000E2D
:10EFE0001EEC0BF00A000900F550EE6E0009FBE183
:10EFF000010E0401666F676B656B0101C3A903D045
:10F000000401652B010104010CD00401F76B000120
:10F0100037EC23F03DDC01016993699569970401A0
:10F0200000D0000119EF7BF00401DF6B030EEA6EE4
:10F03000D50EE96E000E0001B8EC09F00A000900D7
:10F04000F550EE6E0009FBE1030EEA6EE70EE96E85
:10F05000000EC9EC09F00A000900F550EE6E000937
:10F06000FBE1010E0401666F676B036A0301C45183
:10F07000C90FE96E030E0320EA6EEF50070A000184
:10F080000FE0010A10E0030A11E0010A12E0070A8A
:10F0900013E0010A14E0030A15E0090A3DE043D039
:10F0A0000401DF2B00010401DF2B00010401DF2B31
:10F0B00000010401DF2B00010401DF2B000104012A
:10F0C000DF2B00010401DF5301E1DF2B0301C451F9
:10F0D00002080FE1CAC100F00401DF51016E04E033
:10F0E000D8900032012EFCD7656B00B0652B11D093
:10F0F0000301C45103080DE1CBC100F00401DF514D
:10F10000016E04E0D8900032012EFCD7656B00B090
:10F11000652B010169830CD00401F76B000137EC0A
:10F1200023F048EC74F0010169936995699700D068
:10F13000000119EF7BF005010951F00B006E003A58
:10F140000F0E00160050000A00010FE0010A41E016
:10F15000030AD8B48DD0010AD8B4BFD0070AD8B4F6
:10F1600007D1010AD8B435D165D1050109510F0B7A
:10F17000090815E3010E0A5D036A0B25E96E0C51BF
:10F180000320EA6E300EEF6E036A0A510B25E96E1A
:10F190000C510320EA6E09513009EF6E19D0095164
:10F1A0000F0B0F0815E3010E0A5D036A0B25E96ECC
:10F1B0000C510320EA6E310EEF6E036A0A510B25E3
:10F1C000E96E0C510320EA6E0A0E095D3009EF6EFC
:10F1D00046D1050109510F0B030816E3010E0A5D24
:10F1E000036A0B25E96E0C510320EA6E310EEF6EB7
:10F1F000036A0A510B25E96E0C510320EA6E0A0ED0
:10F20000095D3009EF6E33D009510F0B0D0816E37D
:10F21000010E0A5D036A0B25E96E0C510320EA6EAC
:10F22000320EEF6E036A0A510B25E96E0C51032072
:10F23000EA6E140E095D3009EF6E19D009510F0BFB
:10F240000F0815E3010E0A5D036A0B25E96E0C51E8
:10F250000320EA6E330EEF6E036A0A510B25E96E46
:10F260000C510320EA6E1E0E095D3009EF6EF7D0D7
:10F27000050109510F0B070816E3010E0A5D036A29
:10F280000B25E96E0C510320EA6E330EEF6E036A14
:10F290000A510B25E96E0C510320EA6E1E0E095D22
:10F2A0003009EF6E19D009510F0B0F0815E3010E4D
:10F2B0000A5D036A0B25E96E0C510320EA6E340ED9
:10F2C000EF6E036A0A510B25E96E0C510320EA6EBA
:10F2D000280E095D3009EF6EC2D0050109510F0BF0
:10F2E000010816E3010E0A5D036A0B25E96E0C5155
:10F2F0000320EA6E340EEF6E036A0A510B25E96EA5
:10F300000C510320EA6E280E095D3009EF6E2FD0F4
:10F3100009510F0B0B0816E3010E0A5D036A0B255A
:10F32000E96E0C510320EA6E350EEF6E036A0A5146
:10F330000B25E96E0C510320EA6E320E095D30098F
:10F34000EF6E15D0010E0A5D036A0B25E96E0C51B4
:10F350000320EA6E360EEF6E036A0A510B25E96E42
:10F360000C510320EA6E3C0E095D3009EF6E77D038
:10F37000050109510F0B050816E3010E0A5D036A2A
:10F380000B25E96E0C510320EA6E360EEF6E036A10
:10F390000A510B25E96E0C510320EA6E3C0E095D03
:10F3A0003009EF6E15D0010E0A5D036A0B25E96E78
:10F3B0000C510320EA6E370EEF6E036A0A510B25DB
:10F3C000E96E0C510320EA6E460E095D3009EF6EBE
:10F3D00046D0050109510F0B090816E3010E0A5D1D
:10F3E000036A0B25E96E0C510320EA6E380EEF6EAE
:10F3F000036A0A510B25E96E0C510320EA6E500E88
:10F40000095D3009EF6E15D0010E0A5D036A0B2508
:10F41000E96E0C510320EA6E390EEF6E036A0A5151
:10F420000B25E96E0C510320EA6E5A0E095D300976
:10F43000EF6E15D0010E05010A5D036A0B25E96E1A
:10F440000C510320EA6E450EEF6E036A0A510B253C
:10F45000E96E0C510320EA6E450EEF6E00D00001FC
:10F46000000C040EEA6EE30EE96E0801E56BE76B33
:10F47000130EE66F00016BEC25F0040EEA6EF60E3B
:10F48000E96E0801E56BE76B130EE66F00016BECAC
:10F4900025F0036A0301C451C90FE96E030E03206E
:10F4A000EA6E0C01E26BEFCFE1FCE46B120EE36F4E
:10F4B000000158EC29F002C003F001505C0F016E0E
:10F4C000020E032201C009F503C00AF5040E08016B
:10F4D000D06FE30ECF6F03C0D2F801C0D1F8D46B68
:10F4E000120ED36F00017AEC25F00C0E0401E36FCD
:10F4F000040E0801D06FE30ECF6F000149EC21F03C
:10F50000050E0801E56F00013FEC20F0010169B52F
:10F510001ED00401E251120DF350036AD50F016EA3
:10F52000030E032201C009F503C00AF5040E080109
:10F53000D06FF60ECF6F03C0D2F801C0D1F8D46BF4
:10F54000120ED36F00017AEC25F045D0010169B7A6
:10F550001CD0040EEA6EF60EE96E200E0801E56F6F
:10F56000E76B090EE66F00016BEC25F0E2C409F5CC
:10F57000090E05010A6F040E0C6FF60E0B6F0001E9
:10F58000DADD0501006B27D00101040EEA6EF60EEC
:10F59000E96E200E0801E56FE76B090EE66F0001CA
:10F5A0006BEC25F0E2C409F5090E05010A6F040EA3
:10F5B0000C6FF60E0B6F0001BEDD730E0501016FBF
:10F5C000650E026F630E036F046BFFC400F52E0E11
:10F5D0000401FF6F05010A0E0401F66F3E0EF76F7E
:10F5E000040E0801D06FF60ECF6F000149EC21F038
:10F5F000000C010169A305D0000165EF74F020D073
:10F60000010169830301C451000A000107E0010AF6
:10F6100008E0030A08E0010A06E007D0D0EF74F022
:10F6200008D010D406D000D504D0010169930001A0
:10F6300000D0010169A305D065C4E2F4000111DF27
:10F64000010104012AEF87F004016751655D03E1C0
:10F65000010E6625656F65070301C4530AE1C951B0
:10F660000D0807E104016551030DF3CFE2F4E2C494
:10F67000BEFF65C4E2F40001F4DE50EF7BF0040E3F
:10F68000EA6EDF0EE96E0801E56BE76B030EE66FCD
:10F6900000016BEC25F0010169A304D00001D4D76F
:10F6A00001D10101036A0301C451C50FE96E030EC4
:10F6B0000320EA6EEF50000A000105E0010A31E084
:10F6C000030A4EE0EFD0036A0301C451C90FE96E8B
:10F6D000030E0320EA6E020EEF6E036AC451C50FDB
:10F6E000E96E030E0320EA6E010EEF6E036AC45149
:10F6F000C90FE96E030E0320EA6EEFCFE2F4036A4E
:10F70000C451C90FE96E030E0320EA6E010EEF2407
:10F710000401E36FE2C4F8F4F96F000168EC66F0ED
:10F72000C1D0036A0301C451C90FE96E030E03205F
:10F73000EA6EEF2A036AC451C50FE96E030E032077
:10F74000EA6E020EEF6E030E0401DF6FE06B040E33
:10F750000801D06FDF0ECF6F000149EC21F0A2D07D
:10F76000036A0301C451C90FE96E030E0320EA6E58
:10F77000EF2A036AC451C90FE96E030E0320EA6E33
:10F78000EFCFE2F4036AC451CD0FE96E030E0320FC
:10F79000EA6EEF500401E25D67E066E30301C453E3
:10F7A00024E1036AC451C50FE96E030E0320EA6E1B
:10F7B000EF6A036AC451C90F016E030E03220401EC
:10F7C00003C0E3F4036A0301C451D10FE96E030ED1
:10F7D0000320EA6EEFCFE4F40401E3C4EAFF01C0C2
:10F7E000E9FFE4C4EFFF23D00301036AC451C50F4E
:10F7F000E96E030E0320EA6E020EEF6E036AC45137
:10F80000C90F016E030E0322040103C0E3F4036A6F
:10F810000301C451D10FE96E030E0320EA6E010EFD
:10F82000EF240401E3C4EAFF01C0E9FFEF6E036ABD
:10F830000301C451D10FE96E030E0320EA6EEFCF2E
:10F84000E2F4036AC451D10FE96E030E0320EA6E9D
:10F85000010EEF240401E36FE2C4F8F4F96F000134
:10F8600068EC66F01ED00401036A0301C451C90F9D
:10F87000E96E030E0320EA6E010EEF5C0401E26FF5
:10F88000036A0301C451C90FE96E030E0320EA6E37
:10F89000EFCFE3F4E2C4F8F4E3C4F9F4000168EC58
:10F8A00066F000D081EF82F004016651655D03E1EE
:10F8B000010E675D656F652B0301C4530AE1C951F1
:10F8C0000D0807E104016551030DF3CFE2F4E2C432
:10F8D000BEFF65C4E2F40001C4DD80EF7CF0040EDD
:10F8E000EA6EDF0EE96E0801E56BE76B030EE66F6B
:10F8F00000016BEC25F0010169A304D00001D4D70D
:10F9000073D10101036A0301C451C50FE96E030EEF
:10F910000320EA6EEF500208D8A496D0036AC451BF
:10F92000C90FE96E030E0320EA6EEF52D8B48CD0F3
:10F93000036AC451C90FE96E030E0320EA6EEF0695
:10F94000C4534BE0036AC451C90FE96E030E032090
:10F95000EA6EEF5242E1036AC451C50FE96E030E2D
:10F960000320EA6E020EEF6E036AC451CD0FE96EFA
:10F97000030E0320EA6E010EEF5C0401E26F036ADE
:10F980000301C451CD0FE96E030E0320EA6EEFCFE1
:10F99000E3F4E2C4F8F4E3C4F9F4000168EC66F0BF
:10F9A000036A0301C451C90F016E030E032204014F
:10F9B00003C0E3F4036A0301C451CD0FE96E030EE3
:10F9C0000320EA6EEFCFE4F40401E3C4EAFF01C0D0
:10F9D000E9FFE4C4EFFF36D00301036AC451C90F45
:10F9E000E96E030E0320EA6EEF5216E1036AC4517A
:10F9F000C90FE96E030E0320EA6EEF2A036AC451B1
:10FA0000C50FE96E030E0320EA6EEF6A010E0401D2
:10FA1000DF6FE06B0ED00301036AC451C50FE96EBE
:10FA2000030E0320EA6E010EEF6E020E0401DF6F7B
:10FA3000E06B040E0801D06FDF0ECF6F000149ECC0
:10FA400021F00401D1D00301036AC451C90FE96E4A
:10FA5000030E0320EA6EEFCFE2F4036AC451D10F24
:10FA6000E96E030E0320EA6EEF500401E25DD8B4A4
:10FA70007AD0D8A078D0036A0301C451C90FE96EC7
:10FA8000030E0320EA6EEF06036AC451C90FE96E44
:10FA9000030E0320EA6EEF50010849E3036AC451E4
:10FAA000C90FE96E030E0320EA6EEF06C45311E19D
:10FAB000036AC451C50FE96E030E0320EA6EEF6AB4
:10FAC000036AC451C90FE96E030E0320EA6EEF6AA0
:10FAD00012D0036AC451C90FE96E030E0320EA6E07
:10FAE000010EEF6E036AC451C50FE96E030E0320C9
:10FAF000EA6E020EEF6E036AC451D10FE96E030E77
:10FB00000320EA6EEFCFE2F4036AC451D10FE96E2D
:10FB1000030E0320EA6E010EEF240401E36FE2C43A
:10FB2000F8F4F96F000168EC66F01BD00301036A7A
:10FB3000C451C90FE96E030E0320EA6EEFCFE2F461
:10FB4000036AC451C90FE96E030E0320EA6E010E69
:10FB5000EF240401E36FE2C4F8F4F96F000168ECEC
:10FB600066F042D00401036A0301C451C50FE96E77
:10FB7000030E0320EA6E020EEF6E036AC451CD0F2E
:10FB8000E96E030E0320EA6E010EEF5C0401E26FE2
:10FB9000036A0301C451CD0FE96E030E0320EA6E20
:10FBA000EFCFE3F4E2C4F8F4E3C4F9F4000168EC45
:10FBB00066F0036A0301C451C90F016E030E0322EC
:10FBC000040103C0E3F4036A0301C451CD0FE96EDD
:10FBD000030E0320EA6EEFCFE4F40401E3C4EAFF6E
:10FBE00001C0E9FFE4C4EFFF04012AEF87F004013C
:10FBF000CB6BCA2D1CD0CB6BC851F00B006E036AC7
:10FC00000050006E035005E1800E005C000109E029
:10FC10000401035005E1400E005C000105E0040111
:10FC200005D00401CB2B00010401CB2B2ED0020EFA
:10FC3000CB6FC851006EC951036E035005E1800EB1
:10FC4000005C000117E00401035005E1400E005C78
:10FC5000000113E00401800E035C04E10052000186
:10FC60000FE00401400E035C04E1005200010BE0D0
:10FC700004010BD00401CB2B00010401CB2B0001AC
:10FC80000401CB2B00010401CB2BCBC401F00001FC
:10FC9000000C0401C56BC691C6931B6AF2BE1B8E95
:10FCA000F29E440E0C01E86FE96B000168EC1AF05B
:10FCB0001BBEF28E02C0C4F401C0C3F4FF0E0401E7
:10FCC000C31BC41BC4C47CF4C3C47BF4A9A105D06A
:10FCD00078C47CF477C47BF478D1C351006EC451EE
:10FCE000036E035005E100520001D8B482D0040134
:10FCF000800E035C05E100520001D8B485D00401F8
:10FD0000400E035C05E100520001D8B47DD004012F
:10FD1000035006E1400E005C0001D8B475D0040128
:10FD2000035006E1800E005C0001D8B46DD00401E0
:10FD3000035006E1010E005C0001D8B4E6D00401D6
:10FD4000035006E1020E005C0001D8B4DED00401CD
:10FD5000035006E1040E005C0001D8B4D6D00401C3
:10FD6000035006E1080E005C0001D8B4CED00401B7
:10FD7000035006E1100E005C0001D8B4C6D00401A7
:10FD8000035006E1200E005C0001D8B4BED004018F
:10FD9000010E035C05E100520001D8B4B6D00401A5
:10FDA000020E035C05E100520001D8B4AED004019C
:10FDB000040E035C05E100520001D8B4A6D0040192
:10FDC000080E035C05E100520001D8B49ED0040186
:10FDD000100E035C05E100520001D8B496D0040176
:10FDE000200E035C05E100520001D8B48ED004015E
:10FDF0008ED05AB406D05AAE04D06051030801E246
:10FE0000478A5D905A9E8CD00401C6815ABE73D039
:10FE10005DB071D05AB46FD0C4C4C9F4C3C4C8F4BF
:10FE2000CA6B0001E4DE036A0150E30FE96E010EC4
:10FE30000320EA6EEF38006E0F0E001600500AE045
:10FE40005A8E606B030E0401C56FF28AD76AD66AB8
:10FE500051D000010101C4A14CD0C4C4C9F4C3C431
:10FE6000C8F40401CA6B0001C2DE01C0C7F4C4C4F7
:10FE7000C9F4C3C4C8F40401CA6B0001B8DE036A44
:10FE80000150E30FE96E010E0320EA6EEFCFC8F4D4
:10FE9000E80EF66E310EF76E000EF86E050E0801D4
:10FEA000E56F000169EC29F0C7C4E6F8370E0801D8
:10FEB000E76F000182EC29F0F00EF66E310EF76E5E
:10FEC000000EF86E090E0801E56F000169EC29F0DB
:10FED000C8C4E6F8370E0801E76F000182EC29F08C
:10FEE0000A0E9EA8FED7AD6E0D0E9EA8FED7AD6E73
:10FEF0000101040107D05D905A9E479A5AA402D08E
:10FF000046805A86C58B00010BD00401C6815D90E6
:10FF10005A9E479A5AA402D046805A86000100D0C1
:10FF20000401C6A105D0C5C47DF47D8F5D9A4DD076
:10FF300078C47CF477C47BF40101C4A147D00401E8
:10FF4000C35302E1C45341E0C6B33FD0C351FF0ADB
:10FF5000C76FC451FF0AC86F000EF66E320EF76EFF
:10FF6000000EF86E100E0801E56F000169EC29F033
:10FF7000C8C4E6F8370E0801E76F000182EC29F0EB
:10FF8000C7C4E6F8370E0801E76F000182EC29F0DC
:10FF9000200E9EA8FED7AD6EC4C4E6F8370E080149
:10FFA000E76F000182EC29F0C3C4E6F8370E0801C0
:10FFB000E76F000182EC29F00A0E9EA8FED7AD6E15
:10FFC0000D0E9EA8FED7AD6E04010101000119EFD0
:10FFD000ABF0EF5210E0EACF45F5E9CF44F5EF5032
:10FFE0009EA8FED7AD6E45C5EAFF44C5E9FFE92AE4
:08FFF000D8B4EA2AEED7000C98
:020000040001F9
:100000000401DA6BD96BDC6BDB6BDD6BDE91040E0C
:10001000EA6EC50EE96E0801E56BE76B140EE66F3C
:1000200000016BEC25F00101C4A168EF80F0040130
:10003000C3C4E9FFC4C4EAFFECCFE0F4ED52EFCF54
:10004000DFF4C3C4E9FFC4C4EAFFECCFE2F4ED522D
:10005000EFCFE1F4FF0EE11BE21B220EF66E310E34
:10006000F76E000EF86E0C0E0801E56F000169ECEA
:1000700029F0E0C4E6F8370E0801E76F000182ECD2
:1000800029F0DFC4E6F8370E0801E76F000182ECC3
:1000900029F0200E9EA84AEF80F0AD6EE2C4E6F88B
:1000A000370E0801E76F000182EC29F0E1C4E6F8A1
:1000B000370E0801E76F000182EC29F00A0E9EA8B6
:1000C0005FEF80F0AD6E0D0E9EA864EF80F0AD6E18
:1000D0000401C3C4E9FFC4C4EAFFECCF03F0ED524E
:1000E000EFCFD9F403C0DAF4C351E96EC451EA6E1C
:1000F000EF50006EE92AEF50E906036E0350D8A4D2
:1001000089EF80F0020E005C0001D8B430EF81F07E
:1001100004010350D8A494EF80F0040E005C0001A9
:10012000D8B4DEEF81F004010350D8A49FEF80F033
:10013000200E005C0001D8B4E1EF81F0040103500F
:10014000D8A4AAEF80F0400E005C0001D8B4E4EF20
:1001500081F004010350D8A4B5EF80F0800E005C5C
:100160000001D8B4E7EF81F00401010E035CD8A4CC
:10017000C0EF80F000520001D8B47AEF82F00401A1
:100180000350D8A4CBEF80F0080E005C0001D8B477
:100190007FEF82F004010350D8A4D6EF80F0100E58
:1001A000005C0001D8B484EF82F00401100E035CFF
:1001B000D8A4E1EF80F000520001D8B489EF82F0BA
:1001C0000401020E035CD8A4ECEF80F000520001A1
:1001D000D8B48EEF82F00401040E035CD8A4F7EFCC
:1001E00080F000520001D8B448EF83F00401080EFB
:1001F000035CD8A402EF81F000520001D8B401EFF3
:1002000084F004010350D8A40DEF81F0010E005CCE
:100210000001D8B486EF84F00401200E035CD8A45A
:1002200018EF81F000520001D8B43CEF85F00401D2
:10023000400E035CD8A423EF81F000520001D8B433
:10024000F4EF85F00401800E035CD8A42EEF81F05A
:1002500000520001D8B47CEF86F004012AEF87F049
:100260000101D351F00BD8B4DBEF81F0D351F00B87
:10027000D008D8B4C3EF81F05AB042EF81F05AA44D
:1002800050EF81F05A8AA0925AAC50EF81F0010EE3
:100290000801D36F00012AEC20F0010144EF81F046
:1002A0000401A9B97BEF81F0A989040EEA6EC50E9D
:1002B000E96E000E0001A2EC0EF00A000900F550F4
:1002C000EE6E0009D8A45EEF81F00101D391C4A3C2
:1002D00078EF81F0C153D8A478EF81F0380EF66E34
:1002E000310EF76E000EF86E0001B9EC2DF0010131
:1002F0009FEF81F00401A999040EEA6EC50EE96E24
:10030000000E0001B5EC0EF00A000900F550EE6E8B
:100310000009D8A485EF81F00101D381C4A39FEF28
:1003200081F0C153D8A49FEF81F0440EF66E310ED8
:10033000F76E000EF86E0001B9EC2DF001011B6A9A
:10034000F2BE1B8EF29E480E0C01F16F010EF26F91
:10035000A9C4F3FC0001F5EC1BF01BBEF28E040EE9
:100360000801A86FC50EA76F0001C3EC25F04880F7
:100370005AB0BEEF81F05AA4C0EF81F05A9AA08221
:10038000DBEF81F00101040EEA6EC50EE96E000E8E
:100390000001C8EC0EF00A000900F550EE6E0009ED
:1003A000D8A4CCEF81F0040E0801A86FC50EA76F8A
:1003B0000001C3EC25F004012AEF87F004012AEFC5
:1003C00087F004012AEF87F004012AEF87F0040187
:1003D000A9B15DEF82F0020EC325E96E000EC421C3
:1003E000EA6EEFCFDFF4000EDFBD010E000AD8A4E5
:1003F0003FEF82F01B6AF2BE1B8EF29E460E0C018E
:10040000E86FE96B000168EC1AF01BBEF28E02C0C7
:10041000DCF401C0DBF4010E0401DD6FDD51630883
:10042000D8A03FEF82F0DB51FF0ADF6FDC51FF0AFB
:10043000E06FDF518008D8A422EF82F0E053D8B4F7
:1004400024EF82F02AEF87F00A0E0801D36F000133
:100450002AEC20F01B6AF2BE1B8EF29E460E0C01A7
:10046000E86FE96B000168EC1AF01BBEF28E02C067
:10047000DCF401C0DBF40401DD2B0EEF82F001019E
:10048000C4A351EF82F0C153D8A451EF82F04E0EB5
:10049000F66E310EF76E000EF86E0001B9EC2DF01D
:1004A00001010401DF6B0001CDEC70F08E9097909C
:1004B00004012AEF87F078EF82F00101C4A36FEF07
:1004C00082F0C153D8A46FEF82F05C0EF66E310E4D
:1004D000F76E000EF86E0001B9EC2DF00101010E6F
:1004E0000401DF6F0001CDEC70F004012AEF87F00A
:1004F0002AEF87F0F9EF7AF004012AEF87F03FEF57
:100500007BF004012AEF87F06FEF7CF004012AEF03
:1005100087F08EEC74F004012AEF87F00101D351CB
:10052000F00BD8B445EF83F05AB09AEF82F05AA49A
:10053000A8EF82F05A8AA0925AACA8EF82F0010E7E
:100540000801D36F00012AEC20F001019CEF82F03A
:100550000401A9B7C3EF82F0140E05016C6F010E00
:100560006D6F000132EC50F00101D395036A020176
:100570001051E30F016E010E032201C0E9FF03C019
:10058000EAFFEF940401A9871B6AF2BE1B8EF29E5C
:10059000480E0C01F16F010EF26FA9C4F3FC0001CB
:1005A000F5EC1BF01BBEF28E040EEA6EC50EE96E72
:1005B000000EDBEC0EF00A000900F550EE6E0009AB
:1005C000D8A4DCEF82F0040E0801A86FC50EA76F57
:1005D0000001C3EC25F00101C4A3FDEF82F0C1537B
:1005E000D8A4FDEF82F0680EF66E310EF76E000EA5
:1005F000F86E0001B9EC2DF001010401DE9100015B
:100600009FEC5CF0160E05016C6F010E6D6F000122
:1006100032EC50F00401DEB13DEF83F01B6AF2BE14
:100620001B8EF29E460E0C01E86FE96B000168EC30
:100630001AF01BBEF28E02C0DCF401C0DBF4040130
:10064000DB51FF0ADF6FDC51FF0AE06FDF53D8A4F4
:100650002FEF83F0E0510208D8B432EF83F0DE814F
:100660003BEF83F0160E05016C6F010E6D6F0001FC
:1006700032EC50F004010BEF83F05AB043EF83F0FB
:100680005AA445EF83F05A9AA08204012AEF87F01A
:100690000101D351F00BD8B4FEEF83F05AB054EF00
:1006A00083F05AA462EF83F05A8AA0925AAC62EFA8
:1006B00083F0010E0801D36F00012AEC20F0010144
:1006C00056EF83F00401A9B77DEF83F0140E050106
:1006D0006C6F010E6D6F000132EC50F00101D3958B
:1006E000036A02011051E30F016E010E032201C0E3
:1006F000E9FF03C0EAFFEF940401A9871B6AF2BE79
:100700001B8EF29E480E0C01F16F010EF26FA9C410
:10071000F3FC0001F5EC1BF01BBEF28E040EEA6E3A
:10072000C50EE96E000EEEEC0EF00A000900F55061
:10073000EE6E0009D8A496EF83F0040E0801A86FAE
:10074000C50EA76F0001C3EC25F00101C4A3B7EFEC
:1007500083F0C153D8A4B7EF83F0760EF66E310E56
:10076000F76E000EF86E0001B9EC2DF001010001EA
:100770009FEC5CF0170E05016C6F010E6D6F0001B0
:1007800032EC50F00401DE91DEB1F6EF83F01B6A2B
:10079000F2BE1B8EF29E460E0C01E86FE96B000163
:1007A00068EC1AF01BBEF28E02C0DCF401C0DBF470
:1007B0000401DB51FF0ADF6FDC51FF0AE06FDF53FA
:1007C000D8A4E8EF83F0E0510408D8B4EBEF83F04D
:1007D000DE81F4EF83F0170E05016C6F010E6D6F73
:1007E000000132EC50F00401C4EF83F05AB0FCEF8A
:1007F00083F05AA4FEEF83F05A9AA08204012AEFF4
:1008000087F00101D351F00BD8B483EF84F05AB0D4
:100810000DEF84F05AA41BEF84F05A8AA0925AACD0
:100820001BEF84F0010E0801D36F00012AEC20F0C9
:1008300001010FEF84F00401A9A742EF84F0A9970A
:10084000040EEA6EC50EE96E000E000101EC0FF019
:100850000A000900F550EE6E0009D8A429EF84F0D3
:100860000101D385C4A33FEF84F0860EF66E310EEE
:10087000F76E000EF86E0001B9EC2DF0010162EF89
:1008800084F00401A987040EEA6EC50EE96E000E1D
:10089000000114EC0FF00A000900F550EE6E00099B
:1008A000D8A44CEF84F00101D395C4A362EF84F087
:1008B000960EF66E310EF76E000EF86E0001B9EC72
:1008C0002DF00101040E0801A86FC50EA76F0001ED
:1008D000C3EC25F01B6AF2BE1B8EF29E480E0C0183
:1008E000F16F010EF26FA9C4F3FC0001F5EC1BF0EF
:1008F0001BBEF28E48805AB081EF84F05AA483EF79
:1009000084F05A9AA08204012AEF87F00101D351A2
:10091000F00BD8B439EF85F05AB092EF84F05AA4B6
:10092000A0EF84F05A8AA0925AACA0EF84F0010E96
:100930000801D36F00012AEC20F0010194EF84F04C
:100940000401A9BDBBEF84F01D0E05016C6F010E03
:100950006D6F000132EC50F00101D397036A020180
:100960001051E30F016E010E032201C0E9FF03C025
:10097000EAFFEF960401A98D1B6AF2BE1B8EF29E60
:10098000480E0C01F16F010EF26FA9C4F3FC0001D7
:10099000F5EC1BF01BBEF28E040EEA6EC50EE96E7E
:1009A000000E27EC0FF00A000900F550EE6E00096A
:1009B000D8A4D4EF84F0040E0801A86FC50EA76F69
:1009C0000001C3EC25F00101C4A3F5EF84F0C1538D
:1009D000D8A4F5EF84F0A80EF66E310EF76E000E77
:1009E000F86E0001B9EC2DF001011F0E05016C6FCE
:1009F000010E6D6F000132EC50F00401DE91DEB1AA
:100A000029EF85F0420E006E002EFED700001B6A13
:100A1000F2BE1B8EF29E460E0C01E86FE96B0001E0
:100A200068EC1AF01BBEF28E02C0DCF401C0DBF4ED
:100A30000401DB51FF0ADF6FDC51FF0AE06FDF2D9D
:100A400026EF85F0E053D8B427EF85F0DE81FFEF85
:100A500084F0200E05016C6F010E6D6F000132EC09
:100A600050F05AB037EF85F05AA439EF85F05A9A12
:100A7000A08204012AEF87F00101D351F00BD8B412
:100A8000F1EF85F05AB048EF85F05AA456EF85F0A3
:100A90005A8AA0925AAC56EF85F0010E0801D36F26
:100AA00000012AEC20F001014AEF85F00401A9BD04
:100AB00071EF85F01D0E05016C6F010E6D6F000169
:100AC00032EC50F00101D397036A02011051E30F99
:100AD000016E010E032201C0E9FF03C0EAFFEF9699
:100AE0000401A98D1B6AF2BE1B8EF29E480E0C01FA
:100AF000F16F010EF26FA9C4F3FC0001F5EC1BF0DD
:100B00001BBEF28E040EEA6EC50EE96E000E3AECC4
:100B10000FF00A000900F550EE6E0009D8A48AEF24
:100B200085F0040E0801A86FC50EA76F0001C3EC85
:100B300025F00101C4A3ABEF85F0C153D8A4ABEFFE
:100B400085F0B60EF66E310EF76E000EF86E0001EF
:100B5000B9EC2DF001011E0E05016C6F010E6D6FD9
:100B6000000132EC50F00401DE91DEB1E1EF85F0DE
:100B7000420E006E002EFED700001B6AF2BE1B8ED6
:100B8000F29E460E0C01E86FE96B000168EC1AF06A
:100B90001BBEF28E02C0DCF401C0DBF40401DB51A9
:100BA000FF0ADF6FDC51FF0AE06FDF53D8A4DEEFEE
:100BB00085F0E0512008D8B4DFEF85F0DE81B5EF95
:100BC00085F0200E05016C6F010E6D6F000132EC97
:100BD00050F05AB0EFEF85F05AA4F1EF85F05A9A31
:100BE000A08204012AEF87F00101D351F00BD8B4A1
:100BF00079EF86F05AB000EF86F05AA40EEF86F037
:100C00005A8AA0925AAC0EEF86F0010E0801D36FFB
:100C100000012AEC20F0010102EF86F00401A9ADE9
:100C200028EF86F0A99D040EEA6EC50EE96E000E4F
:100C300000014DEC0FF00A000900F550EE6E0009BE
:100C4000D8A41CEF86F00101D3874AEF86F0040197
:100C5000A98D1B6AF2BE1B8EF29E480E0C01F16F2D
:100C6000010EF26FA9C4F3FC0001F5EC1BF01BBEF2
:100C7000F28E040EEA6EC50EE96E000E60EC0FF007
:100C80000A000900F550EE6E0009D8A441EF86F085
:100C90000101D3971B6AF2BE1B8EF29E480E0C0117
:100CA000F16F010EF26FA9C4F3FC0001F5EC1BF02B
:100CB0001BBEF28E040E0801A86FC50EA76F0001BF
:100CC000C3EC25F048800101C4A371EF86F0C40E87
:100CD000F66E310EF76E000EF86E0001B9EC2DF0D5
:100CE00001015AB077EF86F05AA479EF86F05A9A4C
:100CF000A08204012AEF87F00101D351F00BD8B490
:100D000027EF87F0D351F00BD008D8B40FEF87F05E
:100D10005AB08EEF86F05AA49CEF86F05A8AA092C1
:100D20005AAC9CEF86F0010E0801D36F00012AEC4B
:100D300020F0010190EF86F00401A9BBC7EF86F017
:100D4000A98B040EEA6EC50EE96E000E000173EC6D
:100D50000FF00A000900F550EE6E0009D8A4AAEFC2
:100D600086F00101D393C4A3C4EF86F0C153D8A485
:100D7000C4EF86F0D20EF66E310EF76E000EF86EEE
:100D80000001B9EC2DF00101EBEF86F00401A99B05
:100D9000040EEA6EC50EE96E000E000186EC0FF03F
:100DA0000A000900F550EE6E0009D8A4D1EF86F0D4
:100DB0000101D383C4A3EBEF86F0C153D8A4EBEFBA
:100DC00086F0DE0EF66E310EF76E000EF86E000144
:100DD000B9EC2DF00101040E0801A86FC50EA76F34
:100DE0000001C3EC25F01B6AF2BE1B8EF29E480E7A
:100DF0000C01F16F010EF26FA9C4F3FC0001F5ECD8
:100E00001BF01BBEF28E48805AB00AEF87F05AA43E
:100E10000CEF87F05A9AA08227EF87F00101040EA9
:100E2000EA6EC50EE96E000E000199EC0FF00A00A3
:100E30000900F550EE6E0009D8A418EF87F0040EF3
:100E40000801A86FC50EA76F0001C3EC25F00401CF
:100E50002AEF87F00001000C05010E6B106B0F6B81
:100E600025915DAE40EF87F00001ACEC2DF0320E25
:100E70000801D36F00012AEC20F0050131EF87F063
:100E800025B1C0EF87F0630E9EA844EF87F0AD6EEA
:100E90006E0E9EA849EF87F0AD6E0DC5ADF81F0E22
:100EA0000801AE6F000168EC30F0320E0801D36F1C
:100EB00000012AEC20F00501106B0F6B0001675355
:100EC000D8A481EF87F005010F2BD8B4102B105157
:100ED0000008D8B079EF87F0FF0AD8A475EF87F043
:100EE0000F51F408D8B079EF87F0000E016EC2EF11
:100EF00087F0020E0801D36F00012AEC20F05FEFAB
:100F000087F06753D8B4AFEF87F0050E0501276F60
:100F1000110E266F140E286F0001CEEC2DF0012C5F
:100F2000ADEF87F0050111516308D8A4ACEF87F04D
:100F300012516808D8A4ACEF87F013516E08D8A4FA
:100F4000ACEF87F00D513009145DD8A4ACEF87F0F9
:100F5000010E016EC2EF87F0000181EF87F00501FD
:100F60000E2B0E510208D8B0B7EF87F02581640E22
:100F70000801D36F00012AEC20F0050140EF87F053
:100F8000000E016E0001000C05010E6B106B0F6B63
:100F900025915DAED8EF87F00001ACEC2DF0320E5C
:100FA0000801D36F00012AEC20F00501C9EF87F09A
:100FB00025B148EF88F0630E9EA8DCEF87F0AD6E98
:100FC000630E9EA8E1EF87F0AD6E106B0F6B000112
:100FD0006753D8A40AEF88F005010F2BD8B4102B63
:100FE00010510008D8B002EF88F0FF0AD8A4FEEF35
:100FF00087F00F51F408D8B002EF88F0000E016EB0
:101000004AEF88F0020E0801D36F00012AEC20F0AD
:10101000E8EF87F06753D8B437EF88F0050E050185
:10102000276F110E266F140E286F0001CEEC2DF0E5
:10103000012C35EF88F0050111516308D8A434EF75
:1010400088F012516808D8A434EF88F00D513009A7
:10105000135DD8A434EF88F00001ACEC2DF0010E44
:10106000016E05014AEF88F000010AEF88F00501E2
:101070000E2B0E510208D8B03FEF88F02581320EBA
:101080000801D36F00012AEC20F00501D8EF87F0AA
:10109000000E016E0001000C0101C2A164EF88F096
:1010A00005010D510308D8A05DEF88F0010E0D5D1C
:1010B000016E8DEF88F061EF88F00DC501F08DEFC6
:1010C00088F08DEF88F00101C2A37CEF88F0050164
:1010D0000D510408D8A074EF88F0030E0D25016EA1
:1010E0008DEF88F079EF88F0050E0D5D016E8DEFC4
:1010F00088F08DEF88F00101C2A588EF88F0010E1D
:1011000005010D5D016E8DEF88F08DEF88F0010116
:10111000000E016E05018DEF88F00001000C050145
:101120000D510008D8B09CEF88F00D510608D8A0EA
:101130009CEF88F0C2EF88F00101C4A1C1EF88F0F4
:10114000EC0EF66E330EF76E000EF86E180E0801F8
:10115000E56F000169EC29F00DC5E6F8570E0801AE
:10116000E76F000182EC29F0070EF66E340EF76E81
:10117000000EF86E040E0801E56F000169EC29F01D
:10118000010105010001B8EF8FF005010F6B0D5152
:10119000010A0001D8B4E3EF88F0030AD8B4E8EFFD
:1011A00088F0010AD8B4EDEF88F0070AD8B4F2EF5E
:1011B00088F0010AD8B4F7EF88F0030AD8B4FCEF3E
:1011C00088F001EF89F0DF0E05010F6F06EF89F05F
:1011D000EF0E05010F6F06EF89F0F70E05010F6F97
:1011E00006EF89F0FB0E05010F6F06EF89F0FD0E8B
:1011F00005010F6F06EF89F0FE0E05010F6F06EF78
:1012000089F0FF0E05010F6F06EF89F00101C4B7E9
:101210000DEF89F0FF0E05010F1B05010E53D8A439
:1012200025EF89F01B6AF2BE1B8EF29E400E0C0168
:10123000F16F010EF26F0FC5F3FC0001F5EC1BF02E
:101240001BBEF28E3FEF89F005010101C4A92EEF0C
:1012500089F005010F9F30EF89F0010105010F8F23
:101260001B6AF2BE1B8EF29E400E0C01F16FF26BF8
:101270000FC5F3FC0001F5EC1BF01BBEF28E000C59
:101280000501106B106B10510108D8A0CEEF89F04A
:10129000640E0801D36F00012AEC20F00EC527F57B
:1012A0000DC526F50FC528F5CEEC2DF0012CB6EFB7
:1012B00089F005010DC5E9FF0EC5EAFFEF504508AD
:1012C000D8A47DEF89F0010E0D25E96E000E0E21E8
:1012D000EA6EEF506608D8A47DEF89F0020E0D2566
:1012E000E96E000E0E21EA6EEF506608D8A47DEF7D
:1012F00089F0010E016ED0EF89F000016753D8B478
:10130000B4EF89F00EC512F50DC511F50FC513F533
:1013100079EC2EF0012CB2EF89F005010DC5E9FF43
:101320000EC5EAFFEF504508D8A4B1EF89F0010ED1
:101330000D25E96E000E0E21EA6EEF506608D8A466
:10134000B1EF89F0020E0D25E96E000E0E21EA6E56
:10135000EF506608D8A4B1EF89F0010E016ED0EF0E
:1013600089F000017EEF89F04EEF89F00501102D24
:10137000CBEF89F0320E0801D36F00012AEC20F088
:10138000ACEC2DF0240EF66E3E0EF76E000EF86EED
:10139000B9EC2DF00501102B43EF89F0000E016E22
:1013A0000001A4EF90F00501116B106B126B136B31
:1013B0000EC5EAFF0DC5E9FF0801E56BE76B0FC538
:1013C000E6F800016BEC25F00501116B106B115173
:1013D0000308D8A008EF8AF0D8A4F4EF89F01051E0
:1013E000E708D8A008EF8AF0020E0801D36F0001C9
:1013F0002AEC20F06753D8B402EF8AF0050108EF19
:101400008AF000010501102BD8B4112BE7EF89F009
:1014100000016753D8A411EF8AF0000E016E40EF6F
:101420008BF00501126B5DAE38EF8BF0036A125141
:101430000D25016E0E51032201C014F503C015F5F0
:10144000000184EC2DF015C5EAFF14C5E9FF01C0C9
:10145000EFFF036A050112510D25E96E0E510320BD
:10146000EA6EEF500D08D8A41CEF8BF0000167075F
:1014700005010DC5E9FF0EC5EAFFEF504508D8A4E8
:101480005EEF8AF0010E0D25E96E000E0E21EA6E68
:10149000EF503008D8B458EF8AF0010E0D25E96EF0
:1014A000000E0E21EA6EEF503108D8A45EEF8AF0EC
:1014B000000E016E000140EF8BF005011351000A90
:1014C0000001D8B46EEF8AF0010AD8B498EF8AF020
:1014D000030AD8B4CDEF8AF005EF8BF00501125165
:1014E0000308D8B095EF8AF00DC5E9FF0EC5EAFFF5
:1014F000EF505408D8A495EF8AF0010E0D25E96E3F
:10150000000E0E21EA6EEF506B08D8A495EF8AF01A
:10151000020E0D25E96E000E0E21EA6EEF506508F1
:10152000D8A495EF8AF0010E136F000105EF8BF040
:10153000050112510308D8B0CAEF8AF00DC5E9FFC2
:101540000EC5EAFFEF504208D8A4CAEF8AF0010E98
:101550000D25E96E000E0E21EA6EEF507308D8A437
:10156000CAEF8AF0020E0D25E96E000E0E21EA6E1A
:10157000EF507908D8A4CAEF8AF0030E0D25E96E62
:10158000000E0E21EA6EEF503108D8A4CAEF8AF09F
:10159000020E136F000105EF8BF0050112510308D5
:1015A000D8B002EF8BF00DC5E9FF0EC5EAFFEF5092
:1015B0004208D8A402EF8BF0010E0D25E96E000E53
:1015C0000E21EA6EEF507308D8A402EF8BF0020EE2
:1015D0000D25E96E000E0E21EA6EEF507908D8A4B1
:1015E00002EF8BF0030E0D25E96E000E0E21EA6E60
:1015F000EF503008D8A402EF8BF0010E016E00010D
:1016000040EF8BF0000105EF8BF00501126B320EFD
:101610000801D36F00012AEC20F00EC5EAFF0DC5CA
:10162000E9FF0801E56BE76B0FC5E6F800016BEC1D
:1016300025F035EF8BF00501036A12510D25E96E97
:101640000E510320EA6EEF500A08D8B42FEF8BF04A
:10165000122B0F51125DD8A02FEF8BF0126B0A0ED8
:101660000801D36F00012AEC20F0050113EF8AF086
:101670000A0E0801D36F00012AEC20F0000E016E63
:1016800020EF91F005010D6B0D6B0D510108D8A0F5
:10169000C2EF8BF05DAE59EF8BF00001ACEC2DF09A
:1016A000320E0801D36F00012AEC20F005014AEF49
:1016B0008BF0650E9EA85AEF8BF0AD6E440E9EA87F
:1016C0005FEF8BF0AD6EC80E0801D36F00012AECFE
:1016D00020F0050E0501276F0E0E266F140E286FE1
:1016E0000001CEEC2DF0012CB8EF8BF005010E516E
:1016F0004508D8A4B8EF8BF00F514608D8A4B8EF2E
:101700008BF010514408D8A4B8EF8BF014510D0899
:10171000D8A49AEF8BF013510F0B0D6F12510F0BD2
:101720000A0DF3500D2711510F0B640DF3500D27C7
:10173000B4EF8BF013510D08D8A4A9EF8BF0125120
:101740000F0B0D6F11510F0B0A0DF3500D27B4EF56
:101750008BF012510D08D8A4B3EF8BF011510F0B81
:101760000D6FB4EF8BF00D6B0DC501F0C4EF8BF076
:10177000320E0801D36F00012AEC20F005010D2B79
:1017800045EF8BF0000E016E0001000C016A026A49
:10179000006A036A05011051D8A4D3EF8BF00F51F2
:1017A000D8B4F0EF8BF0100E116FD8900D370E37C4
:1017B000003603361051035CD8A4E1EF8BF00F51D3
:1017C000005CD8A0EBEF8BF00F51005ED8A00306B1
:1017D0001051035ED88001360236112FD5EF8BF001
:1017E0000001000C05010D6B0F6B0E6B24915DAEBB
:1017F00006EF8CF00001ACEC2DF0320E0801D36F37
:1018000000012AEC20F00501F7EF8BF024B17FEF07
:101810008CF0470E9EA80AEF8CF0AD6E310E9EA89C
:101820000FEF8CF0AD6E0F6B0E6B00016753D8A4F9
:1018300038EF8CF005010E2BD8B40F2B0F51000898
:10184000D8B030EF8CF0FF0AD8A42CEF8CF00E51FA
:10185000F408D8B030EF8CF0000E016E81EF8CF000
:10186000020E0801D36F00012AEC20F016EF8CF075
:101870006753D8B46EEF8CF0050E0501276F100E7C
:10188000266F140E286F0001CEEC2DF0012C6CEFAA
:101890008CF0050110515408D8A46BEF8CF0115155
:1018A0004108D8A46BEF8CF012514B08D8A46BEF11
:1018B0008CF013514508D8A46BEF8CF0145131080B
:1018C000D8A46BEF8CF00001ACEC2DF0010E016E92
:1018D000050181EF8CF0000138EF8CF005010D2B34
:1018E0000D510208D8B076EF8CF02481320E080139
:1018F000D36F00012AEC20F0050106EF8CF0000EFA
:10190000016E0001B4EF91F005010E6B106B0F6BCF
:1019100025915DAE98EF8CF00001ACEC2DF0320E0D
:101920000801D36F00012AEC20F0050189EF8CF04B
:1019300025B108EF8DF0430E9EA89CEF8CF0AD6EA4
:10194000430E9EA8A1EF8CF0AD6E106B0F6B0001E3
:101950006753D8A4CAEF8CF005010F2BD8B4102B15
:1019600010510008D8B0C2EF8CF0FF0AD8A4BEEF27
:101970008CF00F51F408D8B0C2EF8CF0000E016E5D
:101980000AEF8DF0020E0801D36F00012AEC20F05F
:10199000A8EF8CF06753D8B4F7EF8CF0050E050173
:1019A000276F110E266F140E286F0001CEEC2DF05C
:1019B000012CF5EF8CF0050111514308D8A4F4EF88
:1019C0008CF012514808D8A4F4EF8CF00D51300976
:1019D000135DD8A4F4EF8CF00001ACEC2DF0010EF7
:1019E000016E05010AEF8DF00001CAEF8CF00501D0
:1019F0000E2B0E510208D8B0FFEF8CF02581320E6D
:101A00000801D36F00012AEC20F0050198EF8CF05B
:101A1000000E016E0001CCEF91F005010D510008A0
:101A2000D8B01AEF8DF00D510608D8A01AEF8DF03E
:101A300040EF8DF00101C4A13FEF8DF0CE0EF66EA8
:101A4000330EF76E000EF86E150E0801E56F0001FB
:101A500069EC29F00DC5E6F8570E0801E76F0001A3
:101A600082EC29F0E60EF66E330EF76E000EF86E7D
:101A7000040E0801E56F000169EC29F00101050180
:101A8000000140EF93F0780E0401A9130101D3A5E2
:101A90004DEF8DF00401A9970101D3A153EF8DF013
:101AA0000401A9990101D3A359EF8DF00401A99B69
:101AB0000101D3A75FEF8DF00401A99D01011B6A0D
:101AC000F2BE1B8EF29E480E0C01F16F010EF26FFA
:101AD000A9C4F3FC0001F5EC1BF01BBEF28E000C58
:101AE0000401C66BC56B020EC76FDC6BDD6BDE6B72
:101AF000DF6BE16BE06BE29105010B6B0C6B040E8D
:101B0000EA6EC80EE96E0801E56BE76B140EE66F2E
:101B100000016BEC25F00101C4A1E1EF8DF004019F
:101B2000C3C4E9FFC4C4EAFFECCF0EF5ED52EFCF1A
:101B30000DF5C3C4E9FFC4C4EAFFECCF10F5ED52C4
:101B4000EFCF0FF5FF0E05010F1B101BCC0EF66E2D
:101B50002E0EF76E000EF86E0C0E0801E56F0001F8
:101B600069EC29F00EC5E6F8370E0801E76F0001B1
:101B700082EC29F00DC5E6F8370E0801E76F000189
:101B800082EC29F0200E9EA8C3EF8DF0AD6E10C53B
:101B9000E6F8370E0801E76F000182EC29F00FC567
:101BA000E6F8370E0801E76F000182EC29F00A0E13
:101BB0009EA8D8EF8DF0AD6E0D0E9EA8DDEF8DF0D6
:101BC000AD6E0401C3C4E9FFC4C4EAFFECCF03F067
:101BD000ED52EFCFC5F403C0C6F4C551006EC65137
:101BE000036E200E035CD8A4FCEF8DF000520001C0
:101BF000D8B4A3EF8EF00401100E035CD8A407EF55
:101C00008EF000520001D8B4A6EF8EF00401080E49
:101C1000035CD8A412EF8EF000520001D8B4A9EFF3
:101C20008EF00401040E035CD8A41DEF8EF0005268
:101C30000001D8B4ACEF8EF00401020E035CD8A40E
:101C400028EF8EF000520001D8B4AFEF8EF00401FF
:101C5000010E035CD8A433EF8EF000520001D8B41B
:101C6000B2EF8EF004010350D8A43EEF8EF0200EA8
:101C7000005C0001D8B42AEF90F004010350D8A40E
:101C800049EF8EF0100E005C0001D8B42DEF90F0FB
:101C900004010350D8A454EF8EF0080E005C00013C
:101CA000D8B430EF90F004010350D8A45FEF8EF069
:101CB000040E005C0001D8B433EF90F0040103502F
:101CC000D8A46AEF8EF0020E005C0001D8B436EFA3
:101CD00090F004010350D8A475EF8EF0010E005C63
:101CE0000001D8B439EF90F004010350D8A480EF7C
:101CF0008EF0800E005C0001D8B4B1EF93F00401C7
:101D00000350D8A48BEF8EF0400E005C0001D8B4D5
:101D1000B4EF93F00401800E035CD8A496EF8EF02C
:101D200000520001D8B4B7EF93F00401400E035CF9
:101D3000D8A4A1EF8EF000520001D8B4BAEF93F00E
:101D4000040166EF95F00401DC2B00010401DC2B9B
:101D500000010401DC2B00010401DC2B0001040163
:101D6000DC2B00010401DC2B0101C151000A000140
:101D7000D8B4D1EF8EF0010AD8B4D3EF8EF0030AB5
:101D8000D8B4F0EF8EF0060AD8B400EF8FF00C0A4A
:101D9000D8B42AEF8FF0180AD8B473EF8FF073EF2E
:101DA0008FF096EF8FF0ACEC2DF0320E9EA8D6EFB0
:101DB0008EF0AD6E2A0E9EA8DBEF8EF0AD6EDCC409
:101DC000ADF81F0E0801AE6F000168EC30F0210E77
:101DD0009EA8E8EF8EF0AD6EACEC2DF096EF8FF094
:101DE000DCC40DF52CEC87F0DCC40DF5C4EC87F0F9
:101DF0000152D8A4FEEF8EF066EF95F096EF8FF0CB
:101E0000DCC40DF54CEC88F001C00BF5ACEC2DF00A
:101E1000020E9EA809EF8FF0AD6EE40EF66E2E0E48
:101E2000F76E000EF86E040E0801E56F000169EC14
:101E300029F00BC5ADF81F0E0801AE6F000168EC6C
:101E400030F03B0E9EA822EF8FF0AD6EACEC2DF083
:101E500096EF8FF0ACEC2DF0580E9EA82DEF8FF082
:101E6000AD6E310E9EA832EF8FF0AD6E2C0E9EA897
:101E700037EF8FF0AD6EDCC4ADF81F0E0801AE6F0A
:101E8000000168EC30F00D0E9EA844EF8FF0AD6EAF
:101E9000ACEC2DF00401E16BCDC1E0F4E1C4E2FC57
:101EA000E0C4E1FC0C01E46B640EE36F000158EC4C
:101EB00029F002C0E1F401C0E0F4E1C40DF5050130
:101EC0000D2B0D07D8B408D0FF0E0801D36F000109
:101ED0002AEC20F00501F5D7E0C4D3F800012AEC84
:101EE00020F096EF8FF0430E9EA874EF8FF0AD6E4A
:101EF000480E9EA879EF8FF0AD6E410E9EA87EEF42
:101F00008FF0AD6EDCC4ADF81F0E0801AE6F00019E
:101F100068EC30F00A0E9EA88BEF8FF0AD6E0D0EC0
:101F20009EA890EF8FF0AD6E96EF8FF03F0E0401FC
:101F3000AB13C551FF0A006EC651FF0A036E005075
:101F4000AA170350AB171B6AF2BE1B8EF29E4A0EF5
:101F50000C01EA6FEB6BABC4EDFCAAC4ECFC000116
:101F600021EC1CF01BBEF28EDCC40DF58FEF88F067
:101F7000DCC40EF2040EEA6EC80EE96E000E5FECD1
:101F80000DF00A000900F550EE6E0009D8A4C2EF6A
:101F90008FF00401DC513009D56F5DBA04EF90F089
:101FA000040E0801A86FC80EA76F0001C3EC25F04E
:101FB0000101C4A304EF90F0C153D8A404EF90F042
:101FC000EC0EF66E2E0EF76E000EF86E050E080182
:101FD000E56F000169EC29F0DCC4ADF81F0E0801C3
:101FE000AE6F000168EC30F00A0E9EA8F5EF8FF09E
:101FF000AD6E0D0E9EA8FAEF8FF0AD6E3E0E9EA850
:10200000FFEF8FF0AD6E01010101C5AB1FEF90F046
:10201000036A0401DC51E30FE96E010E0320EA6E4E
:10202000EF50F00BD8B41FEF90F0DC510201105DBF
:10203000D8B41EEF90F0DCC416F24C8004010EC23E
:102040000DF5010E05010E6F0001C5EC88F00401CD
:1020500066EF95F00401DD2B00010401DD2B00018A
:102060000401DD2B00010401DD2B00010401DD2B47
:1020700000010401DD2B0EC2DEF40101C151000A92
:102080000001D8B45AEF90F0010AD8B45CEF90F098
:10209000030AD8B453EF91F0060AD8B4DCEF91F0FC
:1020A0000C0AD8B4A0EF92F0180AD8B4E9EF92F075
:1020B000E9EF92F00CEF93F00401E2810001ACEC47
:1020C0002DF0320E9EA862EF90F0AD6E2A0E9EA803
:1020D00067EF90F0AD6EDDC4ADF81F0E0801AE6F76
:1020E000000168EC30F0210E9EA874EF90F0AD6E08
:1020F000020E05010D6FFA0E0801D36F00012AECE4
:1021000020F005010D2FF7D7040E276FE30E266F81
:10211000280E286F0001CEEC2DF0012C49EF91F034
:10212000ACEC2DF0F80EF66E2E0EF76E000EF86E7B
:10213000B9EC2DF0040E05010E6FE30E0D6F280EA5
:102140000F6F000140EF89F0012C49EF91F004017D
:10215000EA510F0B05010D6F0401E9510F0B0A0D38
:10216000F35005010D250401E06FE16BE0C4CDF1F2
:10217000E6C40CF505010C513208D8B0C4EF90F05C
:10218000320E0C6FCBEF90F00C512F08D8A0CBEF94
:1021900090F0300E0C6F0001ACEC2DF0310E9EA8CB
:1021A000CFEF90F0AD6E2A0E9EA8D4EF90F0AD6EFA
:1021B000300E9EA8D9EF90F0AD6E05010C519EA88F
:1021C000DFEF90F0AD6E250E9EA8E4EF90F0AD6EBF
:1021D000E1C4E2FCE0C4E1FC0C01E46B640EE36FDB
:1021E000000158EC29F002C0E1F401C0E0F4E1C4C0
:1021F0000DF505010D2B0D07D8B408D0FF0E080111
:10220000D36F00012AEC20F00501F5D7E0C4D3F824
:1022100000012AEC20F0020E05010D6FFA0E0801F4
:10222000D36F00012AEC20F005010D2FF7D7040E23
:102230000E6FE30E0D6F280E0F6F0001D3EF89F0C4
:10224000012C49EF91F0ACEC2DF0320E9EA826EF58
:1022500091F0AD6E2A0E9EA82BEF91F0AD6EDEC40C
:10226000ADF81F0E0801AE6F000168EC30F0210ED2
:102270009EA838EF91F0AD6E040E0501276FE30EB6
:10228000266F280E286F0001CEEC2DF00401E2919C
:1022900000010401E2A150EF91F0000166EF95F01A
:1022A00000010CEF93F042EC8BF001C00CF5DDC4A3
:1022B0000DF52CEC87F0DDC40DF5C4EC87F0012C96
:1022C000DAEF91F005010C53D8A46DEF91F0000105
:1022D00042EC8BF001C00CF505010C53D8B4ACEF07
:1022E00091F00E6B0CC50DF5106B0A0E0F6F00010F
:1022F000C6EC8BF002C00EF501C00DF502C0E2FC89
:1023000001C0E1FC030E0C01E46FE80EE36F000175
